:1000000000800020BD010000C58900007D8900003E
:100010007D8900007D8900007D8900007D890000C8
:100020007D8900007D8900007D890000C589000070
:10003000C58900007D890000718100007582000083
:10004000C5890000C5890000C5890000C589000078
:10005000C5890000C5890000C5890000C589000068
:10006000C5890000C5890000C5890000C589000058
:10007000C5890000C5890000C5890000C589000048
:10008000C5890000C5890000C5890000C589000038
:10009000C5890000C5890000C5890000C589000028
:1000A0007565000081650000C5890000C5890000F4
:1000B000C5890000C5890000C5890000C589000008
:1000C000C5890000C5890000C5890000C5890000F8
:1000D000C5890000C5890000C5890000C5890000E8
:1000E000C5890000C5890000C5890000C5890000D8
:1000F000C589000065A90000C589000091AA00001B
:10010000C58900009D930000C5890000C5890000D5
:10011000C5890000C5890000C5890000C5890000A7
:10012000C5890000C5890000C5890000C589000097
:10013000C5890000C5890000C5890000C589000087
:10014000C5890000C5890000C5890000C589000077
:10015000C5890000C5890000C5890000C589000067
:10016000C5890000B9960000C5890000C589000056
:10017000C5890000C5890000C5890000C589000047
:10018000C5890000C5890000C5890000C589000037
:10019000C5890000C5890000C5890000C589000027
:1001A000C5890000C5890000C5890000C589000017
:1001B000C5890000C5890000C5890000564B4CF276
:1001C000205210B51A804DF628121A8000BF00BFC9
:1001D00008F0FCFB514B4FF010621A60504A9A60D5
:1001E000504ADA60504A136813F4807304D14F49BF
:1001F0000B604FF4A85313604D4B1A78110703D5C9
:100200001A7842F008021A704A4B4B492A221A7097
:100210004A4A4B4B8B4204D252F8040F43F8040B6A
:10022000F8E7484B484900228B4202D243F8042B9E
:10023000FAE74649464A002352F8230041F82300D2
:1002400001336F2BF8D1434B434A802103F8011B44
:100250009342FBD1414B3D4A1A60414B8A221A70AE
:10026000A3F5805324225A70A0221A709A7992071B
:10027000FCD59A79D406FCD43A4A937903F00C035E
:10028000082B384BF9D103221A7140225A719A79FE
:100290009006FCD5334A9179324B4906FBD5324A58
:1002A000324911600221516020221A709A7902F0BD
:1002B0000C020C2AFAD12E4B2E4A1A602E4B2F4AD2
:1002C0001A6000225A60072243F8042C2C4AC3F813
:1002D0000C2D62B608F02AFF144B1B68DA0705D50F
:1002E000284808F0F7FC284B284A1A60284B1B784E
:1002F0005B0609D5244C254B22689A4204D121483B
:1003000008F0E8FC002323600BF07AFE08F064FBA1
:1003100008F092FAFEE700BF0E200540308004404E
:10032000823F04000100002B10D0034014D0034092
:1003300002D0074000E007401C99FF1F40E5000085
:100340004088FF1F1C99FF1FC09FFF1F0082FF1FD7
:100350000000000000E400E05FE400E008ED00E0E1
:100360000050064000400640448004400000030165
:1003700004800440C010050014E000E0FF76010096
:1003800000002020D26E385D1CE00340A5C3945AC3
:1003900000F00740FFFFFFFFFFFFFFFFFFFFFFFF32
:1003A000FFFFFFFFFFFFFFFFFFFFFFFFFFFFFFFF5D
:1003B000FFFFFFFFFFFFFFFFFFFFFFFFFFFFFFFF4D
:1003C000FFFFFFFFFFFFFFFFFFFFFFFFFFFFFFFF3D
:1003D000FFFFFFFFFFFFFFFFFFFFFFFFFFFFFFFF2D
:1003E000FFFFFFFFFFFFFFFFFFFFFFFFFFFFFFFF1D
:1003F000FFFFFFFFFFFFFFFFFFFFFFFFFFFFFFFF0D
:10040000FFFFFFFFFFFFFFFFFFFFFFFFDEF9FFFF23
:1004100010B5054C237833B9044B13B10448AFF33E
:1004200000800123237010BD1C99FF1F00000000F5
:1004300044E50000084B10B51BB108490848AFF36C
:1004400000800848036803B910BD074B002BFBD0A0
:10045000BDE81040184700BF000000002099FF1FB2
:1004600044E500001C99FF1F0000000070B44C8898
:10047000A04220D901230133DBB21CB2660031F85F
:10048000144084421D46F6D3A04211D005F1004528
:10049000013D965B31F8151032F81530401AF21A0A
:1004A00000FB02F0641A90FBF4F4E01870BC704793
:1004B000905B70BC704702260125E5E700280CDA46
:1004C000064A434282FB0320DA17C2EB600000EBCE
:1004D0004000A3EB8000C0F10C007047ABAAAA2A31
:1004E0002DE9F84F0C2008F04DF80C2008F002FD23
:1004F000E049142008F00EFD0221032008F0A0FDC1
:100500000221042008F09CFD0221052008F098FD3E
:100510000221062008F094FD01210A2008F090FD38
:100520000121092008F08CFD01210D2008F088FD33
:100530000121282008F084FD0121142008F080FD0D
:1005400002210B2008F07CFD01210C2008F078FD31
:1005500000210C2008F060FD002004F053FA172859
:10056000044600F258822021002004F02DF84FF4B8
:10057000AF61022004F028F804204FF47A6104F0FF
:1005800023F80B2008F04EFD002800F0398240F6D9
:100590002821062004F018F840F6E441082004F071
:1005A00013F84FF4AF610A2004F00EF840F6FC0196
:1005B0000C2004F009F84FF49661222004F004F8AE
:1005C0004FF41661242003F0FFFF7D212A2003F061
:1005D000FBFF202C00F007822021002003F0F4FF15
:1005E0000C210E2003F0F0FF0121102003F0ECFF9E
:1005F0000221122003F0E8FF0021142003F0E4FFA1
:100600000021162003F0E0FF0221182003F0DCFF98
:1006100001211A2003F0D8FF02211C2003F0D4FF8F
:1006200004211E2003F0D0FF1421202003F0CCFF72
:100630000121262003F0C8FF0321282003F0C4FF76
:1006400004212C2003F0C0FF0F212E2003F0BCFF5B
:100650000021302003F0B8FF0C21322003F0B4FF5A
:100660000021342003F0B0FF0021362003F0ACFF5E
:100670000021382003F0A8FF00213A2003F0A4FF56
:1006800000213C2003F0A0FF00213E2003F09CFF4E
:100690000021402003F098FF0021422003F094FF46
:1006A0001F21442003F090FF1321462003F08CFF0C
:1006B0000E21482003F088FF11214A2003F084FF17
:1006C0000A214C2003F080FF00214E2003F07CFF24
:1006D0000621502003F078FF0221522003F074FF1E
:1006E0000C21542003F070FF0021562003F06CFF12
:1006F0000021582003F068FF01215A2003F064FF15
:1007000003215C2003F060FF0A215E2003F05CFF00
:100710000021602003F058FF022004F073F9564BCB
:10072000564C1880042004F06DF9554BDFF8B4A145
:100730001880062004F066F9524B534D18800820AB
:1007400004F060F9514BDFF8A09118800A2004F002
:1007500059F94F4BDFF894B118800C2004F052F98E
:100760004C4B4D4F18800E2004F04CF94B4B4C4E27
:100770001880102004F046F94A4BDFF87481188085
:10078000122004F03FF9484B1880142004F03AF985
:10079000464B1880162004F035F9454B1880182078
:1007A00004F030F9434B18801A2004F02BF9424B27
:1007B00018801C2004F026F9404B18801E2004F0FD
:1007C00021F93F4B1880202004F01CF93D4B188084
:1007D000222004F017F93C4B1880242004F012F971
:1007E0003A4B1880262004F00DF92080282004F0D0
:1007F00009F9374B18802A2004F004F9AAF8000000
:100800002C2004F0FFF8334B18802E2004F0FAF867
:10081000314B1880302004F0F5F8304B188032202E
:1008200004F0F0F82E4B1880342004F0EBF8288008
:10083000362004F0E7F86880382004F0E3F8A88058
:100840003A2004F0DFF8E8803C2004F0DBF828814F
:100850003E2004F0D7F86881402004F0D3F8A88146
:10086000422004F0CFF8A9F80000442004F0CAF8B0
:1008700040E000BF001B3746B699FF1F8299FF1F5B
:10088000929AFF1F449AFF1F5499FF1F2E9AFF1F31
:100890005C9AFF1F109AFF1F6A89FF1F8099FF1F34
:1008A0007089FF1FB899FF1F6299FF1F209AFF1FD1
:1008B0004099FF1FEC99FF1F329AFF1F589AFF1FA4
:1008C000FA99FF1F909AFF1F5E9AFF1FEE99FF1F74
:1008D000E499FF1F1A9AFF1F249AFF1F5099FF1FC8
:1008E000889AFF1F189AFF1FAE99FF1F509AFF1F8B
:1008F0006C89FF1FA94BAA4D1880462004F082F88E
:10090000ABF80000482004F07DF8ABF802004A2064
:1009100004F078F8ABF804004C2004F073F8ABF85E
:1009200006004E2004F06EF89E4B1880502004F014
:1009300069F89D4B1880522004F064F89B4B188096
:10094000542004F05FF83880562004F05BF8984B90
:100950001880582004F056F8964B18805A2004F05E
:1009600051F8954B18805C2004F04CF8934B18809C
:100970005E2004F047F83080602004F043F8BAF8B5
:10098000003021882970A3F5AF7E8D498D4CB9F8D0
:100990000020208040F23A7303FB0EF381FB03E159
:1009A000DB17A3EB6113884C8848DFF858C28849ED
:1009B0003233C8F8003002F00203238002F004034F
:1009C000038002F008038CF80030824C824802F069
:1009D000100C02F02003A1F800C05A21238005F07A
:1009E00079FE18BBFEE7042008F01CFB00287FF40A
:1009F00093AE062008F016FB00283FF4EDAD8BE621
:100A00004FF49661062003F0DFFD4FF4FA610820F1
:100A100003F0DAFDC5E5042008F004FB002859D0F6
:100A20004FF6FF739C427FF4D4AD9CE56B4A6C4853
:100A30001268DFF8D4B10023012105F023FF03F091
:100A40007BFD0B2008F0EEFA011E0CBF01230023F2
:100A50008BF8003002D1112008F0F2FADFF888910B
:100A6000604CDFF8A8810023C9F800302360C8F883
:100A700000304FF0010A11E007F0B8FD2368184478
:100A800020600AF001010D2008F0C6FA0AF1010AFF
:100A9000FA2008F0FDFABAF1050F22D00F2008F075
:100AA000E9FCD8F8003003440E20C8F8003007F005
:100AB0009DFDD9F800309BF800100344C9F80030C0
:100AC00015200029D8D1112008F0D4FC236818443F
:100AD0002060D6E7062008F0A5FA00283FF443ADD1
:100AE0009EE7D8F80030D9F800103F4A2068DFF8B8
:100AF00020E13688DFF81CC1002BB8BF0333002982
:100B0000B8BF0331891011603988384F9B10002815
:100B1000A3EB0102B8BF033019448010CEF80020C7
:100B20003960DFF8F4E0324FC8F800308219C6EBC4
:100B30000008002120600D203B60CCF80080CEF83A
:100B4000002008F069FAFA2008F0A2FA01210D202D
:100B500008F062FAFA2008F09BFA00210D2008F054
:100B60005BFA04F0D7F940F2DC5008F091FA214B1F
:100B7000012604201E6008F055FA10B91E4B28709B
:100B80001E701E4B1E4A1B781370184605F0D8F8CD
:100B900001210D20BDE8F84F08F03EBA609AFF1F12
:100BA000759AFF1F7E99FF1F6489FF1FA889FF1F89
:100BB0008E9AFF1F2C9AFF1F7099FF1F6689FF1FD7
:100BC000B5814E1BB299FF1F5A9AFF1FDC99FF1F78
:100BD000089AFF1F4C9AFF1F389AFF1F7489FF1F46
:100BE000BC99FF1F9C99FF1F0C9AFF1F709AFF1F53
:100BF000009AFF1F7499FF1FE699FF1FB899FF1F06
:100C0000309AFF1F749AFF1F849AFF1F8899FF1F55
:100C10001C9AFF1FF099FF1F409AFF1FF0B40E8827
:100C200086420DD203F10043013B31F81350854257
:100C300002D9F0BCFFF71ABC32F81300F0BC7047C1
:100C40001088F0BC704700BF094B1B880C2B09D8DB
:100C5000084A80B252F8232028B143F6FE73984226
:100C600003D9108C7047108870470349FFF7FEBB0B
:100C70001A9AFF1FC4CC0000A4CB000008B5214A7B
:100C8000214B12881868824234DA204B1B88991A4B
:100C90008342A8BF0346B1F5F87FA3EB020321DA34
:100CA000C3EB031303EB431393FBF1F105310A206C
:100CB00008F022F8164B1978F1B1164B16491B684B
:100CC00083F30703C3EB031303EB431381FB0321FC
:100CD0001944DB17C3EBA11105310920BDE8084019
:100CE00008F00AB8C3EB43131B01013193FBF1F188
:100CF0000531DCE70021DAE70920BDE8084007F00C
:100D0000FBBF00BFB699FF1F149AFF1F929AFF1FE7
:100D1000629AFF1F349AFF1F09040281374A38493B
:100D20001088384AF8B5384B12881B68834248DB74
:100D30009342A8BF134698420B60C8BF002342DD10
:100D4000101AB0F5804FAABF9B03C3EB8333013069
:100D500093FBF0F0FFF778FF2C4B2D4F1C883B687E
:100D6000C0F3C61505FB04F47F2CA8BF7F249D4269
:100D7000064608D0274B1B88002B38D1264B1B88F2
:100D8000002B30D13D60254D2B689E4205D0214B74
:100D90001B885A1F032A1DD92E60214D2B689C42A7
:100DA0000ED0204B188848B11A4B1F4A1B88D35CC1
:100DB000834203D0C0B2E1B204F00AFF2C60F8BD58
:100DC000F8BD034608609A42D4BFC0EB0203C0EBF3
:100DD0000303B5E7144AD05C2030C0B206F07F01AF
:100DE00004F0F6FED8E7284604F066FFCAE70E4A8C
:100DF0002946D05C04F0ECFEC0E700BFB699FF1FA7
:100E0000149AFF1F929AFF1F6499FF1F7099FF1F8A
:100E10004499FF1F6299FF1F209AFF1F6C99FF1FC3
:100E20003C99FF1F2C9AFF1F7889FF1F2DE9F04F77
:100E3000172087B008F01EFBA34B1860162008F09F
:100E400019FBA24BA24A1B8810600C2B00F07D837B
:100E5000DFF8C0A29F4ABAF800109F4B52F8214019
:100E600000221A709D4B9E4A1B889E491288013BA6
:100E700031F91350002A00F0A7809B4B1B78002B00
:100E800049D1112008F0F6FA984B0193D3F800905D
:100E90000746B94549DD964B964E1B88012B00F05D
:100EA000CD82954B03933068944B00930AF036FE45
:100EB0004FF07C510AF086FE914A009B1288D3F8CD
:100EC00000800292834620460AF028FE029A039B85
:100ED00053F822100AF076FE014600200AF068FD61
:100EE0000BF036F8C5EB0805C9EB0502BD42B8BFEB
:100EF0003D469042C9EB0505C0F2C98200FB05F5ED
:100F000095FBF2F00AF00AFE7E4BDFF80C92039399
:100F10004FF07C5149E0152007F068FB734B0193BB
:100F2000D3F800900746B945B5DC764B0393D3F868
:100F30000090B94580F2A5806D4B6E4E1B88012B49
:100F400000F038836C4A6D4B3068049200930AF0CD
:100F5000E5FD4FF07C510AF035FE6949009B098898
:100F6000029183462046D3F800800AF0D7FD02990B
:100F7000049A52F821100AF025FE0AF0E9FF4544D0
:100F8000BD42C9EB0502A8BF3D46C9EB050590422D
:100F9000BABF00FB055501324543DFF87C9195FB54
:100FA000F2F00AF0BBFD4FF07C51574B02930AF070
:100FB00009FE59460AF0FEFC0AF0CAFF534B04939F
:100FC0003060D9F800B074E04F4B02931E460F20FA
:100FD00008F050FAD6F8008005904045C0F2A6818E
:100FE0004A4B0493D3F80080059B434540F3C982E4
:100FF0003F4B404E1B88012B00F017833E4A306860
:1010000001920AF08BFD4FF07C510AF0DBFD3C4B66
:1010100003901B88009320460AF080FD009B019AF4
:10102000DFF8F49052F82310D9F800B00AF0CAFDA6
:101030000AF08EFF059A5D449542C8EB0503A8BFF0
:101040001546C8EB05059842BABF00FB05550133AC
:10105000454395FBF3F00AF061FD284B00934FF0F8
:101060007C511D46214B01930AF0ACFD03990AF017
:10107000A1FC0AF06DFF234B03933060D5F800808C
:1010800017E01E4B1B4E00931D461F4B306802930A
:101090001E4B04930AF042FD4FF07C510AF092FD82
:1010A0000AF056FFDFF87090D5F80080D9F800B04C
:1010B000306017490988013903295BD8DFE811F04E
:1010C000D00014012E00F2004C99FF1F889AFF1FD8
:1010D000049AFF1F2889FF1F9499FF1F6489FF1F2F
:1010E000B299FF1F44CD0000849AFF1FF099FF1FA3
:1010F0008E9AFF1F7899FF1F1CCD00009C99FF1F3F
:10110000FA99FF1F409AFF1F1C9AFF1F709AFF1F3A
:10111000A889FF1F329AFF1F8899FF1F58460AF0BF
:10112000FDFCAA490AF04EFD054605980AF0F6FCBA
:10113000A7490AF047FD014628460AF03BFC0AF0A1
:1011400007FF8346C9F800B040460AF0E7FC9F4914
:101150000AF038FD054638460AF0E0FC9C490AF0E2
:1011600031FD014628460AF025FC0AF0F1FE009BFD
:1011700080461860974898490788984B08881D68EA
:101180009749DFF8B0E20988C7EB0B0307EB0B02C6
:10119000029F3B60C0EB080700EB08030498026065
:1011A000019A1760039A8D421360BEF8002080F206
:1011B000AA810027C1EB020E8A4B7445186880F2A1
:1011C0009681631C884207FB03F70EF1010E97FB23
:1011D000FEF7C0F249828242A8BF0246521A03FBC0
:1011E00002F494FBFEF48D4200F35781884200F331
:1011F00054817D4C20680AF091FC7C490AF0E2FCA5
:101200007B490AF0D7FB0AF0A3FEA0F5FF531C3B75
:10121000082B98BF4FF40050336818440028206012
:10122000C0F26381B0F5804F80F27481714B1B78FE
:101230001BB1B0F5005F40F075816F4D2B78002B2E
:1012400040F078816D4D20682B68674C984204D03F
:1012500080B204F09BFD23682B6007B0BDE8F08FDF
:1012600058460AF05BFC66490AF0ACFC0546059856
:101270000AF054FC63490AF0A5FC014628460AF02E
:1012800099FB0AF065FE8346C9F800B040460AF0B3
:1012900045FC5B490AF096FC054638460AF03EFCE0
:1012A00058495CE758460AF039FC50490AF08AFC74
:1012B000054605980AF032FC53490AF083FC0146C2
:1012C00028460AF077FB0AF043FE8346C9F800B0CF
:1012D00040460AF023FC45490AF074FC05463846AE
:1012E0000AF01CFC48493AE758460AF017FC4749FF
:1012F0000AF068FC054605980AF010FC44490AF01B
:1013000061FC014628460AF055FB0AF021FE83469F
:10131000C9F800B040460AF001FC3C490AF052FC12
:10132000054638460AF0FAFB394918E7394B3A4E78
:101330001B88012B00F05E81384A306801920AF068
:10134000EDFB4FF07C510AF03DFC354B04901B88BF
:10135000009320460AF0E2FB009B019ADFF8D89048
:1013600052F82310D9F800B00AF02CFC01460020F6
:101370000AF01EFB0AF0ECFD059AC5EB0B05954241
:10138000C8EB0503B8BF1546C8EB05059842BABFC0
:1013900000FB05550133454395FBF3F00AF0BEFB16
:1013A000204B00931D46204B01934FF07C511F4B67
:1013B00003930AF007FC04990AF0FCFA0AF0C8FD4E
:1013C0001B4B04933060D5F8008072E6CDCC4C3FC7
:1013D000CDCC4C3E6A89FF1F7089FF1F4C99FF1FBF
:1013E0005C9AFF1F049AFF1F6089FF1F9A99193F9B
:1013F000CDCC4C45129BFF1F7D99FF1F2089FF1FFD
:101400003333733FCDCC4C3DCDCCCC3E6666663F8E
:10141000CDCCCC3D8E9AFF1F7899FF1F1CCD0000CC
:10142000FA99FF1F9C99FF1FF099FF1F409AFF1F19
:10143000709AFF1F109AFF1F8899FF1F904B00930F
:101440003068904B03930AF069FB4FF07C510AF02F
:10145000B9FB8D4A8A4B1288D3F8008002928346EA
:1014600020460AF05BFB029A039B53F822100AF015
:10147000A9FB0AF06DFDC5EB0805C9EB0502BD42ED
:10148000B8BF3D468242C9EB05057FF737AD00FB8B
:101490000555013295FBF2F034E5BAF80030002B27
:1014A0003FF4A7AE3B1B002BB8BF5B42092B48DDC6
:1014B00007F500500130001B0AF030FB7349744CF3
:1014C0000AF080FB054620680AF028FB71490AF003
:1014D00079FB014628460AF06DFA0AF039FD3368B7
:1014E000184400282060BFF69DAE002214E0884218
:1014F00007FB04F7B8BF002397FBFEF780F2B68026
:1015000093FBFEF46FE69542D4BFC1EB0507C1EB38
:1015100002074FE643F6FF725F4B22601B78002BF9
:101520003FF48BAE00210D2007F076FD5B4B0122CE
:101530001A7087E601210D2007F06EFD00232B7045
:1015400080E64FF40050524C66E6012007F092FF0F
:10155000534B1B6898427FF77BACDFF85CA1514A84
:10156000BAF80010504B52F8210001221A700AF00C
:10157000D5FA4FF07C510AF025FB0AF0E9FC04464D
:1015800070E43F4B494E00931D46494B3068019330
:10159000484B03930AF0C2FA4FF07C510AF012FB59
:1015A0000AF0D6FCDFF81491D5F80080D9F800B025
:1015B00030607EE5334B04933068314B00930AF082
:1015C000ADFA4FF07C510AF0FDFA2F4A009B1288C9
:1015D000D3F800800292834620460AF09FFA029ACE
:1015E000049B53F822100AF0EDFA014600200AF09D
:1015F000DFF9C2E4234A306801920AF08FFA4FF013
:101600007C510AF0DFFA204B04901B88009320469F
:101610000AF084FA009B019ADFF8A09052F8231098
:10162000D9F800B00AF0CEFAA4E6164A3068019262
:101630000AF074FA4FF07C510AF0C4FA124B03908E
:101640001B88009320460AF069FA009B019ADFF894
:101650006C9052F82310D9F800B00AF0B3FA0146A2
:1016600000200AF0A5F9E3E40A46B7E59042D4BFAA
:10167000C1EB0003C1EB020304FB03F340E700BF2F
:101680009C99FF1F1CCD0000FA99FF1FCDCCCC3ECA
:101690006089FF1F9A99193F129BFF1F7D99FF1FB9
:1016A0006C89FF1F2889FF1F9499FF1F7899FF1FDE
:1016B000F099FF1F409AFF1F329AFF1F8899FF1F62
:1016C00030B58DB06D460024E1B23E4804F0C6FF4F
:1016D00001340C2C45F8040BF6D13B4B1B88002B36
:1016E0004DD03A4B0A9A1B889A424BDA009A9342A1
:1016F00048DD029A934245DD049A934242DD344B21
:101700001978002946D03348334A34490088128872
:1017100009680244B1EB620F34DD00241C7004F050
:10172000FFFA21460D2007F077FC322007F0B0FCCD
:1017300001210D2007F070FC322007F0A9FC2146A2
:101740000D2007F069FC322007F0A2FC01210D20DA
:1017500007F062FC322007F09BFC21460D2007F0C9
:101760005BFC322007F094FC0D20012107F054FCB3
:101770004FF42F700DB0BDE8304007F089BC144A1B
:10178000117809B90DB030BD13700DB0BDE830400F
:1017900004F0C6BA0F4C104A114824881288006819
:1017A0002244B0EB620FEDDD01240D201C7007F028
:1017B00033FC322007F06CFC0D20214607F02CFC96
:1017C0003220D7E7389AFF1F089AFF1F189AFF1F89
:1017D000A699FF1F109AFF1F5C9AFF1F049AFF1F14
:1017E0004C99FF1F2DE9F0417B4C7C4D20680AF09D
:1017F00095F97B490AF0E6F90646102007F03AFE13
:101800000AF08CF977490AF0DDF931460AF0D2F88E
:101810000AF09EFB2B882060002B3FD0724F3A8845
:1018200090423BDB01467148067836B94FF0010E15
:10183000042B80F800E000F0B380012B6AD0022B6B
:1018400000F0BC80032B36D1694B1B88092B32D0AA
:1018500023683C88674AA342128853DB9342D4BF73
:10186000C4EB0303C4EB0203141B7E2CDFF8888156
:10187000D5BFC3EB8313C3EBC3135B00013493FBEE
:10188000F4F4D8F800300134A34203D0E1B24A2086
:1018900004F09EF9C8F80040BDE8F081534A117881
:1018A00049B10024012B147016D0022B1FD0032B3A
:1018B00003D0042B28D0BDE8F0814D4B1B88092BA9
:1018C000F9D04D4D2B68002BF5D021464A2004F06D
:1018D0007FF92C60BDE8F081474D2A68002AEAD0E4
:1018E0001846214604F074F92C60BDE8F081424DA1
:1018F0002B68002BDFD02146042004F069F92C600E
:10190000BDE8F0810023AFE721464020BDE8F0416B
:1019100004F05EB9374B1B888B42D4BFC2EB030681
:10192000C2EB01069A1ADFF8D0807E2AD8BFC6EB38
:101930008616D8F80030C6BFC6EBC6160132760050
:1019400096FBF2F60136B34203D0F1B2012004F067
:101950003FF92B88C8F80060022B7FF473AF23682F
:101960003E88244AB34212882CDA0023961B7E2E2E
:10197000DFF88480D5BFC3EB8313C3EBC3135B00D5
:10198000013693FBF6F6D8F800300136B34220D08A
:10199000F1B2042004F01CF92B88C8F8006051E76C
:1019A0007F21402004F014F92B88012BD4D1216829
:1019B0003A88104B91421B88B4DBADE70D4A23688F
:1019C00012883E889A42D4BFC6EB0203C6EB0303DB
:1019D000CCE70223E1E700BF789AFF1F589AFF1F68
:1019E0009A99193FCDCCCC3E5E9AFF1F8499FF1F78
:1019F0006299FF1FEE99FF1F9899FF1F38B5184B8A
:101A00001B88D3B9174A184914880968174AA14294
:101A100012881DDA141B7F2CC6BFDB010134C3EB17
:101A2000C31393FBF4F4124D2B689C4203D0E1B234
:101A3000052004F0CDF82C6038BD0E4B0E490F4A3E
:101A40001B680C6812681C1BA41A84F30704EAE7DD
:101A50009142D4BFC4EB0103C4EB0203DAE700BF39
:101A6000B299FF1F449AFF1F6C9AFF1F2E9AFF1F07
:101A7000349AFF1F009AFF1F2489FF1F649AFF1FDB
:101A800010B50C4C236843B90B4B1B88022B0CD0B0
:101A90000A4A00231370236010BD0021052004F0C2
:101AA00097F8054B1B88022BF2D10021412004F04E
:101AB0008FF8EDE7349AFF1FEC99FF1F629AFF1F22
:101AC00010B5254B1B787BB1152006F08FFD234AFE
:101AD000234B1288186082B9224A12883ABB224BE3
:101AE0001B78002B33D110BD112007F0C3FC1B4A1B
:101AF0001B4B12881860002AEED00F2007F0BAFCAA
:101B0000184B1A4A1B881060002BE8D0184A194954
:101B100012680968521A9042E1DC134C227892B99B
:101B2000022B0ED17F21412004F052F809E0124926
:101B30001B6809889942D2DC0B4C23781BB9022A16
:101B4000F0D001232370BDE81040FFF757BFBDE878
:101B50001040FFF795BF00BF849AFF1FB299FF1F87
:101B60006C9AFF1FEC99FF1F629AFF1F649AFF1F78
:101B7000009AFF1F2489FF1F449AFF1F2DE9F04F91
:101B800091B004AD0024E1B2744804F067FD013463
:101B90000C2C45F8040BF6D1714B724CB3F800E0F5
:101BA0000C9B00227345227014DB0A9B9E4500F3B8
:101BB000C080089B6C4A9E4503DD1378002B40F0E3
:101BC000C880069B9E4540F3BA804FF0020C84F813
:101BD00000C009E0089B644A9E45CCBF4FF0060C4C
:101BE0004FF0050C84F800C00E9F059E07980999D8
:101BF00082F800C0BE45D4BF00270127B645D4BF38
:101C00000026012686450B9ADFF898810D9B0F9DD3
:101C1000DFF894A1DFF894918AF80060D4BF002027
:101C200001208E45D4BF0021012188F8001096457F
:101C30004E49DFF87CB14E4E89F80000D4BF002237
:101C400001229E45D4BF002301230A70AE45494AB4
:101C50008BF80070D4BF002501250120137035706A
:101C600007F008FC444B454A1D681188444BA842C4
:101C7000D4BF002201220B291A7001D90C2901D0EE
:101C8000A8424EDC002301933E4B9AF800E01F78F7
:101C900099F800C098F800209BF800303349367856
:101CA00091F800903349DFF80CA191F80080247876
:101CB000A7EB4E07CCEB070CA2EB8202C3EB8377BA
:101CC0006244C3EB8703134403EB4903434403EB30
:101CD0008606BAF800202C4F0C2313FB046632440E
:101CE000019B3E600C3A1344A8421946274AC4BFE0
:101CF000274B1E701368994217D0264B264C186844
:101D00000290029820601B680393244C039B248854
:101D100011601B1AA34284BF214B196011B0BDE8AA
:101D2000F08FA1F10C030193AEE71B48194B00683B
:101D3000E9E74FF0040C84F800C00B4A54E7049B19
:101D40009E45C6BF4FF0010C84F800C04FF0000C58
:101D50004AE74FF0030C84F800C045E7389AFF1FAC
:101D6000189AFF1F4999FF1FF899FF1F8A9AFF1FB2
:101D70008C9AFF1FB499FF1F6C89FF1F889AFF1F61
:101D80004899FF1F5C89FF1F809AFF1F6899FF1FFA
:101D90008B9AFF1F6C9BFF1F9099FF1F909AFF1F4C
:101DA000A099FF1F869AFF1FAC99FF1F859AFF1FFE
:101DB000B099FF1F8099FF1F2DE9F04F0E208FB0C3
:101DC00006F014FC09F0AAFE01468948894D8A4FA5
:101DD00004F09EFD864804F071FD0AF0B9F880F326
:101DE0000C002860FFF7CAFE3E68012E00F0B080AC
:101DF000022EDFF870A200F0B081032E00F02782DF
:101E00007E4C7F4B7F4E019323687F4F0A930A9B42
:101E10003A689B1A022B1ED9DFF84C8298F80030E2
:101E2000002B00F0F483794B1A78002A0CBF0122B2
:101E300000221A7000F0E68398F80030002B40F082
:101E4000E983FFF7CFFCFEF719FFFFF739FC2368A2
:101E50000B930B9B3B6023686D4F0C930C9B3A6874
:101E60009B1A502B5CD86B4B31686B481A78183929
:101E70002A2303FB01F10160002A47D0674A136857
:101E8000994240F3598166480068D0F17F0048BF0D
:101E9000033003EBA0030133994280F25B811160B0
:101EA000604B1B68A92202FB03F3002BBCBF03F5A8
:101EB0007F533F339B13543B1944282081F30C017B
:101EC00006F01AFF2B68BAF80000019A83421288C4
:101ED0001FDA0024111A40F60B639942C3BF40F683
:101EE0000C62013102FB04F3634393FBF1F000F554
:101EF000FA70FEF7A9FE0146142006F0FDFE03F07D
:101F0000FBFE03F029FD0FB0BDE8F08F434B1960D5
:101F1000C6E79342D4BFC0EB0304C0EB0204D9E789
:101F200002F0CCFD404B1B7823B9404B1B78002BB3
:101F300000F0EE810D2007F075F8B0FA80F1490944
:101F40000D2007F069F823680D930D9B3B608AE72D
:101F5000374B384A18881378834204D0C3B21846E6
:101F6000137003F005FEDFF80481334AB8F800006F
:101F70001378834204D0314C2378002B40F0288220
:101F8000DFF8E0A02B68BAF800201C4C9A4280F2DF
:101F9000B98121682A4A079107982A4910600222CC
:101FA0000B603A60284B1F88002F61D1274B1B889C
:101FB000002B5DD1264B1F680E2006F017FBA7F201
:101FC0001F37874202DC234B00221A70224B1B88EA
:101FD000002B40F05183144E14482049204A33709E
:101FE00003700B701370064B064E01930CE700BF95
:101FF000BC99FF1F6499FF1F7499FF1F6C9BFF1F03
:10200000929AFF1FA099FF1F289AFF1F8699FF1F12
:10201000E899FF1F629AFF1F489AFF1FF499FF1F5C
:10202000349AFF1F6089FF1F7C99FF1FA499FF1F2F
:10203000B899FF1F309AFF1F759AFF1FE699FF1F7F
:102040003899FF1FE099FF1F5A9AFF1FDC99FF1F65
:102050000C9AFF1F7C9AFF1F4C9AFF1FFC99FF1FD1
:10206000A799FF1FB699FF1F749AFF1F8299FF1F40
:10207000DFF84CB3DFF84C93BBF80000B9F8003040
:10208000B649B74A18440B684010984205DA1368FD
:10209000984202DA002F40F08D83B24B02921F4625
:1020A0000E200391019306F0A1FA3F68029AA7F56A
:1020B000487E704580F29C81AB480088002800F083
:1020C00097810399BBF800C0B9F800000B6812684B
:1020D0000CEB00014910994280F29181914240F34A
:1020E0008E81A2480768791C002940F399858029D0
:1020F00000F395859E4E9F4A9F4B3688128801605B
:1021000018683244B0EB620FC0F2ED87A7F14802C5
:102110000F2A00F2D583994B0021473F0D201F80E5
:1021200006F07AFF962006F0B3FF01210D2006F09D
:1021300073FF019B1F683FE7BFF6B1AE9048006890
:10214000D0F17F0048BF0330801001301B1A994244
:102150003FF7A5AE13601946A2E62E68BAF8003024
:10216000B34280F2EF80874C874822680892874A02
:10217000089900681288091A914202D8002A7FF44F
:1021800040AE834A834912680191B242B8BF3246D9
:1021900093420888804940F32D86804A098813605D
:1021A000002900F00A83DFF8208288F800107C4EB6
:1021B000FEF7B4FD30687F2840F32986794B7F38DD
:1021C00083FB0032C317C3EB620303EB4303A0EBB3
:1021D00083007330744B03931B883060002B40F0F6
:1021E0004687724B02931B78002B00F07584DFF852
:1021F000DCB19BF80030002B00F06E846C4B049433
:102200004FF000094C4699460CE003F17300C0B250
:1022100098F8001003F004FD9BF800300134A3424D
:1022200040F35984336859F8040F5E4A1844A0F10A
:102230007F0382FB032ED917C1EB6E0101EB410135
:102240007F28A3EB8103E0DCFEF738F9DFE7D5F860
:102250000080BAF80010414540F30681554B1B78C9
:10226000002B40F00181544C20787F2840F35F8799
:10227000A3F155337F3803F1004383FB0032C317CA
:10228000C3EB620303EB4303A0EB83007330464BC5
:1022900003931B88C0B22070002B40F08387434B10
:1022A00002931B78002B00F0B685DFF820B19BF875
:1022B0000030002B00F0AF853D4EDFF8E8804FF096
:1022C00000090BE003F17300C0B203F0D1FC9BF8EE
:1022D000003009F101094B4540F39D8556F8043F54
:1022E00020781844A0F17F0388FB0321DA17C2EBA2
:1022F000610202EB42027F28A3EB8203E2DCFEF7DD
:10230000DDF8E1E72B4A1278002A3FF44BAE40E6B5
:10231000264B1B78002B7FF40DAE284B1B78002B2F
:102320007FF408AE234B1B78002B7FF403AE0D2007
:1023300006F078FE00287FF406AE01210D2006F09D
:102340006BFE00E61B4A1278002A7FF40CAF0123D3
:102350003B60104B0B4C124E019355E54C99FF1FFF
:10236000049AFF1F0C9AFF1FDC99FF1F809AFF1F22
:102370005E9AFF1FEE99FF1F789AFF1FB899FF1F03
:10238000349AFF1F6C9BFF1F3899FF1F249AFF1F71
:10239000E099FF1F929AFF1F4099FF1F149AFF1F99
:1023A000A099FF1FABAAAA2A7E99FF1FFC99FF1FC5
:1023B0008089FF1FA699FF1F229AFF1FA799FF1F61
:1023C000109AFF1F5C9AFF1F8599FF1F6889FF1FE6
:1023D000C3B21846137003F0D9FB904B904A1946CC
:1023E000904B18460023137023700B700370C7E5E1
:1023F000BBF80000B9F8001012680144491091427E
:10240000BFF6DAAD0E2006F0F1F8019B1F68A7F5C4
:1024100048729042BFF6D0AD83480278002A7FF41C
:10242000CBAD824E327801210170002A40F0158236
:102430007F4A1278002A40F084867E4A1278002A69
:1024400000F0E8867C4B1B78002B7FF4B5AD7B4B0E
:102450001B78002B3FF4B0ADB8F80030784A0A334F
:10246000A8F800301170A7E5764E30687F2840F359
:102470005981754B7F3883FB0032C317C3EB62036E
:1024800003EB4303A0EB83007330704C2778874243
:1024900000F058856E4B1B88002B00F046816D4B79
:1024A00001937F2F40F39D8467487F3F80FB073077
:1024B000FB17C3EB600000EB4000A7EB800073301C
:1024C000564B02931B78C0B22070002B40F0FE8365
:1024D000544B04931B78002B40F0D9855E4B059339
:1024E0001B78002B40F065865C4B0393059B1B78A3
:1024F000A3B35B4B22781B881344A3F118007F28F9
:1025000040F3ED85504A973B82FB0321DA17C2EB7B
:10251000610202EB4202A3EB820303F17300C0B23B
:1025200003F0A6FB4F4B504A1978237832F811205C
:102530001344A3F118007F2840F3CD85424A973B0E
:1025400082FB0321DA17C2EB610202EB4202A3EB2A
:10255000820303F17300C0B203F08AFB029B1B7875
:10256000002B00F0F284039B3C4F1988002900F0F7
:10257000858530687F2840F33984334B7F3883FB6F
:102580000032C317C3EB620303EB4303A0EB8300EA
:1025900073303060002940F0FE84029B1B78002BD2
:1025A00000F09281DFF8C8B09BF80030002B00F0FB
:1025B0008B812E4FDFF8BC804FF000090DE003F156
:1025C0007300C0B298F8001003F02AFB9BF80030AB
:1025D00009F101094B4540F37781336857F8040F3F
:1025E000194A1844A0F17F0382FB0321DA17C2EBDA
:1025F000610202EB42027F28A3EB8203DFDCFDF7DE
:102600005DFFDEE7FEF712FCFFF75AFA1FE4FEF764
:1026100085FB08E4FEF782FB13E400BFFC99FF1F73
:10262000A499FF1FA799FF1F7C9AFF1F4999FF1FBD
:10263000AC99FF1F859AFF1F869AFF1FB099FF1F55
:10264000E699FF1FA099FF1FABAAAA2A229AFF1F93
:102650004099FF1F929AFF1F7C99FF1F7E99FF1FD1
:10266000609AFF1F689AFF1F509AFF1F8089FF1F03
:102670006889FF1F8599FF1F002006F0FBFEA94B0C
:10268000A94F1A683978A94E9042D4BF002301237C
:102690009942337040D090423EDDA54A92F800C086
:1026A000BCF1000F00F0B784A24A92F80080B8F1A4
:1026B000000F40F0AE84A049A04EA14809780296D0
:1026C0004FF0010E059086F8008080F8008082F8B7
:1026D00000E0002940F081859A4A1278002A00F033
:1026E0001685994A049210461278002A40F00C850B
:1026F0009649934E0978327001220596027059B1BD
:102700008E498C4A029100211170029A059E117027
:10271000049A0120307011703B708D4B8D4E0193E7
:10272000FFF772BBFDF7CAFEAFE68B4A8848126816
:1027300001909142008805DC8242D4BFC1EB0203C4
:10274000C1EB0003411AB1F5804FC0F2B5849B0381
:10275000481C93FBF0F0FEF777FAC0F3C61009F0BF
:10276000DDF97E4B8046188809F0D8F97C4981460E
:10277000404609F027FA0146484609F023FA414647
:1027800009F018F94FF07E51804609F0B9FB002896
:1027900040F0FC847349404609F0D0FB002840F02B
:1027A000CA84404609F0FAFBC0B2DFF8E48188F839
:1027B000000076E66C4B019393E41A469042D4BF36
:1027C000C3EB0001C3EB0201C01AB0F5804FC0F2A9
:1027D0008C848A03013092FBF0F0FEF735FAC0F3E7
:1027E000C61009F09BF95D4B0646188809F096F96A
:1027F0005B498046304609F0E5F90146404609F05C
:10280000E1F9314609F0D6F84FF07E51064609F05D
:1028100077FB002840F0CA845249304609F08EFB0D
:10282000002840F08B84304609F0B8FBC0B2DFF8D6
:10283000608188F80000BAE43D4A1278002A7FF4EB
:10284000BBAB4A4A4A481278243A82F347020260F4
:10285000D1B25B2003F0BCF93278032A30D1394E73
:102860003178002940F02185424F3A78002A40F023
:102870000F85DFF8BC8098F80020002A40F0FB8428
:102880003D4A1278002A40F0E9843C490A802A4AED
:102890001278002A40F0D584394A7F21118032789D
:1028A00072B93A7862B998F800204AB9354E7F215A
:1028B0000720328003F08CF97F210B2003F088F988
:1028C000019B1F68FFF778BB049B1B78002B00F06F
:1028D00087803368A3F10C007F2840F3F9832A4AEC
:1028E0008B3B82FB0321DA17C2EB610202EB42024F
:1028F000A3EB820303F17300DFF89480C0B298F871
:10290000001003F08DF9029B1B78002B68D0DFF8D4
:1029100084B09BF80030002B62D01C4F4FF00009B0
:1029200047E000BF6C89FF1F699AFF1FA599FF1F31
:10293000B099FF1FA499FF1F8A9AFF1FFC99FF1FE0
:102940007C99FF1FAC99FF1FA799FF1F4899FF1F94
:10295000929AFF1FA099FF1F149AFF1F5099FF1F03
:10296000CDCCCC3D0000FE420C9AFF1F8B9AFF1F7E
:102970003C9AFF1F869AFF1F859AFF1F209AFF1F10
:102980004099FF1F6299FF1FABAAAA2A8089FF1FE7
:102990008599FF1F6889FF1F03F17300C0B298F883
:1029A000001003F03DF99BF8003009F101094B4597
:1029B00016DD336857F8042FAF491A44A2F18B0390
:1029C00081FB0310D917C1EB6001A2F10C0001EBF0
:1029D00041017F28A3EB8103DEDCFDF76FFDDDE71E
:1029E000059B1B78002B40D0A44A336812881344FF
:1029F000A3F118007F2840F368839F4A973B82FB2E
:102A00000321DA17C2EB610202EB4202A3EB82035D
:102A100003F17300DFF8B082C0B298F8001003F041
:102A2000FFF897490B78022B9ABF5A1CD2B20022AA
:102A30000A709449336831F812201344A3F1180046
:102A40007F2840F33F838C4A973B82FB0321DA17B0
:102A5000C2EB610202EB4202A3EB820303F17300BB
:102A600098F80010C0B203F0DBF8039B1B88002B22
:102A700000F08B82029B1B783BB9049B1B7823B927
:102A8000059B1B78002B00F0D8837F4B1B78002B15
:102A900000F0EF807D490B78082B00F2EA807C483B
:102AA000326800687B4F0133DBB203F1FF3E101A3E
:102AB00047F82E000B70BAF80010D5F8008022708D
:102AC0004145754CBFF6A0A92268744B0992099A3A
:102AD0001A60FFF799B9049C6B4B1B78002B40F0F0
:102AE000638233686E4A1278002A4AD0A3F10C0040
:102AF0007F2840F30083604A8B3B82FB0321DA1777
:102B0000C2EB610202EB4202A3EB820303F173000A
:102B1000C0B298F8001003F083F8029B1B787BB3D7
:102B2000DFF868B19BF8003053B35E4B02944FF06E
:102B300000094C4699460BE003F17300C0B298F8C7
:102B4000001003F06DF89BF800300134A34216DD4D
:102B5000336859F8041F484A1944A1F18B03D81768
:102B600082FB032EC0EB6E0EA1F10C000EEB4E0E9D
:102B70007F28A3EB8E03DFDCFDF7A0FCDEE7029CE1
:102B80003368494A1278002A3ED03C4A10880344F0
:102B9000A3F118007F2840F3B482374A973B82FBA9
:102BA0000321DA17C2EB610202EB4202A3EB8203BC
:102BB00003F17300C0B298F8001003F031F8304907
:102BC0000B78022B9ABF5A1CD2B200220A702D49F0
:102BD000336831F812201344A3F118007F2840F322
:102BE0008D82254A973B82FB0321DA17C2EB6102F3
:102BF00002EB4202A3EB820303F17300C0B298F828
:102C0000001003F00DF83368039A1288002A00F0D0
:102C1000F981264903220B703A60FFF7F5B8802648
:102C20002349244A0F8824491288096806603A44D7
:102C3000B1EB620FBFF644AE204A1178002940F094
:102C40009281B8F800201E48B2423FF439AE1D4AC6
:102C5000068001260D20167006F0DEF9962006F09B
:102C600017FA31460D2006F0D7F9019B1F68FFF7D0
:102C7000A3B932681FE700BFABAAAA2A609AFF1F58
:102C8000689AFF1F509AFF1FA499FF1F6889FF1FB2
:102C9000A899FF1F8489FF1F6C9BFF1F1C9BFF1FB0
:102CA000A799FF1F8089FF1F7C99FF1F229AFF1F92
:102CB0005E9AFF1FEE99FF1F789AFF1F4899FF1F2A
:102CC0008299FF1FE699FF1F8599FF1FBC4B039355
:102CD0001B88002B40F00883BA4B0493BA4B059332
:102CE000DFF81CB39BF8003063B3B84FDFF8E08225
:102CF0004FF000090AE003F17300C0B202F0B8FF20
:102D00009BF8003009F101094B451BDD57F8043FE2
:102D100020781844A0F17F0388FB0321DA17C2EB67
:102D2000610202EB42027F28A3EB8203E3DCFDF7A2
:102D3000C5FBE2E7A44B059302F09AFF029B1B78C8
:102D4000002BCDD1049B1B78002B3FF4CFAB237815
:102D5000A3F10C007F2840F397819D4A8B3B82FBB7
:102D60000321DA17C2EB610202EB4202A3EB8203FA
:102D700003F17300C0B202F07BFF029B1B78002BB3
:102D800000F08E81DFF878B29BF80030002B00F065
:102D90009D828E4FDFF838824FF000090BE003F17F
:102DA0007300C0B202F064FF9BF8003009F1010922
:102DB0004B457FF79BAB57F8043F22781A44A2F1AA
:102DC0008B0388FB0310D917C1EB6001A2F10C0043
:102DD00001EB41017F28A3EB8103E0DCFDF76EFBF3
:102DE000DFE73846FDF76AFBFFF76ABBFDF766FBD6
:102DF000FFF7CFBB774E09888242A8BF02463260F8
:102E000000297FF4D0A993423FF7DEACD6E4FDF76A
:102E100055FBFFF7DFB96B4B1B78002B43D02378B2
:102E2000A3F10C007F2840F3CC81694A8B3B82FBE5
:102E30000321DA17C2EB610202EB4202A3EB820329
:102E400003F17300C0B202F013FF029B1B7853B36F
:102E5000DFF8ACB19BF800302BB35C4EDFF870812B
:102E60004FF000090AE003F17300C0B202F000FF66
:102E70009BF8003009F101094B4514DD56F8043F79
:102E800020781844A0F18B0388FB0321DA17C2EBEA
:102E900061020C3802EB42027F28A3EB8203E2DCE2
:102EA000FDF70CFBE1E7484B1B78A3B34A4B2278B4
:102EB0001B881344A3F118007F2840F38881444AFB
:102EC000973B82FB0321DA17C2EB610202EB42025D
:102ED000A3EB820303F17300C0B202F0C9FE3F4BC3
:102EE0003F4A1978237832F811201344A3F11800CF
:102EF0007F2840F36981364A973B82FB0321DA172A
:102F0000C2EB610202EB4202A3EB820303F1730006
:102F1000C0B202F0ADFE039B1B88002B00F03E8187
:102F2000304B1B78002B40F034812A4BBAF800104C
:102F3000D5F800802C4E00221A6001233B602B4BF9
:102F40000193BDE5294B0193BAE5049B1B78002B47
:102F50007FF409AB059B1B78002B7FF404AB039B2C
:102F60001988FFF706BB4B2E40F302811836802EDE
:102F7000B8F800201E49A8BF802696423FF4A0ACB6
:102F80001C4A0E800126002164E61B4B307819781C
:102F900002F046FE6EE5DFF86080C0B298F80010DF
:102FA00002F03EFEFFF7F9BA7F21402002F010FE4A
:102FB0001249134A33680B600021117092E500BF7B
:102FC0007E99FF1FA799FF1F7C99FF1F8089FF1F14
:102FD000ABAAAA2A149AFF1F609AFF1F689AFF1FC4
:102FE000509AFF1FA499FF1FA099FF1F929AFF1FDD
:102FF0008299FF1FE699FF1F8599FF1FA899FF1F60
:103000006889FF1FD8B298F8001002F009FE3368F3
:10301000FFE500211170B74A117841B1B64A02921A
:103020001278002A00F0D680029800220270B34A7B
:103030001278002A7FF455ABBCF1000F67D100294C
:1030400065D1AF48AC4E90F800E0AE480490AE4871
:103050000590AC48AD4A0170AB48029611703170D2
:103060000170BEF1000F3FF457ABFFF74CBBC0B28D
:1030700098F8001002F0D4FDFFF7B3B8207802F002
:10308000F7FD3988FFF775BAFDF718FA72E6A04B1D
:1030900003931B88002B7FF44DAE9B4B059356E6A4
:1030A000059B1B78002B7FF424AA049B1B78002B24
:1030B0003FF455AFFFF757BAC3EB833393FBF1F0FF
:1030C000FFF749BBFDF7FAF9CAE4FDF7F7F9A1E408
:1030D000FDF7F4F910E4FDF7F1F9FFF73CBAFDF75D
:1030E000EDF9FFF71CBA0E46A6E5C1EB813191FB65
:1030F000F0F0FFF772BBFDF7E1F909E5FDF7DEF946
:103100007CE5FDF7DBF955E5049900220A707C4A5D
:103110001278002A3FF400AB7B4A05921278002A0D
:1031200000F0DB80059900220A70FFF7F5BAFDF781
:10313000C5F9FFF7ACB87F20FFF737BB7F20FFF75B
:1031400076BB744B1B78002B51D0734B1B78002B34
:103150007EF432AF714B1B78002B3EF42DAFB8F8E4
:1031600000306F4A0A3BA8F800301170FEF724BF08
:10317000243E002EB8F8002040F3A380B2423FF472
:103180009FABB6B2664AA8F80060FBE60120FFF7E5
:103190000CBB0021402002F01BFDC6E6207802F0A7
:1031A00067FDBDE602F064FDFFF779B80120FFF787
:1031B0003EBB574B03931B88002B7FF4BDADFFF73D
:1031C00095B9FDF77BF93DE6FDF778F9A0E6FDF747
:1031D00075F981E64C484D4A059000261670029814
:1031E000059A4FF0010E80F800E016701FE74A4B79
:1031F0001B78002B7EF4E0AE484B1B78002B3EF48E
:10320000DBAEB8F80030464A013BA8F80030117038
:10321000FEF7D2BE404A1278002A7FF40DAB3F4B36
:103220001B78002B3EF4C8AEB8F800303C4A01339E
:10323000A8F800301170FEF7BFBE207802F018FD2C
:1032400023E4384A002010807F21072002F0C0FCD0
:103250007F210B2002F0BCFCFFF721BB324A01208A
:1032600010807F21072002F0B3FC7F210B2002F0A9
:10327000AFFCFFF70CBB2D4A042010807F210720F4
:1032800002F0A6FC00210B2002F0A2FCFFF7F8BA26
:10329000264A022010807F21072002F099FC7F211E
:1032A0000B2002F095FCFFF7E4BA204800210280D1
:1032B000072002F08DFC7F210B2002F089FCFFF734
:1032C000D3BA012A3FF4FCAA01265BE7059B1B78D1
:1032D000002B7FF40EA9FFF746B90749029109496F
:1032E0000A4A0491FFF70FBA064B0493064B059365
:1032F00022E500BF8A9AFF1FFC99FF1FAC99FF1FB0
:103300004899FF1FA799FF1F7C99FF1FA499FF1FD2
:103310007E99FF1F859AFF1F869AFF1FB099FF1F96
:10332000E699FF1F4099FF1F209AFF1F6299FF1F18
:1033300010B505F0F7F9064803F028F900234FF01F
:103340007E5204480121BDE8104003F07DBA00BF61
:10335000389AFF1FBC99FF1F43682A20198801F083
:1033600033B900BF10B5044622206368198801F004
:103370002BF9E36824201988BDE8104001F024B936
:1033800010B504460A206368198801F01DF9E36846
:103390000C201988BDE8104001F016B910B504469C
:1033A00006206368198801F00FF9E368082019887E
:1033B000BDE8104001F008B910B50446022063686A
:1033C000198801F001F9E36804201988BDE810406C
:1033D00001F0FAB870B50E4C84B012250422012316
:1033E00006460390029320468DE824001423102102
:1033F00004F06CFB062209230293039601952046F4
:1034000000921423102104F061FB04B070BD00BFD2
:10341000AC9AFF1F2DE9F041224D82B0012602B285
:1034200084B20092284601967823192104F094FA78
:1034300004F10C0212B28DE844002846A719782343
:10344000192104F1020804F087FA3FB20FFA88F854
:1034500019233A46284619460196CDF8008004F013
:103460007BFA78233A4628461946CDF80080019623
:1034700004F10A070B3404F06FFA3FB224B2782348
:103480003A46284619468DE8500004F065FA19239B
:1034900000943A4601962846194604F05DFA02B0B7
:1034A000BDE8F081AC9AFF1F2DE9F0411E4682B0C5
:1034B0001446002A6AD0099B4D4A00EBC305012C33
:1034C0006F8929896868A7EB010382FB03E21A442C
:1034D0004FEAE373C3EBA21302887BD0042C38D1EC
:1034E00012FA83F3994203DC9F423946A8BF19467A
:1034F000089A0180B6F90030BDF920803D48971D3B
:103500004FF0000E3FB2194642460097CDF804E056
:1035100004F022FA29896A896B68521A1B885C2A8E
:10352000A3EB010359DD03EB43030132C3EB431368
:1035300093FBF2F303F11B0213B201203280194610
:103540004246019000972B4804F006FA2A4B0022CD
:103550001A702A4B022CB3F9001045D0082C31D137
:1035600000221A8091422DD0089AB6F900302148E5
:103570000632012412B2009219460194BDF92020AE
:1035800004F0EAF9204602B0BDE8F0811C4D1D4A66
:103590002B681268CB1A93420F4617D9164A338804
:1035A00011781448012918BF01241470089A0632B2
:1035B0001BB212B28DE814001946BDF9202004F0A8
:1035C000CBF92F60012002B0BDE8F081204602B0A7
:1035D000BDE8F0819BB2D31A84E75C2101FB03F3C1
:1035E00093FBF2F21B32A7E74A1C12B21A80B9E72A
:1035F000C94216B2AC9AFF1F209BFF1F9E9AFF1F65
:103600001C9BFF1F10D4000030B583B000230C4674
:1036100005B2009326225B231C210C4803F0ECFE2C
:10362000294601232622094803F0F6F9002C24B28A
:1036300005DB214601232622044803F0EDF9044A64
:10364000044B15801C8003B030BD00BFAC9AFF1F37
:10365000AA89FF1FAC89FF1F70B5944C237882B0F4
:103660001BB1934B4FF6FF721A80924BB3F90030A7
:10367000C3B9914A8E4B1068B3F9002080F30C0057
:103680005B2303FB00F000131C3082425AD04FF042
:10369000FF31FFF7B9FF894803F012FF00232370C1
:1036A00002B070BD012B32D0022B6AD0032B4FD059
:1036B000042BF3D1272200258DE8240076231C213A
:1036C0007E487F4E04F048F917E0B0F5AF7FA8BF01
:1036D0004FF4AF70323803FB00F386FB0321DB1796
:1036E000C3EB61111C3109B201231D442722734829
:1036F00003F092F90C2D00F08180E9B2714802F0DC
:10370000ADFF31284FF05B03DFDC1C21ECE76E4B93
:103710001A68B2F52F7F32DB41F25C239342A8BFD7
:103720001346A3F52F735B22684802FB03F380FB6B
:103730000320DB17C3EBA0201C305D4BB3F9003036
:103740008342A4D1624BB3F9003001339FD1A5E786
:10375000604B1B68B3F5FA7F11DBB3F57A6FA8BF36
:103760004FF47A63A3F5FA725B485B2303FB02F321
:1037700080FB0320DB17C3EB20201C30DDE71C207F
:10378000DBE7564B1B68B3F5FA7F33DBB3F57A6F93
:10379000A8BF4FF47A63A3F5FA724F485B2303FB8B
:1037A00002F380FB0320DB17C3EB20201C304C4BC3
:1037B0001B68B3F5FA7F1FDBB3F57A6FA8BF4FF430
:1037C0007A63A3F5FA7244495B2303FB02F381FB9E
:1037D0000321DB17C3EB21211C31354BB3F900303A
:1037E00083427FF456AF3A4BB3F900308B427FF4FB
:1037F00050AF53E71C20DAE71C21EEE7012005F06B
:1038000039FE6FF495733238364A03FB00F082FBC1
:103810000023C017C0EB632303F5AF73312B3ADDF0
:10382000B3F5AF7FA8BF4FF4AF735B22323B244D9B
:1038300002FB03F385FB0325DB17C3EB65151C3582
:10384000002005F017FE6FF495733238254A03FB0C
:1038500000F082FB0023C017C0EB632303F5AF73B6
:10386000312B1ADDB3F5AF7FA8BF4FF4AF735B22E6
:10387000323B134902FB03F381FB0321DB17C3EB4C
:1038800061111C310A4BB3F90030AB4207D0284616
:10389000FFF7BAFEFFE61C25D2E71C21F2E70C4B2E
:1038A000B3F900308B42F2D1F5E600BF949AFF1FC6
:1038B000AA89FF1F9A9AFF1F6499FF1FAC9AFF1FE6
:1038C0004B48371B389AFF1F6C9AFF1FD305854161
:1038D000AC89FF1F789AFF1F011FB8124C99FF1F78
:1038E000049AFF1F67BBCF462DE9F04FDFF8EC824B
:1038F000B74CB8F900604D7854F8264087B082463E
:10390000039305B10D78DFF8FCB2002A34D19BF89F
:1039100000308BBBAF4EB6F90000002800F0CE801F
:10392000012800F02481012032232A4601900093CF
:103930005146A94B2046FFF7B7FD00250746B6F9CB
:103940000030022B40F3F48000233380B8F90030BC
:10395000A24A002BC0F2F880042BC4BF00231380BE
:10396000039B002B40F0F680002D0CBF38464FF033
:10397000FF3007B0BDE8F08F964EE36822689848A4
:1039800004930027059237808BF8007003F08CFCBD
:103990001120FFF73FFD4FF0010919232821CDF831
:1039A00004900091242219468D4803F0D5FF782316
:1039B00028212422CDF8049000918948194603F06B
:1039C000CBFF4946864804F05DFB0222192184485A
:1039D00004F054FBDDF81490484608F071FE4946A7
:1039E00002467F4804F04EFC7D4804F061FC3946F5
:1039F00014227B4804F042FB03227A49784804F001
:103A000041FC774804F054FC39462322744804F002
:103A100035FB03227449724804F034FC704804F00A
:103A200047FC049B002B72D10123704A1846137087
:103A3000FFF7D0FC208963896768191A5C293A88E6
:103A40005BDC131A5C2202FB03F292FBF1F31B33E3
:103A5000674A6348138001271BB21A2219468DE872
:103A60008400142203F078FF049BDBB1218A638A6F
:103A7000E768581A5C283A886FDD521A02EB420256
:103A8000C2EB4212431C92FBF3F31B33524A5448DD
:103A90001380012738221BB28DE884001946322298
:103AA00003F05AFF534A544BB6F90000012111703C
:103AB0004FF6FF721A8000287FF432AFDFF848918A
:103AC0004E4AD9F800301268C3EB0A0393424CD92E
:103AD000464B1A78012A18BF012018700127FFF7FA
:103AE00079FCC9F800A0012D4ED0042D59D0022D2B
:103AF00060D0082D64D0002521E7121A02EB4202A3
:103B0000C2EB42124B1C92FBF3F31B33A0E72F20B6
:103B1000FFF780FC39463222314804F0AFFA032225
:103B200037492F4804F0AEFB2D4804F0C1FB7BE77A
:103B30007FF40CAFE368002B3FF406AFB8F9003018
:103B4000264A002BBFF608AF04231380039B002BEB
:103B50003FF40AAFFFF780FD06E7511A5C2202FB33
:103B600001F292FBF0F31B3390E70746BBE7002717
:103B700014238DE888002A4651461D4B2046FFF746
:103B800093FC3D460746DAE6B8F800308BF8005063
:103B90000133A8F80030636983B1002520469847B7
:103BA000CDE6B8F800300122013BA8F800308BF8D0
:103BB0000020F0E7012333800025C7E61D46BEE65E
:103BC0006369002232804FF0FF35002BE6D1BDE65D
:103BD000B089FF1F9E9AFF1F989AFF1F9A9AFF1F96
:103BE000AC9AFF1FD4CD0000D8CD0000209BFF1F52
:103BF000969AFF1F949AFF1FAA89FF1F10D40000F6
:103C0000DCCD00009C9AFF1F1C9BFF1F064B074A40
:103C100010B41C88064B0846002C14BF11461946E8
:103C2000042210BC08F0BABD5A9AFF1FF8D4000055
:103C3000FCD40000064B074A10B41C88064B08460B
:103C4000002C14BF11461946042210BC08F0A6BD72
:103C5000DC99FF1FF8D40000FCD40000064B074A93
:103C600010B41C88064B0846002C14BF1146194698
:103C7000042210BC08F092BD089AFF1FF8D400007F
:103C8000FCD40000064B074A10B41C88064B0846BB
:103C9000002C14BF11461946042210BC08F07EBD4A
:103CA0004C9AFF1FF8D40000FCD40000064B074AD2
:103CB00010B41C88064B0846002C14BF1146194648
:103CC000042210BC08F06ABD209AFF1FF8D400003F
:103CD000FCD4000070B5284E05460FCE86B06C4669
:103CE0000FC496E8030044F8040B2320218004F05D
:103CF0007DFC40F6B833984230DC204B40F6F502AC
:103D000019889B78ADF80D1090428DF80F302DDD9D
:103D100000EB40001A4B1B491B4E00EB0010C21772
:103D200083FB0043C2EB632381FB0314D917C1EB70
:103D3000A40101EB810186FB0040C2EB6030A3EBE4
:103D40004103303030338DF811008DF8133069465F
:103D50002846162208F022FD06B070BD0B4B1A88CB
:103D60009B78ADF80D208DF80F30D1E7084B18681F
:103D7000CDF81100EBE700BF10D5000000D5000022
:103D8000976A3E2B676666668BAA30450CD50000A5
:103D900004D50000F8B5174C174E2278174D33782C
:103DA0002F888E46003218BF012201467046FFF769
:103DB0009BFD002398423370237015DB14BF012054
:103DC00000202B889F420ED040F23A72A3F5AF73C9
:103DD0000B490C4C02FB03F381FB0312DB17A3EB33
:103DE000621332332360F8BD0749012218460A7076
:103DF0002270E6E7E48AFF1F3E9BFF1F189AFF1F11
:103E0000B5814E1B6C89FF1FA49AFF1F08B50021C6
:103E10000D2005F001F9962005F03AF901210D2059
:103E200005F0FAF8962005F033F900210D2005F091
:103E3000F3F8962005F02CF901210D20BDE808408B
:103E400005F0EAB8014B187801F0DEBF8C99FF1F2E
:103E5000144BB3F9003070B583EAE375A5EBE37555
:103E6000002BACB21ADB012300E0034603EB830016
:103E700040008542F9DA0C4E94FBF3F086FB03E533
:103E800003FB1044DB173030D3EBA503A4B201F8D9
:103E9000010BF1D105480B70106070BD2D230B7024
:103EA0000131E0E77099FF1F6766666628D500005C
:103EB000134BB3F9003030B583EAE374A4EBE37439
:103EC000002BA0B218DB012300E0134603EB8302B2
:103ED00052009442F9DA0B4D90FBF3F285FB03E4B8
:103EE00003FB1200DB173032D3EBA40380B201F8DE
:103EF000012BF1D10B7030BD2D230B700131E2E7A6
:103F0000A889FF1F67666666134BB3F9003030B5AA
:103F100083EAE374A4EBE374002BA0B218DB012363
:103F200000E0134603EB830252009442F9DA0B4D92
:103F300090FBF3F285FB03E403FB1200DB17303246
:103F4000D3EBA40380B201F8012BF1D10B7030BD8B
:103F50002D230B700131E2E76489FF1F67666666F7
:103F6000134BB3F9003030B583EAE374A4EBE37488
:103F7000002BA0B218DB012300E0134603EB830201
:103F800052009442F9DA0B4D90FBF3F285FB03E407
:103F900003FB1200DB173032D3EBA40380B201F82D
:103FA000012BF1D10B7030BD2D230B700131E2E7F5
:103FB0006A89FF1F67666666134BB3F9003030B538
:103FC00083EAE374A4EBE374002BA0B218DB0123B3
:103FD00000E0134603EB830252009442F9DA0B4DE2
:103FE00090FBF3F285FB03E403FB1200DB17303296
:103FF000D3EBA40380B201F8012BF1D10B7030BDDB
:104000002D230B700131E2E76689FF1F6766666644
:10401000134BB3F9003030B583EAE374A4EBE374D7
:10402000002BA0B218DB012300E0134603EB830250
:1040300052009442F9DA0B4D90FBF3F285FB03E456
:1040400003FB1200DB173032D3EBA40380B201F87C
:10405000012BF1D10B7030BD2D230B700131E2E744
:104060007089FF1F67666666F0B40C4D0C4F0E46F4
:104070000FCD8CB001AC0FC40FCD0FC495E8070075
:104080003B8884E807000CAA02EB8303304653F810
:104090002C1C04220CB0F0BC08F080BB64CE0000E5
:1040A0006299FF1F30B40A4B0A4D0C4693E8070093
:1040B00084B02B8804AD05E9070005EB8303204697
:1040C00053F80C1C042204B030BC08F067BB00BFDE
:1040D00090CE0000EC99FF1FF0B40A4D0A4F0E4637
:1040E0000FCD86B001AC0FC42A683B88226006AAB7
:1040F00002EB8303304653F8141C0C2206B0F0BCCC
:1041000008F04CBB9CCE0000589AFF1F054B1B8843
:104110001BB9054B186808607047044B18680860A5
:10412000704700BF7E99FF1F30D500002CD50000DE
:10413000164B1B880BB31BB230B583EAE374A4EBB8
:10414000E374002BA0B21CDB012300E0134603EB59
:10415000830252009442F9DA0D4D90FBF3F285FB95
:1041600003E403FB1200DB173032D3EBA40380B26D
:1041700001F8012BF1D10B7030BD064B18680860B7
:1041800070472D230B700131DEE700BFFA99FF1F46
:1041900067666666FCD40000164B1B880BB31BB227
:1041A00030B583EAE374A4EBE374002BA0B21CDB0C
:1041B000012300E0134603EB830252009442F9DA34
:1041C0000D4D90FBF3F285FB03E403FB1200DB17BC
:1041D0003032D3EBA40380B201F8012BF1D10B7084
:1041E00030BD064B1868086070472D230B700131F5
:1041F000DEE700BF2C9AFF1F67666666FCD40000EE
:10420000164B1B880BB31BB230B583EAE374A4EBE7
:10421000E374002BA0B21CDB012300E0134603EB88
:10422000830252009442F9DA0D4D90FBF3F285FBC4
:1042300003E403FB1200DB173032D3EBA40380B29C
:1042400001F8012BF1D10B7030BD064B18680860E6
:1042500070472D230B700131DEE700BF4099FF1F2F
:104260006766666634D50000174B1B881BB31BB20C
:1042700070B583EAE375A5EBE375002BACB21EDBEA
:10428000012300E0034603EB830040008542F9DA96
:104290000E4E94FBF3F086FB03E503FB1044DB17A3
:1042A0003030D3EBA503A4B201F8010BF1D10848DB
:1042B0000B70106070BD074B1868086070472D23A5
:1042C0000B700131DCE700BF249AFF1F676666664A
:1042D00038D50000FCD40000164B1B880BB31BB272
:1042E00030B583EAE374A4EBE374002BA0B21CDBCB
:1042F000012300E0134603EB830252009442F9DAF3
:104300000D4D90FBF3F285FB03E403FB1200DB177A
:104310003032D3EBA40380B201F8012BF1D10B7042
:1043200030BD064B1868086070472D230B700131B3
:10433000DEE700BF5099FF1F67666666FCD4000089
:10434000184B1A8852B3184A128830B50A80B3F94C
:104350000030002B83EAE374A4EBE374BCBF2D238D
:104360008B70A0B2ACBF02310331012300E01346D1
:1043700003EB830252009442F9DA0C4D90FBF3F206
:1043800085FB03E403FB1200DB173032D3EBA403FD
:1043900080B201F8012BF1D10B7030BD044B1868CD
:1043A00008607047329AFF1F3CD50000676666665A
:1043B000FCD40000174B1B881BB31BB270B583EAFB
:1043C000E375A5EBE375002BACB21EDB012300E027
:1043D000034603EB830040008542F9DA0E4E94FB5E
:1043E000F3F086FB03E503FB1044DB173030D3EB1F
:1043F000A503A4B201F8010BF1D108480B701060BD
:1044000070BD074B1868086070472D230B70013191
:10441000DCE700BF909AFF1F6766666638D500002C
:10442000FCD40000054B1B881BB9054B18680860BD
:104430007047044B18680860704700BFB299FF1FAF
:1044400044D5000040D50000054B1B881BB1054B2F
:10445000186808607047044B18680860704700BF10
:104460008E9AFF1F4CD5000048D50000F0B480EABA
:10447000E075A5EBE0750028ACB21FDB1DBF2B2358
:104480000B704E1C0E46012300E0134603EB830223
:1044900052009542F9DA0B4F94FBF3F287FB0305C8
:1044A00003FB1244DB173032D3EBA503A4B206F8AA
:1044B000012BF1D133700846F0BC70472D230B70EF
:1044C0004E1CE0E767666666054B18880C2803D02B
:1044D0000C3800B2FFF7CABF024A10680860704784
:1044E000889AFF1F50D50000024B1888183800B278
:1044F000FFF7BCBF609AFF1FC3681888183800B266
:10450000FFF7B4BF034B1888A0EB8000400000B257
:10451000FFF7ACBF8C99FF1F024B1888033800B21D
:10452000FFF7A4BFE499FF1F024B18880C3800B2B4
:10453000FFF79CBF8099FF1F30B5134C85B0012554
:104540002B463C2202212046009502F0D3FC204657
:1045500002F0AAFE00224021802320460191009310
:1045600011460A4B029503F04DFB204602F0A8FFCE
:1045700007480849084A0023036083800B608B804A
:104580001360938005B030BDAC9AFF1F08CF0000C8
:104590000C9BFF1F389BFF1F289BFF1F10B500EBD4
:1045A000C00000F10F02D2B293B284B09C1E981CDE
:1045B0003D2303918DE819003921024803F086FA62
:1045C00004B010BDAC9AFF1F70B5CEB20C460546C4
:1045D00004F0F0F8864203D03146284604F004F98E
:1045E0000135284604F0E6F8240A844205D0214625
:1045F0002846BDE8704004F0F7B870BD38B5FDF747
:10460000BDFA0D4B1B7833B90C4B10201988FFF7FE
:10461000DBFF012038BD0A4D0A4C2B782288B3FA03
:1046200083F382F008025B09114642202B7022803E
:10463000FFF7CAFF002038BD4899FF1FB899FF1F38
:10464000749AFF1FAE99FF1F024B10201988FFF7C5
:10465000BBBF00BFB899FF1F024B4E201988FFF760
:10466000B3BF00BF7E99FF1F024B44201988FFF79C
:10467000ABBF00BF609AFF1F024B2C201988FFF7C9
:10468000A3BF00BF1A9AFF1F024B1E201988FFF715
:104690009BBF00BFFA99FF1F70B55C4D2B78064693
:1046A000002B35D11C4673780BB9204670BDFDF741
:1046B00065FA574A574B5848127831781B7800787A
:1046C00002EB43034A1E03EB80030E2AEDD801A040
:1046D00050F822F06147000083470000AB4600001D
:1046E00061470000AB460000AB460000AB4600004F
:1046F0002B470000AB460000AB460000AB46000075
:10470000AB460000AB460000AB4600002747000068
:10471000AE21424802F078FB404802F0C5FD00237C
:104720002B700124BFE704F0C5FF3D4B3D491B78CA
:10473000002B3DD03C4B3D4A09881B8812680B4436
:10474000B2EB630F59DA3A4B1B78002B4BD0AF21F9
:10475000324802F059FB374A012313702B70A4E74B
:1047600083B93548038804294FF6FF7103F1FF32FE
:104770000CBF01230B46134403F07F030133038076
:104780000FE073B1013B2D4A32F813304BB12A4E82
:104790002B482C492C4A33800123002606700B70CD
:1047A0001370244A0221012311702B70204670BD22
:1047B0001D4B1E4A09881B8812680B44B2EB630F1D
:1047C000C5DB224E224D33882A88B3FA83F382F068
:1047D00002025B093380114642202A80FFF7F4FE73
:1047E000FFF714FB61E7AF210C4802F00DFB114A03
:1047F0000621012311702B7057E7164E144D338894
:104800002A88B3FA83F382F00402E2E7E48AFF1F06
:104810008A9AFF1FB499FF1F8C9AFF1FAC9AFF1F43
:104820004899FF1F5E9AFF1FEE99FF1F789AFF1F9E
:10483000A599FF1FA49AFF1F8299FF1F5499FF1F7C
:10484000759AFF1FE699FF1F149BFF1F5A9AFF1FBF
:10485000AE99FF1FDC99FF1FC3680E201988FFF770
:10486000B3BE00BF024B28201988FFF7ADBE00BFC2
:10487000E499FF1F064A07491388098823F00203B9
:1048800043EA41039BB2194642201380FFF79CBEC6
:10489000AE99FF1F5A9AFF1F064A074913880988D5
:1048A00023F0040343EA81039BB21946422013809C
:1048B000FFF78ABEAE99FF1FDC99FF1F064A074922
:1048C0001388098823F0100343EA01139BB21946A9
:1048D00042201380FFF778BEAE99FF1F089AFF1F92
:1048E000064A07491388098823F0200343EA411345
:1048F0009BB2194642201380FFF766BEAE99FF1F98
:104900004C9AFF1F024B5A201988FFF75DBE00BF6B
:104910007099FF1F024B16201988FFF755BE00BF84
:104920004099FF1F024B2E201988FFF74DBE00BF94
:10493000249AFF1F024B30201988FFF745BE00BFA5
:104940005099FF1F024B18201988FFF73DBE00BF8A
:10495000EC99FF1F024B1A201988FFF735BE00BFE4
:10496000329AFF1F024B1C201988FFF72DBE00BF93
:10497000589AFF1F024B20201988FFF725BE00BF61
:10498000909AFF1F024B32201988FFF71DBE00BF0F
:10499000889AFF1F024B52201988FFF715BE00BFEF
:1049A000A889FF1F024B50201988FFF70DBE00BFDA
:1049B0006489FF1F024B54201988FFF705BE00BF12
:1049C0006A89FF1F024B5C201988FFF7FDBD00BFFD
:1049D0006689FF1F024B5E201988FFF7F5BD00BFF7
:1049E0007089FF1F024B60201988FFF7EDBD00BFE3
:1049F000B299FF1F024B56201988FFF7E5BD00BF93
:104A00008E9AFF1F38B5054603F0D4FE4FF0000420
:104A100060F30704681C03F0CDFE60F30F24A0B21E
:104A200038BD00BF38B5094D46242046FFF7EAFFE0
:104A300035F8021B00B28842204601D0FFF7C4FDC2
:104A40000234E4B24E2CF0D138BD00BF509AFF1FA3
:104A500008B51220FFF7D6FF054B1988884206D00B
:104A60001220FFF7B1FDBDE8084001F04DB908BDC7
:104A70006299FF1F08B55820FFF7C4FF054B19883E
:104A8000884206D05820FFF79FFDBDE8084001F09E
:104A90003BB908BD2C9AFF1F08B51420FFF7B2FFE1
:104AA000054B1988884206D01420FFF78DFDBDE81C
:104AB000084001F029B908BD209AFF1F014B0122CF
:104AC0001A7070473E9BFF1FF0B585B003F02AFEB9
:104AD0004D4C4E4B02934E4A0192042300932046C4
:104AE0004C4B4D4F4D4E4E4D4022802102F00AF866
:104AF00020464C4C4C4A4D4907F070FAA7614C488F
:104B00004C4FE7614C4F87614C494D4FC7614D4F4A
:104B10008F614D4A4D4FCF614D4F97614D4B4E4F79
:104B2000D7614E4F9F614E4FDF614E4FB7614E4F81
:104B3000F7614E4FAF614E4C4E4FEF614E4FA76144
:104B40004E484F4FE7614F4F87614F494F4FC76105
:104B50004F4F504A8F61504FCF61504F504B97612C
:104B6000504FD761504F514E9F61514FDF61514FB0
:104B7000514DB761514FF761514F524CAF61524F98
:104B8000EF61524F5248A761524FE761524F53496C
:104B90008761534FC761534F8F61534A534FCF6162
:104BA000534F9761534B544FD761544F9F61544EAD
:104BB000544FDF61544F554DB761554FF761554F15
:104BC000554CAF61554F56485649EF61564F574DBA
:104BD000A761E561564F574D574CDFF880E1574AC2
:104BE000574B8761C5618C61564E574F574D584C96
:104BF000C1F81CE0574858499761D5619C61D8615C
:104C0000B16005B0F0BD00BFAC9AFF1FA0860100E7
:104C1000801A0600388EFF1F29450000D48BFF1F25
:104C2000D88DFF1FF88BFF1F1C89FF1F5D6B0000D5
:104C3000C08AFF1F5948000019450000FC8AFF1F69
:104C4000654800000D3C0000908DFF1F7548000076
:104C5000353C00001C8CFF1F994800005D3C0000A3
:104C6000BD480000853C0000E1480000054500000B
:104C7000108DFF1F453E000069400000448BFF1F60
:104C8000514A0000994100008C8BFF1F754A0000BB
:104C9000513E0000E889FF1F05490000AD3C0000BF
:104CA000B48DFF1F994A000001420000688BFF1F6E
:104CB00015490000694200003C8AFF1F2549000099
:104CC000D9420000208BFF1F35490000A54000009D
:104CD0009C8AFF1F4549000041430000648CFF1F70
:104CE00055490000D9400000B08BFF1F6549000006
:104CF000B54300004C8DFF1F75490000C9440000FA
:104D0000608AFF1F85490000B13E00000C8AFF1F2A
:104D100095490000093F0000C489FF1FA549000014
:104D2000C88CFF1FEC8CFF1F613F0000B5490000DD
:104D3000B93F0000C549000011400000FC8DFF1F75
:104D4000408CFF1F308AFF1F25440000E54900000A
:104D500049440000F5490000E5500000D549000035
:104D60002DE9F04F2F4DDFF8CCB0DFF8C4A0DFF80D
:104D7000C8900FCD91B003AC0FC40FCD0FC40FCDB1
:104D80000FC42B6823600025A8462F462E4600E05E
:104D90009846BAF8003024495BF8232028461123AE
:104DA000FBF73CFF00EBC00400EB840089FB003400
:104DB0000444C017C0EB6434C4F13C00C6F13C02AB
:104DC00007F14101012600B208F1410300901BB236
:104DD000019612B209B2154802F0BEFD08EB0603B7
:104DE00005F211153C2B2646ADB24746D0D13422F0
:104DF0006B210E4803F042F900210C4803F042F900
:104E00000B4B1B8810AA02EB830353F8344C20464B
:104E100007F056FC02460548214611B0BDE8F04FA8
:104E200003F030BAB0CE0000A4CB0000AC9AFF1F54
:104E30001A9AFF1FC4CC0000090002802DE9F0433C
:104E4000804685B0002956D10121304803F01AF977
:104E50002F4998F8062098F8083011F802909945E3
:104E600022DA4FEA89064D460C24D8F80C30274840
:104E70009B595F6822B2002103F000F9384607F021
:104E80001FFC39460246214803F0FCF91F4803F095
:104E90000FFA98F8083001350934AB42A4B206F194
:104EA000040601DD422CE0D1B9F1000F13D109F164
:104EB000060999450CDA3C2301213B220391029318
:104EC0000093019239233F223A21104802F0FEFD5F
:104ED00005B0BDE8F0830F2301213B22039102932B
:104EE0000093019239230C223A21084802F0EEFD8A
:104EF00098F80830DBE700213423009301913F2329
:104F00000C22024802F0F6FC9EE700BFAC9AFF1F9D
:104F1000389BFF1F10B5154C0121204603F0B8F84F
:104F20002046012103F0AEF8204600220F2103F0B5
:104F3000A5F8204602220E4903F0A4F920463422A7
:104F4000552103F09BF8204602220A4903F09AF902
:104F500020460522084903F095F9204603F0A8F9F8
:104F60002046BDE8104002F0ABBA00BFAC9AFF1F6C
:104F700054D5000058D500005CD5000070B50D4632
:104F8000064607F09DFB00EB40008400002D36D064
:104F9000284607F095FB00EB4000400023185B100B
:104FA00003F16001091A282209B21748C3F160040D
:104FB00003F064F80121144803F064F8284607F070
:104FC0007FFB29460246104803F05CF90E4803F0C7
:104FD0006FF902210C4803F055F821B221220A484A
:104FE00003F04CF8304607F06BFB314602460648AA
:104FF00003F048F90448BDE8704003F059B9641063
:10500000C4F16004E5E700BFAC9AFF1F214B70B507
:10501000B3F9003083EAE374A4EBE374002B82B0AD
:10502000A1B22FDB68466D46012300E0134603EB77
:10503000830252009442F9DA174E91FBF3F286FB99
:1050400003E403FB1211DB173032D3EBA40389B264
:1050500005F8012BF1D119462B70FFF78FFF0F4B8D
:105060001B786BB101210E4803F00CF83322742138
:105070000B4803F003F801220A49094803F002F93A
:1050800002B070BD2D238DF800300DF1010568468A
:10509000CAE700BFB899FF1F67666666749AFF1F6C
:1050A000AC9AFF1F4CD7000010B50D4B1B5C51F89C
:1050B0002340237884B013B1012004B010BD04AAAA
:1050C00001A942F8103D2046A3699847A38A9B078F
:1050D000F2D401A80099FFF751FF012004B010BDE0
:1050E0000C9BFF1FF8B51F4D287840B91E4B1B685D
:1050F000994203D31D4A012313702B70F8BD0C464F
:1051000000261B48184F02F0CFF804F6B833324699
:1051100017483B6031212E7002F0B0FF0121144886
:1051200002F0B6FF3146124802F0ACFF05221149E9
:105130000F4803F0A7F80E4803F0BAF80C2210212C
:105140000B4802F09BFF0B220B49094803F09AF829
:1051500005220A49064803F095F8054803F0A8F827
:105160000120F8BDE48AFF1F249BFF1FA49AFF1FA4
:10517000AC9AFF1F64D500006CD500005CD5000020
:1051800010B5424C424882B002F08EF82378C3B981
:1051900006213F4802F076FF2378012B37D90A22F7
:1051A000022B11463A486BD002F068FF39490322BE
:1051B000374803F067F8364802B0BDE8104003F006
:1051C00077B8354B1A7801210523002A35D1019192
:1051D000009311462E4802F00FFC304B1A78002A3B
:1051E00036D0052301220192009300220A2128488B
:1051F00002F080FB2A4B1A78002A35D101210523C1
:10520000019100931421224802F0F6FBC0E7254CDF
:105210002388092B32D9632B8CBF0A211F210A2234
:105220001B4802F02BFF2188194803F091F8184819
:1052300002B0BDE8104003F03BB80022019100939A
:105240001146134802F056FB144B1A78002AC8D1B5
:1052500005230121019100930A210D4802F0CCFBA6
:105260000F4B1A78002AC9D001220523019200931E
:1052700000221421064802F03DFB89E73021CEE7E9
:1052800002F0FCFE0322084992E700BF149BFF1FB7
:10529000AC9AFF1F7CD500008A9AFF1FB499FF1FAC
:1052A0008C9AFF1F8299FF1F78D500002DE9F041ED
:1052B000754C2278002A05460F4614BF4FF00108AE
:1052C0004FF000084ED1714E3368CB1AB3F5FA6F28
:1052D00004D86B78A3B94046BDE8F0816C4B6D48AB
:1052E0006D49DFF8D0E11A7001230370098823703B
:1052F00026208EF80020FFF767F96B78002BEAD0A4
:105300003760FCF73BFC654A654B664912782878A4
:105310001B78097802EB4303421E03EB81030E2A3C
:10532000D9D801A151F822F019540000E55300002A
:10533000D752000019540000D7520000D752000085
:10534000D7520000CD530000D75200007F53000019
:10535000D7520000D7520000D7520000D7520000A9
:105360007B530000AF215048484E01F04DFDFFF740
:1053700007FF002337602370ABE704F09BF94A482E
:1053800001F092FF0221484802F07CFE0F22232107
:10539000454802F073FE05224449434802F072FF7B
:1053A000414802F085FF1E2223213F4802F066FE9D
:1053B00005223F493C4802F065FF3B4802F078FF78
:1053C000394802F07DF800F0ABFC84E7394D2B78CA
:1053D000012B50D9304B26201988FFF7F5F8002310
:1053E0002B7078E7002B3FF476AF013B324A32F85E
:1053F0001330002B3FF46FAF274C304825492D4A1E
:1054000023804FF001080023037081F8008082F8A8
:105410000080FFF7B5FE5EE793B1013B264A32F804
:10542000131019B31C4B254D1A4C224A1980002623
:10543000012326202E7023701370FFF7C5F815E0A6
:10544000154C1E4922880B7004284FF6FF7002F19C
:10545000FF310CBF012202460A440E4E154D02F0E8
:105460007F0201320121228031702B70FFF788FE0C
:105470004FF001082FE70649064A01230020087073
:1054800013702370A6E700BFE48AFF1F349BFF1F41
:10549000A49AFF1FE699FF1F8299FF1F8A9AFF1F98
:1054A000B499FF1F8C9AFF1FAC9AFF1F80D5000094
:1054B00088D50000149BFF1F5499FF1F759AFF1F8A
:1054C0002DE9F04F05468BB00F46AD480121164639
:1054D00002F0DEFDAA8812F0010440F0B180DFF88E
:1054E000CC8298F80030002B7ED1AB79A54AD15CF4
:1054F000A1B9DFF8BCA279781AF8039041B33978E2
:105500000139072900F2B880DFE811F0F2005401F8
:10551000B6006C01B600B600B600EA007C78002C3C
:1055200000F0CB800139EC68387854F82170FC68C1
:10553000411EB4F80080072900F2A880DFE811F0CE
:1055400074015901A6006C01A600A600A600A000E7
:10555000DFF854A2DAF80020B21AB2F5967F76D9B5
:10556000894A107801281ABF012010701170874AEB
:1055700018BF0146D05CC0EB0900C0B2FFF70EF8BF
:105580000124CAF80060AB889B0771D57B78002B9B
:105590006ED0FCF7F3FA7E4B7E4A7F481B78127878
:1055A00039780078022515FB02330A2903EB8003C2
:1055B00000F04E810C295BD1002B59D003F119006A
:1055C000764E774A013B0021400000F0FE0026F8AD
:1055D00013100123157088F80030FEF7F5FF714BAA
:1055E000032220461A702FE0654801F05DFE01217C
:1055F000634802F047FD62482246214602F03EFD24
:10560000AB88580725D42C68204607F059F8214666
:1056100002465B4802F036FE594802F049FE092274
:1056200001238DE80C0000217F23554802F094F9F6
:1056300000212846FFF702FC002388F8003054E7D9
:10564000AB683146384698470BB0BDE8F08F084646
:10565000FAE72B6804A8984704A807F031F804A9D2
:105660000246474802F00EFE454802F021FED6E70A
:1056700020460BB0BDE8F08F00240AF8039082E7C3
:105680000021D1543846FB699847FC68A4F8008093
:10569000002725223C238DE8840041211822384828
:1056A00002F028F9E968A879FFF7FEFC364A3E4B7C
:1056B00017701E600BB0BDE8F08F3B490A68B21A44
:1056C000B2F5967FD4D9304F0E603E78012E00F0AF
:1056D000B380E968184601233B70FFF7E5FCB3E7A8
:1056E0002F4AE9791170012288F800200024C4E7CC
:1056F0002A7A013A4A45BFDD09F10106F6B2B14501
:10570000BAD0224A039212F803B0CBEB0900C0B220
:105710000021FEF743FF2B7A052B5C461BD9CBEB10
:1057200006010429039A40F3AB80A6F1040BBBF1F8
:10573000000FC0F2AD80063B9B45A8BF9B465FFAB9
:105740008BF4AB791148D25C5A4504D0C454012182
:105750002846FFF773FB301BC0B201210A4CFEF74D
:105760001DFF00213423019100930548217040233F
:105770000B223F2102F0BEF8B1460124AB797CE751
:10578000AC9AFF1F289BFF1F209BFF1F389BFF1F0A
:105790008A9AFF1FB499FF1F8C9AFF1F5499FF1F0D
:1057A000A49AFF1F149BFF1F1C9BFF1FE48AFF1F6F
:1057B0000C9BFF1F0FFA89F1E8685F4C50F82160DD
:1057C0002168049134785D4904980860002C70D0F9
:1057D000012C7FF451AF5A4A317A88F80040117099
:1057E00000244AE7B9F1000F50D009F1FF36F6B2B4
:1057F00085E7B98A01F0040189B200293FF441AF7D
:105800003B6A03929847039A00283FF43EAFAB7976
:10581000FC680021D15439E77B8A43453BD908F124
:1058200001081FFA88F831E73B8A43453AD208F16C
:10583000FF381FFA88F829E725238DE8180041482A
:105840003C703C231822412102F054F83046FBE61C
:10585000002B3FF40DAF3C4A3C4E1188384A5F1E86
:105860001933580000F0FE00012388F8003026F8B4
:1058700017101570FEF7A8FE354B20461D70E3E6A5
:1058800000293FF758AF06F1FF3B50E74C46F4E6DE
:105890000024A34655E7BB8ADA077FF5F7AEB7F8D1
:1058A0001080F3E6BB8AD9077FF5F0AEB7F8128017
:1058B000ECE62849C85CC0EB090009F1010EC0B252
:1058C00001214FF0340B02F803E0FEF767FEB668E3
:1058D0001C48019440230B223F210124CDF800B045
:1058E00002F008F840230B223F211648CDF800B003
:1058F000019402F081F82146124802F0C3FB3046C1
:1059000006F0DEFEA0EB800000F15F0109B20F227D
:105910000C4802F0B3FB304606F0D2FE3146024698
:10592000084802F0AFFC074802F0C2FCE968A87919
:10593000FFF7BAFBAB79A0E66C9BFF1F1C9BFF1F18
:10594000A49AFF1FAC9AFF1F8299FF1F5499FF1F53
:10595000149BFF1F389BFF1F2DE9F047DFF80892CB
:105960006D4B99F800601B68DFF800A282B000362A
:1059700001934FF0030018BF0126019F9AF80080A1
:1059800003F050FB0546042003F04CFB04460520C1
:1059900003F048FB800040EA4404062003F042FB89
:1059A0002C4364B25D4944EAC0000A7880F00F03DA
:1059B000DBB29A425A4A3CD01760002259480B7019
:1059C00003788DF800808DF8012053B3564A126891
:1059D0004EF66021BA1A8A4219D8022B59D0012BEF
:1059E0005FD0062B48D0032B63D0042B69D0052B46
:1059F00077D0072B7DD0082B00F08380092B68D04F
:105A000016B14A4801F05CFD02B0BDE8F087484A93
:105A1000484C00230121237003701360938089F8A0
:105A200000103A4669464448FFF74AFD3043C6B283
:105A3000E6E71268BA1A1E2A6BD99AF80020934238
:105A400022D0394C3D488AF80030012B276082EA89
:105A5000030207609846B1D0042BAFD137480068E5
:105A6000381AB0F5C87FA9D9354C2068381A3228C1
:105A7000A4D927601A46A1E73A4669463148FFF79C
:105A80001FFD3043C6B2BBE7012B4FF00002E3D14C
:105A9000E4E73A4669462C48FFF712FD3043C6B2A8
:105AA000AEE73A4669462948FFF70AFD3043C6B2D9
:105AB000A6E73A4669462648FFF702FD3043C6B2DC
:105AC0009EE73A4669462348FFF7FAFC3043C6B2E0
:105AD00096E73A4669462048FFF7F2FC3043C6B2E3
:105AE0008EE73A4669461D48FFF7EAFC3043C6B2E6
:105AF00086E73A4669461A48FFF7E2FC3043C6B2E9
:105B00007EE73A4669461748FFF7DAFC3043C6B2EB
:105B100076E7002252E700BF6C9BFF1F2E9BFF1F02
:105B2000A09AFF1FA49AFF1F189BFF1FAC9AFF1F8C
:105B3000289BFF1F129BFF1FDCD40000309BFF1F20
:105B4000A89AFF1F24D400008CD3000014D40000B6
:105B500038D3000044D4000034D40000E8D400005E
:105B600078D40000308AFF1FE48AFF1F139BFF1FB9
:105B700028B11028044BA8BF102018607047024BB2
:105B800001201860704700BF409BFF1F38B50F4DC4
:105B90002B78013B01381B02C4B203F4706320046C
:105BA00043F4404343F00C0300F4FE00184304F0B8
:105BB000A1FB2868013860F03F00C0B203F0C8FBC9
:105BC0002046BDE8384003F0C3BB00BF409BFF1F29
:105BD00070B5124D2B78013B1B0203F4706306462F
:105BE00043F430430806320400F0FE4043F00B0358
:105BF000034302F4FE0018430C4604F07BFB2868C4
:105C0000013860F04F00C0B203F0A2FB304603F051
:105C10009FFB2046BDE8704003F09ABB409BFF1FEE
:105C200070B5124D2B78013B1B0203F470630646DE
:105C300043F410430806320400F0FE4043F0090329
:105C4000034302F4FE0018430C4604F053FB28689B
:105C5000013860F06F00C0B203F07AFB304603F009
:105C600077FB2046BDE8704003F072BB409BFF1FEE
:105C700038B5104D2B78013B1B0203F470630446CA
:105C800043F41043000443F0090300F4FE001843FA
:105C900004F030FB2868013860F06F00C0B203F0F8
:105CA00057FB204603F054FB0020BDE8384003F0CA
:105CB0004FBB00BF409BFF1F38B50E4D2B78013BFB
:105CC0001B0203F47063044643F45043000443F0A2
:105CD0000D0300F4FE00184304F00CFB28680138A3
:105CE00060F02F00C0B203F033FB2046BDE838401F
:105CF00003F02EBB409BFF1F08B5002004F05EFBA5
:105D00000028FAD108BD00BF08B564210720FFF7BD
:105D10005FFF7F210B20BDE80840FFF759BF00BFA0
:105D200010B500217B20FFF753FF0024E0B2FFF7FE
:105D30009FFF0134022003F0ABF9802CF6D110BD97
:105D400010B504464FF4406003F0B2FA03F00AFBCA
:105D50002CB1102C044BA8BF10241C6010BD024BAA
:105D600001241C6010BD00BF409BFF1F10B50446FE
:105D700041F0E00003F0ECFA04F07F0003F0E8FAF1
:105D8000C4F3C610BDE8104003F0E2BA38B5134DB5
:105D90002B78044641F6FF72A0F50050824203F1D1
:105DA000FF33A8BF02461B0202F5005203F47063E2
:105DB000100443F4604343F00E0300F4FE00520469
:105DC000184302F0FE42104304F094FA29680139A6
:105DD0002046C9B2BDE83840FFF7C8BF409BFF1F4F
:105DE00038B504460D46F02003F0B2FA35B125442B
:105DF00014F8010B03F0ACFAAC42F9D1F720BDE87E
:105E0000384003F0A5BA00BF00B50B4B83B0024683
:105E1000998818680090032AADF8041002D903B0DD
:105E20005DF804FB684606218DF80520FFF7D8FFD2
:105E300003B05DF804FB00BF14D8000000207047D9
:105E400090F8392090F83800101A704790F83830E0
:105E500090F839209A4205D95A1C034480F838201A
:105E6000187E70474FF0FF30704700BF90F8383011
:105E700090F839209A4286BF1B18187E4FF0FF30E9
:105E8000704700BF704700BF38B50546B0F85E00E8
:105E900090B195F85D301446C3F1210294420CD8BC
:105EA00005F13B001844224602F0CEFC95F85D3027
:105EB000234485F85D30204638BD01201446287102
:105EC000EEE700BFB0F85E306BB190F85D30202B8C
:105ED00007D8C218013380F85D30012082F83B10EA
:105EE0007047012303710020704700BF00234269FF
:105EF00080F8383080F8393080F85C3080F85D30D8
:105F000080F85E3080F85F3006CA30B40D680469EE
:105F100043662A4383660A60A370426990F8613041
:105F20001649146813441D7A5B7B01EBC5051B02FF
:105F30006D6803F4E06343F064032B6090F8623013
:105F400013449D7CDB7D01EBC5011B02496803F412
:105F5000E06343F064030B6021685368194205D085
:105F6000036927225A70036904229A710369202267
:105F70005A71036980229A7030BC704748E3000070
:105F800043690CCB12681A420CD0094B99420AD9CA
:105F9000084B9942036994BF1A220D225A70036973
:105FA00004229A717047036927225A70F7E700BFED
:105FB0007F1A06003F420F0010B50269D378DBB2AA
:105FC000D90604463DD510215806D17038D503F0C6
:105FD000040303F0FF02002B51D03D49626E002301
:105FE0000B7084F85D30002A5BD0904794F85D30E8
:105FF000002B56D02369D0229A70236994F83B2055
:106000001A712369012284F85C200222DA7010BD23
:10601000304B84F860009C424AD02F4B9C4252D0B7
:1060200094F8391013791F29DBB207D82848007873
:1060300020B16018013184F8391003760223D3703F
:1060400010BD5906C3D4917801F0100101F0FF0092
:106050000029DDD013F001031ED194F85C1094F8F0
:106060005D00884281BF4B1C091984F85C3091F8AF
:106070003B3013712369D0229A702269DEE72369CD
:1060800084F83920C0229A702369114A19790121B4
:1060900011700222DA7010BDC02393702269137947
:1060A000CCE70122002384F85D2084F83B30A1E78F
:1060B000626994F86130094913440322187A02F0A6
:1060C00049FD2269ACE7626994F861300449F3E75D
:1060D000449BFF1F388EFF1FA48EFF1F41610000ED
:1060E0004D6100000369DB7803F0200373B190F881
:1060F00060300133DBB2012B80F860301AD942697D
:1061000090F861301344187A02F0A0BD70B542696E
:1061100003F0FF0590F8613013440446187A02F04A
:1061200095FDA36E5BB184F8385094F83900BDE852
:106130007040184790F85F30002BE0D0704770BD7A
:106140000148FFF7CFBF00BF388EFF1F0148FFF7A0
:10615000C9BF00BFA48EFF1F2DE9F047374FDFF8FE
:10616000E0903B68026982B006460093DDF800804B
:106170000021A025D3789B065BD53B680193019B4A
:10618000C8EB03030F2BF5D949B1102BF2D0002037
:106190009070336980229A7002B0BDE8F08772690E
:1061A00096F8613013440521187A02F049FF7269AC
:1061B00096F861301344012193F812A0504602F082
:1061C0003FFF09240021504602F026FF2B46013BE9
:1061D000FDD10121504602F01FFF2B46013BFDD1AE
:1061E000013CEFD1706996F8611001444FF4A07240
:1061F0000C7A4B7B09EBC4011B02496803F4E06392
:1062000043F064030B6096F862300344997CDB7DB5
:1062100009EBC1011B02496803F4E06343F0640326
:106220000B60013AFDD13269D3789B064FF0010132
:10623000A3D4012002B0BDE8F08700BF6C9BFF1F14
:1062400048E30000F0B503691222DA70026993781E
:1062500003F0200385B004460D46002B5ED0B42326
:1062600093703C4922690B680093009E05E00B681F
:106270000193019B9B1B042B42D8D37803F020038E
:1062800003F0FF00002BF2D094F85D30002B31D0EA
:106290004FF0000E4FF0020C04EB0E0393F83B306E
:1062A00013710B680393039F206907E09B060DD5CC
:1062B0000B680293029BDB1B052B28D8C378DBB24B
:1062C00003F0020202F0FF06002AEFD080F803C0BC
:1062D0002669F378DBB2DF0632462DD49F062BD534
:1062E000DB0731D40EF1010E94F85D305FFA8EFEBB
:1062F0007345D1D800201DBB002384F85E3004E034
:106300009070236980229A70042005B0F0BD8670D9
:106310002369802204209A7005B0F0BD03F0FF06C7
:10632000FFF71AFF10B9042005B0F0BD236984F807
:106330005F60B0229A7094E78023B3700420DAE79C
:1063400026698023B370D7E7BEF1000F0CBF02208F
:106350000320F6E76C9BFF1F2DE9F041066900253D
:10636000122780F8385080F83950F770D0F810C0F4
:106370009CF802E00EF0200E88B0044688461546D0
:106380001E46BEF1000F49D0B4238CF80230784B82
:1063900021691A680092DDF800E006E01A680192AF
:1063A0000198CEEB0000042830D8C87800F0200017
:1063B00000F0FF070028F1D04FEA480242F0010246
:1063C000D2B20A711A680292DDF808E0206906E08C
:1063D0001A6803920399CEEB010105292AD8C178E6
:1063E00001F0020101F0FF070029F1D04FF0020C8B
:1063F00080F803C02269D17811F0110722D12DBB9A
:10640000002E0CBFA0238023937003E08F702369BC
:1064100080229A70384608B0BDE8F0810EF0FF0780
:10642000FFF79AFE0028F5D0236984F85F70B02248
:106430009A70ACE787702369802238469A7008B05A
:10644000BDE8F081802393700027E3E7012D75D02C
:10645000A021917021690A79BE4667464FF0A80CC9
:106460001A680492049805E01A680592059A121AAF
:10647000052A4AD8CA7802F0020202F0FF08002A70
:10648000F2D0CF702169CA78D2B212F0100F08464C
:106490005AD1920658D5013DEDB2012D49D0BEF139
:1064A0001F0F3BD90A79012DDAD11A680692069D91
:1064B00005E01A680792079A521B052A46D8C27847
:1064C00002F0020202F0FF01002AF2D00223C370A0
:1064D0002269D378DBB2D9063AD49B0634D5B023EF
:1064E000BEF11F0F93703FD8226904EB0E0312799F
:1064F0001A760EF1010E5FFA8EFE16B12369802224
:106500009A7084F839E0774684E781F8028023693D
:1065100080229A70774684F839E07BE704EB0E021C
:1065200091F8048082F818800EF1010E5FFA8EFE59
:10653000B9E781F802C021690846B0E7A821917047
:106540002069BE460279B0E7774663E78170DEE7EF
:106550001021A023D170013BFDD12269937803F073
:10656000F7037746937055E723691B79C5E700BFAA
:106570006C9BFF1F0148FFF71FBD00BF388EFF1F38
:106580000148FFF719BD00BFA48EFF1F704700BF71
:1065900038B5144C037801225B000546204684F888
:1065A0003B3084F85E2084F85D20FFF78BFC2046AA
:1065B0000021FFF747FE0B4C2978012320461A469D
:1065C000FFF7CAFE0128F6D194F8383094F8392044
:1065D0009A4205D9E218013384F83830107E38BD6C
:1065E000FF2038BD388EFF1F38B51B4C03780122C1
:1065F0005B000546204684F83B3084F85E2084F832
:106600005D20FFF75FFC20460021FFF71BFE124CC8
:106610002978204601230222FFF79EFE0228F6D1A8
:1066200094F8382094F839108A420FD2531CDBB208
:10663000A018994284F83830007E0AD923440232E7
:106640001B7E84F8382040EA032038BD4FF6FF70E7
:1066500038BD40F47F4038BD388EFF1F0C2901D96A
:10666000002070470231490001F0FE01FFF7BCBF76
:1066700070B50C4C0378164601255B00204684F863
:106680003B3084F85E5084F85D50FFF71BFC3146C8
:106690002046FFF717FC29462046BDE87040FFF76B
:1066A000D1BD00BF388EFF1FF8B505460F46164610
:1066B000412421463A462846FFF7DAFF611C02349E
:1066C000C9B232462846E4B2FFF7D2FF592CF0D1C6
:1066D000F8BD00BF38B504460D463548FFF706FC47
:1066E0006322802120462570FFF7C2FF012002F0BF
:1066F000CFFC204600225E21FFF7BAFF20465D2135
:10670000FFF746FF242801D0002038BD204606228E
:106710000C21FFF7C9FF204601222B21FFF7A8FF1C
:10672000204601222C21FFF7A3FF20460E222D2117
:10673000FFF79EFF204600222E21FFF799FF2046FB
:1067400001222F21FFF794FF204605223021FFF779
:106750008FFF204601223121FFF78AFF20460022C9
:106760003221FFF785FF204600223321FFF780FF0B
:10677000204600223421FFF77BFF204600223521EE
:10678000FFF776FF204600225B21FFF771FF2046CE
:1067900010225C21FFF76CFF204620225D21FFF7CD
:1067A00067FF20468F225E21FFF762FF012038BD80
:1067B000388EFF1F10B4047F4160022CC26002D0EB
:1067C00010BC01F073BC836810BC184790E80C0043
:1067D000F0B41C6859682568164F174E294321608C
:1067E000164D17491760D66015611160417A154A38
:1067F0005C180A3194F8244053F8215002EBC4018C
:1068000049680D60017A5C1803EB8101247ECD6933
:1068100002EBC40149680D60817A581803EB8103CB
:1068200090F83000596B02EBC002F0BC536819605D
:10683000704700BF01401F000110003801100078B0
:1068400000001F8048E3000038B504461046217060
:106850000A491D4605F0B6F901464FF07E5005F095
:1068600065FA074905F0AEF9E5606060256165618C
:1068700002F0ECFBE061204638BD00BFDB0FC940F1
:106880000024744938B504461046217009491D4654
:1068900005F098F901464FF07E5005F047FA064999
:1068A00005F090F9E56060602561656102F0CEFB5E
:1068B000E06138BDDB0FC9400024744938B5037866
:1068C0000446032B20D8DFE803F01A181002C16831
:1068D000406905F06DF80D490546606805F026FA37
:1068E0000146284605F022FA38BD0849406805F0FF
:1068F0001DFAE16805F066F938BDC06838BDC168A9
:10690000406905F055F838BD002038BD00247449B1
:1069100070B504460E4602F099FB0546E069281A58
:1069200005F0FCF8E3682361E5616661A06101465A
:10693000606805F0FBF90146A060104805F0F6F923
:1069400004F0CCFC04F06CF904F0DEFF05460146CF
:106950004FF07E5005F02CF8616905F033F921699C
:106960000646284605F02EF90146304605F022F885
:10697000E0602046BDE87040FFF7A0BF000080BF88
:10698000704700BFF0B50C1EBDF8146034DBB0F9E1
:1069900006701919B942C4BF3B1B1BB2002BA64697
:1069A0001CDD002A1146B8BFD11D02F00705CC102E
:1069B000826A012007FB04E1A840012E0A44C0B20C
:1069C0001ED00CD3022E09D1013B12FA83F3013AF7
:1069D00012F8011F41409A421170F9D1F0BDC04335
:1069E000013B12FA83F3C0B2013A12F8011F0140D1
:1069F00093421170F9D1F0BD23441BB20024C6E7C5
:106A0000013B12FA83F3013A12F8011F01439A4243
:106A10001170F9D1F0BD00BFF8B50D1E0EDB1446A4
:106A20001F46064601F03AFBA84207DD002C05DBB5
:106A3000304601F037FBA04201DCF8BDF8BD30461E
:106A400001F02AFB022853D003284BD0012806D19D
:106A50006540F3886C406540013B5D1B2DB2012F02
:106A600003D02AD3022F14D0F8BD002C2246B6F949
:106A70000630B06AB8BFE21D42F3CF0202FB0355F5
:106A800004F00704435D012101FA04F41C4344555A
:106A9000F8BD002C2246B6F90630B06AB8BFE21D38
:106AA00042F3CF0202FB035504F00704435D0121CA
:106AB00001FA04F45C404455F8BD002C2246B6F9B6
:106AC0000630B06AB8BFE21D42F3CF0202FB0355A5
:106AD00004F00704435D012101FA04F423EA0404ED
:106AE0004455F8BD3389013B591B25460CB2B6E726
:106AF000F18832890139013A4D1B141B2DB224B2A1
:106B0000ADE700BF2DE9F041079E9DF91880089D73
:106B100004461F4600F0C0FF0D4B0E480E4984F896
:106B20003380FF22002F08BF1F4684F82F20002348
:106B300084F8302084F8312084F832202060A66563
:106B4000E565676261652362A3622046BDE8F08166
:106B5000388EFF1FA0D800000110013810B5044680
:106B6000806A034B236008B105F07AFA204610BD15
:106B7000A0D80000F8B5436ADBB190F82C200125BD
:106B8000AA4083F83B2083F85E5083F85D500446AA
:106B9000406A03680E461B6800219847606A0368D4
:106BA00031461B6898472946606ABDE8F840FFF700
:106BB00049BBC26BC56C1368046A23EA0503136002
:106BC0004CB122684FF00043D3625163D36A002B6B
:106BD000FCDA936BF8BD836B466B0825802410E0CC
:106BE0003768426C3A4332601F68826C3A431A60DD
:106BF0001A68876C013D22EA07024FEA54041A60C2
:106C000007D02142ECD13268476C22EA0702326099
:106C1000EAE7F8BD70B50446406A0D4600282BD05F
:106C2000A16DFFF7ADF9002D20460CBFA621A721CD
:106C3000FFF7A0FF606A20B1E16DBDE87040FFF78B
:106C40009FB9216C226D0868236A02430A6093B1E0
:106C5000DA7A82B1D00703D5224A99691160DA7ACB
:106C6000910703D5204AD9691160DA7A520702D513
:106C70001E4A1B6A136070BD236A002B2BD0D97A81
:106C8000626DE1B172B6D97ACE0706D51848D968D7
:106C90000668314099610160D97A880706D51548A0
:106CA000196906683140D9610160D97A4E0705D566
:106CB00011485969066831401962016062B61B6863
:106CC000D968914207D00D4818600D49DA6042F04A
:106CD000804018611960226C216D136823EA01035A
:106CE0001360A0E700E100E004E100E008E100E05B
:106CF00080E100E084E100E088E100E001403F0045
:106D000000003F80436A2DE9F04105460E4690465B
:106D1000002B3ED090F82C100124A14083F83B10AA
:106D200083F85E4083F85D40406A036800211B6879
:106D300008F1FF379847FFB2B8F1000F23D037446E
:106D4000A046013E686A16F8011F03681B68984751
:106D50000134B742E4B216D0202CF3D10121686A85
:106D6000FFF770FA95F82C206B6A520083F83B20ED
:106D700083F85E8083F85D80686A036800211B6881
:106D800098470124DEE7686A0121BDE8F041FFF77A
:106D900059BAC26BC16C136823EA010306EB0804FD
:106DA00013604FF00048A6420ED02B6A16F801EB94
:106DB00063B11A68C2F82C80C2F834E0D36A002BA1
:106DC000FCDAA642936BF0D1BDE8F081AB6BD5F84D
:106DD00034C008208021DCF800206F6C1EEA010F0F
:106DE00014BF3A43BA43CCF800201A68AF6C3A4358
:106DF0001A601A68AF6C013822EA07024FEA5101A3
:106E00001A60E8D1CFE700BF70B50446406A0D466E
:106E1000002828D0A16DFFF7B3F820462946FFF7D8
:106E2000A9FE606A20B1E16DBDE87040FFF7A8B827
:106E3000216C226D0868236A02430A6093B1DA7AF2
:106E400082B1D00703D5234A99691160DA7A910794
:106E500003D5214AD9691160DA7A520702D51F4A4F
:106E60001B6A136070BD236A002B2BD0D97A626D28
:106E7000E1B172B6D97ACE0706D51948D968066845
:106E8000314099610160D97A880706D5154819699A
:106E900006683140D9610160D97A4E0705D512489C
:106EA0005969066831401962016062B61B68D96889
:106EB000914207D00D4818600D49DA6042F08040D9
:106EC00018611960226C216D136823EA01031360B5
:106ED000A3E700BF00E100E004E100E008E100E01A
:106EE00080E100E084E100E088E100E001403F0053
:106EF00000003F802DE9F041044686B0806A9DF88D
:106F000030801E460F461546B4F90830002800F0C0
:106F10004281DA1D48BF03F10E02B4F90630D210E7
:106F200003FB02F2002105F05BFBB4F90820202AE4
:106F300000F39280B4F90610A34B0120203A733974
:106F400002EBD27201EBD1714FF0200E0290732050
:106F50008DE8014042F34F0241F34F01204600F01B
:106F600051FE606A84F82D70002800F04D81002DDC
:106F700040F08A80B4F90830202B14BF3D253C2511
:106F800084F82C50B8F1000F40F0858006B394F9D6
:106F90003300002818DBC0B2012102F051F80121B2
:106FA00094F8330002F038F8012002F071F8002163
:106FB00094F8330002F030F80A2002F069F8012159
:106FC00094F8330002F028F8606A002800F082800C
:106FD000A16DFEF7D5FF04227C492046FFF792FE03
:106FE000217A0139C9B22046FFF7C4FD784904224D
:106FF0002046FFF787FE94F92D30012B14BF142192
:1070000010212046FFF7B6FD042272492046FFF703
:1070100079FEB4F90630802B00F09280602B00F0EE
:10702000A680D9212046FFF7A5FD94F92D30012B2C
:1070300014BFF12122212046FFF79CFD20460622A5
:107040006549FFF75FFE606A50B3E16DFEF798FF98
:10705000012006B0BDE8F081B4F906105F4B0120B5
:10706000403A52394FF0400E029002EBD272522059
:1070700001EBD1718DE8014042F34F0241F34F0122
:10708000204600F0BFFD6CE76DB284F82C50B8F1DB
:10709000000F3FF47BAFFEF729FF002E94D076E778
:1070A000216C226D0868236A02430A6073B1DA7AA0
:1070B00062B1D00703D54A4A99691160DA7A91071B
:1070C0007CD4520702D5474A1B6A1360012006B0E0
:1070D000BDE8F081236A002B2BD0D97A626DE1B133
:1070E00072B6D97ACF0706D53F48D96805682940D6
:1070F00099610160D97A8E0706D53C4819690568FF
:107100002940D9610160D97A4D0705D538485969B8
:10711000056829401962016062B61B68D96891420E
:1071200007D0344818603449DA6042F08040186172
:107130001960226C216D136823EA010313604AE78A
:10714000B4F90830202B00F08680402B7FF469AF23
:107150002A4920460322FFF7D5FD94F92D30012B53
:1071600014BFCF219F212046FFF704FD59E7B4F952
:107170000830102B7FF455AF214920460322FFF73A
:10718000C1FD94F92D30012B14BFAF2110212046F1
:10719000FFF7F0FC45E7DA1D48BF03F10E02B4F932
:1071A0000630D21003FB02F21046059204F050FFA5
:1071B000A06200283FF44DAF059AB3E6114AD969A1
:1071C0001160DA7A7DE700BFF8D80000D8DA000055
:1071D000DCDA0000E0DA0000E4DA0000ECDA0000BB
:1071E00000E100E008E100E080E100E084E100E08F
:1071F00088E100E001403F0000003F80F4D800003B
:10720000ACDD000004E100E0012194F83100244FDE
:1072100001F016FF94F83200012101F011FF94F9FA
:10722000312094F9323057F83220E26357F8333086
:10723000206A23640125E56425651A682A431A60DB
:1072400078B1B8F1000F3FF428AFFFF7BFFA002E76
:107250003FF4BAAE9BE6042212492046FFF752FDE6
:10726000DFE6294694F82F0001F0EAFE294694F85B
:10727000300001F0E5FE94F92F2094F9303057F8F2
:107280003220626357F833306564A5641A68A363DB
:1072900022F001021A60002E3FF496AE77E600BF9E
:1072A00048E30000F0D80000B0F90820D31D48BF23
:1072B00002F10E03B0F90620806ADB1002FB03F234
:1072C000002105F08DB900BFF0B50029BDF81450BC
:1072D0002EDBB0F90660B1422ADA002A59DBB0F998
:1072E000087014461C44BC42C4BFBB1A1BB2002B1E
:1072F0001EDDD2B2D408D0F828E016FB041112F03B
:107300000702DBB20EEB010421D0C2F10807FAB28A
:10731000374F9342BF5C0CD2C3EB020CFF2646FAF8
:107320000CF6012D07EA06073FD005D3022D36D013
:10733000F0BD012D39D030D21EF8016026EA0707D2
:107340000EF801709342F3D3B0F906100C449A1A68
:10735000D2B2072A10D9022D36D0002D14BFFF2635
:10736000002613462670083BB0F90610DBB2072B47
:107370000C44F7D802F00702002AD9D01D4B012D8A
:107380009B5C1DD017D3022DD2D12278534023709D
:10739000F0BD13441BB20022A1E7022D25D11EF837
:1073A000016077400EF80170CCE71EF801603743AA
:1073B0000EF80170C6E7227822EA03032370F0BDBD
:1073C000227813432370F0BD11462378DB432370EA
:1073D0000839B0F90630C9B207291C44F5D812F0B3
:1073E0000702A5D0034B9B5CCFE73444AFE700BF57
:1073F00090D8000080D8000070B4C47DBDF80C5057
:10740000022C18D0032C1FD0012C0BD0002A03DB38
:10741000B0F90840944201DC70BC7047039570BC21
:10742000FFF7B0BAC4880395013CA41A0A4621B2FA
:1074300070BCFFF749BF0689C488013E641AB21ABE
:10744000E41A12B221B2E1E704890395E41A641A3E
:10745000114622B270BCFFF737BF00BF70B4C57DC4
:10746000BDF80C60022D1AD0032D12D0012D03D0CF
:10747000039670BCFFF728BFC488E41AA41A0A4612
:1074800021B2002A03DBB0F90840944213DC70BC3F
:1074900070470489013C641A114622B2F1E7C4889E
:1074A00005890396013CAD1AED1A621A11B22AB28F
:1074B00070BCFFF709BF039670BCFFF763BA00BF4B
:1074C0002DE9F8430446406A002863D0A16DFEF719
:1074D00057FD052274492046FFF714FCA1790139B4
:1074E000C9B22046FFF746FBB4F90820E588A66A32
:1074F000D31D48BF02F10E03DB10626A15FB03F5D2
:107500001FFA85F8002A7BD094F82C300125AB4077
:1075100082F83B3082F85E5082F85D50606A036802
:1075200040211B6808F1FF379847BFB2B8F1000F40
:1075300023D03744A846013E606A16F8011F03684D
:107540001B6898470135B742EDB216D0202DF3D114
:107550000121606AFEF776FE94F82C20636A5200DF
:1075600083F83B2083F85E8083F85D80606A03685F
:1075700040211B6898470125DEE70121606AFEF77C
:1075800061FE606A002800F08D80E16DBDE8F8437F
:10759000FEF7F6BC236A002B2BD0D97A626DE1B1DD
:1075A00072B6D97ACE0706D54048D9680568294011
:1075B00099610160D97A8D0706D53D48196905683A
:1075C0002940D9610160D97A480705D539485969F8
:1075D000056829401962016062B61B68D96891424A
:1075E00007D0354818603549DA6042F080401861AC
:1075F0001960226C216D136823EA0103136068E7A8
:10760000E26BE36C1168276A0B4306EB0809136011
:107610004FF0004E4E450DD016F801CB2FB33A680F
:10762000C2F82CE0C2F834C0D36A002BFCDA4E4515
:10763000936BF1D1226C236D11680B43136097B1EA
:10764000FB7A83B1D90703D51D4BBA691A60FB7A5F
:107650009A0703D51B4BFA691A60FB7A5B0702D5C0
:10766000194B3A6A1A60BDE8F883A36BD4F83480EA
:1076700008208021D8F80020656C1CEA010F14BF97
:107680002A43AA43C8F800201A68A56C2A431A6046
:107690001A68A56C013822EA05024FEA51011A6006
:1076A000E8D1B7E7276AC5E788D8000080E100E0A5
:1076B00084E100E088E100E001403F0000003F80FD
:1076C00000E100E004E100E008E100E02DE9F04F16
:1076D00085B09946BDF93870BDF83CA0BB1AC1EB26
:1076E000090B002BB8BF5B42BBF1000FB8BFCBF159
:1076F000000B5B450D4616460093804648DC4D4521
:107700003A4633464CDC194613460A46C5EB090196
:107710009B1A89B2002B0CB2B8BF5B4204EBD47445
:10772000BE42ACBF4FF0FF3201224D4503910292A1
:107730004FEA640429DC9BB201930DE0D8F8007095
:10774000BF69B847019BE41AA3B21CB20135002CF3
:107750002DB211DBA94518DB009B5B452A46534639
:1077600031464046EADCD8F800205346976929465E
:1077700032464046B847E5E7029A1644039AA945BF
:1077800002EB030436B224B2E6DA05B0BDE8F08FAE
:107790004A462B46B94635464D4517461E46B2DD8C
:1077A000304629463E464D4607468946AEE700BF6D
:1077B00010B404682469A44610BC604730B404685F
:1077C000BDF808500295A46BA44630BC604700BFCA
:1077D00030B40468BDF808500295E46BA44630BC90
:1077E000604700BF70B40468BDF90C60BDF810506C
:1077F00003960495246CA44670BC6047704700BF94
:1078000010B582B0B0F90C200191016800920022FD
:107810000C6CB0F90A301146A04702B010BD00BF91
:10782000704700BF01F003010129C17506D003298B
:1078300004D0C28803894281838170470289C3884A
:1078400042818381704700BF2DE9F0410568134EE6
:107850006F6986B0B7420446BDF8308010D1013B55
:1078600013441BB20093CDF804800B46AD6A20464A
:10787000A8472368DB6AB3420AD106B0BDE8F081AD
:10788000059304920391B84703A925680EC9E6E75A
:10789000204606B0BDE8F041184700BFFD77000064
:1078A0002DE9F0410568124E6F6986B0B742044673
:1078B000BDF830800FD1013BCDF804800B4400921D
:1078C0001BB2AD6A2046A8472368DB6AB3420AD1DF
:1078D00006B0BDE8F081059304920391B84703A96F
:1078E00025680EC9E7E7204606B0BDE8F041184715
:1078F000FD7700002DE9F04F0568DFF858B06F699B
:1079000085B05F450646BDF93890BDF83CA00C46F1
:10791000904615D11F19BC420CDACDF800A02146C3
:1079200001342D6A4B464246304624B2A847BC4239
:107930003568F2DBEB6A5B4507D105B0BDE8F08F37
:107940000393B8473568039BE4E7304605B0BDE8CC
:10795000F04F1847FD7700002DE9F04387B09942BA
:107960000546BDF93840BDF83C6025D0A24212D092
:107970000768DFF88080D7F81490C14532D18DE8D0
:1079800050002846BC6AA0472B68DB6A434524D1D7
:1079900007B0BDE8F083994202DD08461946034668
:1079A00028680E96C46B01335B1A1BB22846A446A6
:1079B00007B0BDE8F0436047A24202DD134622460D
:1079C0001C4628680E96631C846B9B1A1BB22846C3
:1079D000A44607B0BDE8F0436047284607B0BDE8BD
:1079E000F0431847059304920391C84703A92F68F1
:1079F0000EC9C4E7FD7700002DE9F04FD0F800E094
:107A0000DFF89090DEF814B083B0CB450446BDF9A2
:107A10003080BDF834A00D4617461E4631D1CDF852
:107A200000A0DEF824B0294633463A462046D8471F
:107A30002368CDF800A008F1FF323A44D3F824B00F
:107A4000294612B233462046D8472368CDF800A015
:107A50002946D3F820B03A4643462046D847206806
:107A6000CDF800A0711E29444346056A09B23A4682
:107A70002046A8472368DB6A4B4506D103B0BDE822
:107A8000F08FD847D4F800E0C9E7204603B0BDE83E
:107A9000F04F1847FD770000F0B4002401264FF6A0
:107AA000FF75094F07600471C475C4810482447670
:107AB000C4618675067685824582C18002814181D6
:107AC0008281F0BC704700BFB8DD00002DE9F04FA7
:107AD00085B00668BDF84450BDF93880CDF8008007
:107AE00004460195D6F848B00392BDF93C60BDF953
:107AF000407089469A46D8472368019500974246C8
:107B00005146D3F8488020463346C0472068039B3F
:107B10000E930F95856C4B463A4631462046AC464F
:107B200005B0BDE8F04F60472DE9F04F87B017462C
:107B3000BDF9404000912546E91D059344BF2B4601
:107B400003F10E010268BDF8486053690294C91040
:107B500003912B49BDF9444001968B42824645D1A1
:107B6000002C3CDD029B3C445E1EB6B24FF0000987
:107B700023B2049301364D46029B002B28DD059B62
:107B8000002403EB090806E0EDB22B0604F1010422
:107B900011D4A6421CD0A1B211F0070F23B24FEAB4
:107BA0004505F1D1002BB8BF0733DB10013418F8BD
:107BB00003502B06EDD5009BD2F818B019443A4675
:107BC00009B2019B5046D847A642DAF80020E2D11C
:107BD000039B01379944049B3FB2BB42CCD1D36A8B
:107BE000074A934206D107B0BDE8F08F9847DAF80C
:107BF0000020B5E7504607B0BDE8F04F184700BF7A
:107C0000FD77000070B4BDF90C60BDF91050BDF8EF
:107C1000144003960495059470BCFFF785BF00BF20
:107C20002DE9F04F93B090460591C1691090BDF8D1
:107C300070000790BDF874909DF878A00493002917
:107C400000F0CD800A7A0AC9894604998A1AD2B20C
:107C500003EBC203BAF1010FDA780B9293F9052016
:107C60001E8893F802B00F9293F9064079D913B2A7
:107C7000099323B20C93109B1A68A94B11931946D0
:107C800053698B4240F0A6800B9B002B55D01FFA06
:107C900088F300210D93C8462344DDF840900691F7
:107CA0000E930F460C46BBF1000F3FD0BDF81810E5
:107CB0000C9B03971FFA8AF0CB1813FB00F3049078
:107CC0000E9801440D98034409B21BB20A9108931F
:107CD000002505E00135EBB264009B45E4B222D9F2
:107CE000039B2B44590703D1731C18F806409EB21E
:107CF0002306EFD5099BBDF81000E91811FB00F130
:107D00000598BAF1010F0FFA8AF301441CD00798C5
:107D100001900093D26909B217464846089AB847BD
:107D2000D9F80020D6E7039F5F44FFB2069B0B996A
:107D300001330693DBB29942B5D8D36A119A9342C4
:107D400043D113B0BDE8F08F0F9B191893690A9ABD
:107D500029441F4609B2079B4846B847D9F8002076
:107D6000B8E700230C93099385E70A9A0D9B01322B
:107D7000013B52B213F0FF030A920D936FD1DDF86D
:107D80001890079BDDF83C80DDF820A04B4517D00C
:107D9000BAF1010F00F0C8800B9A109DCDF8049045
:107DA0000BEB8B014FEACB030A4400931146DEF83C
:107DB0001C405346424609B22846A047D5F800E089
:107DC000DEF82C30119A9342BBD0109813B0BDE866
:107DD000F04F1847109D284698472A6854E7109A94
:107DE0000598B2F90A308342ABDDB2F90C30434555
:107DF000A7DD062313FB0A03002BA2DD08EBCA0351
:107E0000002B9EDD537E2BB9049BAF2B02D901338F
:107E1000DBB20493109BD3F800E0414B11931A4658
:107E2000DEF81430934240F08E801FFA88F30E93F0
:107E300008339BB2BDF81420059305230D9300234E
:107E40000A93CDF83C800FFA8AF3DDF84080CDF834
:107E500018900B921FFA8AFBCDF820A099460A9A37
:107E6000BDF810000B9C0E9D0523194611FB002345
:107E70002C481146C75C039702FB0B4214FA81F3AE
:107E800012B21BB209920C932C462E461CE0089BA2
:107E90000999012B2AB24B4640462DD0079F0197E6
:107EA000CDF80090DEF81CA0D047D8F800E0039B86
:107EB0005B0801340393059BA4B25D445E44A34276
:107EC000ADB2B6B23FF451AF039BD807DFD4079BE6
:107ED000069A9342EBD0089B012B16D0069B019388
:107EE000CDF80090DEF81CA009994B4632B240460E
:107EF000D047D8F800E0DAE7DEF818A0079B0C9925
:107F000022B2D047D8F800E0D1E7DEF818A00C99EB
:107F10001346404622B2D047D8F800E0C7E700BF7A
:107F2000FD77000008DE00000B99109DCDF8009051
:107F30000531DEF8204009B2424608232846A04712
:107F4000D5F800E03CE7109C20469847D4F800E0C4
:107F50006BE700BFF0B5C36985B004462BB30A29AF
:107F600068D00D294AD01A7A914247D3587A88426C
:107F700044D35D688A1A05EBC205AA78002A50D05E
:107F8000E87800284DD0207E00283AD095F905E009
:107F9000B4F90E00A67DB4F90A70724406FB020221
:107FA000BA4262DCB4F9102030E00A2956D00D291B
:107FB00024D0027E002A4BD0B0F90E00A57DB4F982
:107FC0000A60062212FB0502B2423EDD228AE381EC
:107FD00002EBC50212B218462282A78A668A02956F
:107FE0000B468DE8C00001462046FFF719FEA37D31
:107FF000E28903EB430302EB4303E381012005B075
:10800000F0BDA67DB4F90E00B4F91020B4F814E068
:10801000678A02960B468DE8804001462046FFF7AE
:10802000FFFD2979E389A27D012001FB0233E38171
:1080300005B0F0BD0022C2819A7A817D038A01FBDE
:1080400002330382012005B0F0BDB4F91020C4E76B
:10805000857DB4F91020B0F90E00BEE7028A817D5B
:10806000C38102EBC1030382C8E70020E0819B7A51
:10807000228A03FB062212B22282C7E7C181028252
:10808000704700BF002908BF01218175704700BFFC
:1080900081824182704700BFC07D7047B0F90A00FD
:1080A000704700BFB0F90C00704700BF10B4EFF389
:1080B000108272B6437F33B9017F012907D00329AB
:1080C0000FD00123437702B962B610BC7047124C3F
:1080D0002168A1B1114943610B688361086058614F
:1080E000EFE70F4C216881B10E4943610B68836152
:1080F000086058610C4B4FF080511960E1E7074B65
:108100004161816120601860DBE7064B416181615C
:1081100020601860EEE700BF589BFF1F549BFF1FB5
:10812000489BFF1F4C9BFF1F04ED00E070B5EFF371
:10813000108272B60C4C206880B10C4E0025436949
:10814000236073B19D6102B962B645778368984731
:10815000EFF3108272B620680028F0D102B962B63F
:1081600070BD3360EFE700BF489BFF1F4C9BFF1FB4
:10817000FFF7DCBF184A30B41468002C27D003681E
:1081800021688B420ED2CB1A00218460C16023602B
:10819000E06010600223037530BC704711688B42A9
:1081A000144608D3A2685B1A0360002AF6D18260E5
:1081B000C460A060EEE7D268C2608460E060C56819
:1081C000CB1A0222A8602360027530BC704784601D
:1081D000C4601060DEE700BF509BFF1FF8B5224E61
:1081E00034682CB32368002B3AD1204F1D4604E09D
:1081F0003468ECB12368002B32D1A36803B1DD6091
:1082000020693360036825751B68BB4221D1037F59
:108210004560022BC46020D0FFF748FF6368002B45
:10822000E6D023602046FFF7A5FF3468002CE1D19B
:10823000EFF3108372B60E4A00211068116003B983
:1082400062B628B18468FFF795FF20460028F9D16F
:10825000F8BD224600219847E0E783689847DDE7AC
:10826000013B2360E4E700BF509BFF1FB5670000A0
:10827000609BFF1F024A136801331360FFF7AEBF14
:108280006C9BFF1FF8B50E4671B17AB107461446D4
:1082900000253B6816F8011B1B6838469847013CCF
:1082A0000544F6D12846F8BD0846F8BD1046F8BD8D
:1082B00000B5064A036812885B6883B001A9ADF86F
:1082C00004200222984703B05DF804FB08E3000095
:1082D000F0B507468BB0002A33D0012A08BF0A2226
:1082E00051B3212400E0F4B2B1FBF2F502FB151109
:1082F000C8B2092900F1300198BFC8B20AA988BFE5
:108300003730214488BFC0B201F8240C661E2946CC
:10831000002DE8D133B1013CE4B20AAB23442D2255
:1083200003F8242C3B6801AA11195B683846C4F194
:10833000220298470BB0F0BD30228DF82520212471
:10834000E8E70368C9B21B6898470BB0F0BD00BFEF
:108350000029BABF49422D2300230A22FFF7B8BFE4
:10836000374A384913681B06FCD40B6813F08003A6
:10837000F8D172B634490A78002A5FD0334A3448BB
:10838000F0B4344C176806682568D4680C303E4455
:10839000143200681268304F35442C4420440244A3
:1083A000C2F34E022D4E2E482E4D2F4C42F4004269
:1083B0003A60376806682D682C4A24680C303E44C1
:1083C000006812682A4F35442C4420440244C2F30A
:1083D0004E02284E2848294D294C42F400423A606A
:1083E000376806682D68274A24680C303E440068C8
:1083F0001268254F35442C4420440244C2F34E02F7
:10840000224E2348234D244C42F400423A60376800
:1084100006682D68214A24680C303E4400681268C2
:1084200035442C4420440244C2F34E021C4842F41A
:10843000004202600B7062B6F0BC704762B67047D3
:1084400024B0034024B00B40659BFF1F38B00340AD
:108450003CB0034040B003402CB0034058B0034050
:108460005CB0034060B0034064B003406CB00340B4
:1084700030B0034038B00B403CB00B4040B00B4034
:1084800044B00B404CB00B402CB00B4058B00B40EC
:108490005CB00B4060B00B4064B00B406CB00B4064
:1084A00030B00B4030B42948294A2A4B2A4D602469
:1084B000E121047011701B78284C082B30D00A2B56
:1084C0002748284937D00C2B0CBF35223D221223D8
:1084D0002A60236002600B60234B24491B78244AE6
:1084E000BBB101230B601360224B23491B78234A45
:1084F000012B26D9042B0FD9082B1ED9102B94BF82
:10850000862387230B6013601D4B01221A7030BC39
:1085100070470B601360E7E784230B601360F3E799
:1085200000F58E200F490830012213232A602360B2
:1085300002600B60D0E73922F7E785230B601360F8
:10854000E2E780230B601360DEE700BF00400740D6
:1085500001400740108FFF1F08B003400CB00340DC
:1085600008B00B400CB00B40689BFF1F20B00340CD
:1085700020B00B40118FFF1F24B0034024B00B40EC
:10858000659BFF1F0C2830B417D91023984228BFD1
:1085900018461C46104A114D1178181A8C42287042
:1085A00018D00F4913700B7823B10E490E4A0023DF
:1085B0000B60136030BCFFF775BF0A2802D90C238B
:1085C0001C46E7E7082802D90A231C46E2E70823ED
:1085D0001C46DFE730BC7047108FFF1F649BFF1FF6
:1085E000659BFF1F24B0034024B00B4028282FD8E0
:1085F000334B2DE9F0411E5CFF2E2BD0314B1B7805
:10860000002B2AD132062CD472B62F4D2F4C2F4678
:10861000012326602B7062B672B623681B060CD449
:108620003B781BB9F4E72B78002BF1D062B602F04F
:1086300035F972B623681806F5D5254B1B6800225C
:108640002A7062B6234A107843FA00F0BDE8F08140
:10865000002070470020BDE8F081FFF781FE320660
:10866000D2D572B61C4DDFF87C801C4C06F040075A
:10867000FFB206F03F06D8F80030DFB123F0100358
:10868000C8F8003001232660134A2B7062B672B618
:10869000236819060CD413781BB9ECE72B78002B50
:1086A000E9D062B602F0FAF872B623681B06F5D577
:1086B0000B4BC3E743F01003C8F80030E2E700BFFC
:1086C0000CE30000659BFF1F679BFF1F00B003408A
:1086D00010B00340649BFF1F669BFF1F00B00B4060
:1086E00010B00B400CB00B400A4A0B49136843F41E
:1086F000805313600B7843B9084BC0221A70084BA3
:1087000080F30C0000B218807047044B80221A706E
:10871000F5E700BF2C800440689BFF1F21C00C4080
:1087200000C00C40F0B51B4B1B4E596818689A6886
:10873000DB6885B06C460FC4337899071DD5174A9E
:10874000174C1378174913F0700318BF1370164AAB
:10875000164B8027177000263320032226706D46A3
:1087600008701A7072B6043C45F001052046A8470F
:1087700062B6237813F0700309D10D4B064901E06E
:10878000013B02D00A78D207FAD505B0F0BD2370BC
:1087900005B0F0BD38E300000100024000000240D7
:1087A000040002400B000240070002400A000240A1
:1087B000410D0300B0F5006F0AD210B5094B1B78CC
:1087C000DB07044606D504F1A0500078C0B210BD06
:1087D00000207047FFF7A6FF04F1A0500078C0B258
:1087E00010BD00BF01000240B0F5006F17D238B5D0
:1087F0000F4B1B78DA070D46044611D504F1A05043
:108800000378AB420AD00B4A137813F0700318BFF9
:108810001370074A05701378DB07FCD538BD704725
:10882000FFF780FF04F1A0500378AB42EBD1F5E7EE
:10883000010002400000024008B5F7F751FEF9F7C9
:10884000BBFA02F02BF8FAE7844641EA000313F082
:1088500003036DD1403A41D351F8043B40F8043B47
:1088600051F8043B40F8043B51F8043B40F8043B0A
:1088700051F8043B40F8043B51F8043B40F8043BFA
:1088800051F8043B40F8043B51F8043B40F8043BEA
:1088900051F8043B40F8043B51F8043B40F8043BDA
:1088A00051F8043B40F8043B51F8043B40F8043BCA
:1088B00051F8043B40F8043B51F8043B40F8043BBA
:1088C00051F8043B40F8043B51F8043B40F8043BAA
:1088D00051F8043B40F8043B403ABDD2303211D34A
:1088E00051F8043B40F8043B51F8043B40F8043B8A
:1088F00051F8043B40F8043B51F8043B40F8043B7A
:10890000103AEDD20C3205D351F8043B40F8043B49
:10891000043AF9D2043208D0D2071CBF11F8013B47
:1089200000F8013B01D30B8803806046704700BF0D
:10893000082A13D38B078DD010F003038AD0C3F11C
:108940000403D21ADB071CBF11F8013B00F8013BFE
:1089500080D331F8023B20F8023B7BE7043AD9D3BD
:10896000013A11F8013B00F8013BF9D20B78037092
:108970004B7843708B7883706046704708B5104C15
:1089800008E0236859050DD423681A050FD423681D
:10899000DB0411D423685803F3D500F08DFE23685F
:1089A0005905F1D501F0DEFF23681A05EFD502F075
:1089B0006FF82368DB04EDD500F0F0FCEAE700BFB8
:1089C0003480044008B5FFF7D9FF00BF014B1022E7
:1089D0001A80704700200540704700BF094908B55C
:1089E0000B6830B16A461844A2F58052904202D218
:1089F0000860184608BD03F0FDFA0C2303604FF031
:108A0000FF3008BD148FFF1FFEE700BFEFF3138098
:108A100070B9EFF310836BB9EFF305825AB94FF4D5
:108A20008070EFF311832BB1984228BF184670472E
:108A30004FF0FF3070470F2A01D81846F1E7014B7D
:108A4000D05CEEE7F0E300E0F0B44D1E2E460024CB
:108A500000E00134B0FBF2F302FB1300092800F13F
:108A600030078ABF3730F8B2C0B206F8010F184697
:108A7000002BEED10A1953704CB1107815F8016F24
:108A800028700133E01A834202F80169F5DB0846D9
:108A9000F0BC7047704700BF10B40F4B53F8302044
:108AA00092F880422CB1012369B182F8803010BC69
:108AB000704703EBC0035B681A6841B922F00202F9
:108AC0001A6010BC704782F8003110BC704742F049
:108AD00003021A6010BC704748E300001C4A02EB16
:108AE000C00301295B6811D004291BD052F8300063
:108AF000002280F8802229B1022920D0032922D027
:108B00001A6070474FF480721A60704752F8300054
:108B10004FF4A27280F880121A601A6822F02002C4
:108B20001A60704752F830104FF4A272012081F899
:108B300080021A601A6842F020021A60704740F200
:108B400003121A6070474FF481721A60704700BFB9
:108B500048E30000212848D8F8B5042A44D8DFE8C3
:108B600002F0484B4E0345004FF410262B4B03EB0D
:108B7000C0030D465C68216811F4E06148D0284BC1
:108B8000284A2949C3F89C2104F140422748C3F8E8
:108B9000A411A2F59221264FC3F8A0017C292548F3
:108BA000C3F8A871C3F8AC012CD9A2F594237C2B8F
:108BB0002AD9A2F596237C2B28D9A2F598237C2BC1
:108BC00029D9A2F59A227C2A27D81B4872B6236895
:108BD00023F4702343F08072C4F3840116432360AE
:108BE00040F82150266062B6F8BD70474FF4302639
:108BF000BCE74FF40026B9E74FF44026B6E74FF440
:108C00002026B3E70D48E1E70D48DFE70D48DDE733
:108C1000FFF764FFB3E70C48D8E7F8BD48E300006E
:108C20000082FF1FF188FF1F9988FF1FC588FF1F63
:108C30006D88FF1F4188FF1FF08FFF1F188FFF1FD8
:108C4000508FFF1FA08FFF1FD08FFF1F1A4B03EB0A
:108C5000C00010B4426802F14043A3F592217C2980
:108C600023D9A3F594217C290DD9A3F596217C293C
:108C70001FD9A3F598217C2919D9A3F59A237C2B18
:108C800011D80E4C00E00E4C72B613680D4823F05C
:108C90008773C2F3840123F4803343F0807313603D
:108CA00044F8210062B610BC7047074CECE7074C53
:108CB000EAE7074CE8E700BF48E30000F08FFF1F3A
:108CC000508FFF1F958A0000188FFF1FD08FFF1F46
:108CD000A08FFF1F30B4054B054D064C002210211C
:108CE0001A602A602060196030BC704714D00340BD
:108CF00004D0034000D00340282838B52ED00029E6
:108D000004464FDD5F4B1B78012505FA03F28A42CA
:108D100002D8212837D938BD0338C2B2012A3AD93E
:108D2000202C4AD0192C48D0574A126802FB011255
:108D300022FA03F31D2800F29B80DFE800F0928BFB
:108D4000847D9999766F9999999999999999996842
:108D5000615A53994C99999999999945494B1B781E
:108D60000B2B08D90C2B1CBF0C3B19410846BDE846
:108D70003840FFF7B9BCC3F10C0399400846BDE881
:108D80003840FFF7B1BC2946FFF786FE2946BDE80B
:108D90003840FFF7A3BE3D4A126802FB011222FAD7
:108DA00003F3C7E72128B6D80021FFF775FE204658
:108DB0000121BDE83840FFF791BE354A126802FB39
:108DC000011222FA03F3B5E73249334A0B604FF43C
:108DD0005173136038BD3149314A0B604FF4517300
:108DE000136038BD2F49304A0B6040F24443136092
:108DF00038BD2E492E4A0B6040F24443136038BD03
:108E00002C492D4A0B6040F24443136038BD2B4976
:108E10002B4A0B6040F24443136038BD29492A4A6B
:108E20000B6040F24443136038BD2849284A0B6068
:108E300040F24443136038BD2649274A0B6040F294
:108E40004443136038BD2549254A0B6040F2444332
:108E5000136038BD2349244A0B604FF451731360EB
:108E600038BD2249224A0B604FF45173136038BD5C
:108E7000212C3FF650AF7F29D4BF0021012120468D
:108E800093E700BFF88FFF1F08800340089003405E
:108E900008800B4010800B4048A0044018800B4015
:108EA0004CA004401880034008B0044010800340E8
:108EB00004B004404080034018C0044038800340A0
:108EC00014C004402880034010B0044020800340B8
:108ED0000CB004403080034010C004404880034080
:108EE0001CC004401890034034900440109003408C
:108EF0003090044038B1102828BF1020044AC3B273
:108F0000107813707047024A01231078137070476D
:108F1000F88FFF1F2DE9F8430E4680463249334D46
:108F2000304602F0EDFF47F6122300281ABF1D4617
:108F30004FF002094FF00109002425FA04F002F075
:108F4000E9FD4FF05E51074602F03CFE0146304617
:108F500002F0EAFF30B90134072CEED1E80902F043
:108F6000D9FD07463146384602F0E0FE4FF07C510D
:108F700002F01EFD03F012F84FF6FF729042A8F1C6
:108F8000030328BF1046012B29D9B8F1170F17D8B2
:108F9000174B23FA08F303F0010383F0010223B90E
:108FA000B8F1190F0FD0BDE8F883124B124D1349D9
:108FB0001A6044EAC9042A6008601C60BDE8F883AE
:108FC000B8F1200FECD10E4B0E4D0F49002244EAB0
:108FD000C9041A602A6008601C60BDE8F8830B4B66
:108FE0000B4D0C49F2E700BF001BB740006CDC02E0
:108FF0006006F000008003400480034008800340C6
:1090000000800B4004800B4008800B400090034020
:109010000490034008900340212801D8FFF73CBD8D
:10902000704700BF212806D8044B53F8303093F81E
:109030000002C0B270470020704700BF48E3000044
:10904000212801D8FFF74ABD704700BF72B60C490E
:109050000C4B0D4A1B680868126862B6520102D5B3
:10906000322B88BF01300949C3F5BB334FF47A7204
:10907000FF33A1FB031302FB00F000EB93107047DA
:109080006C9BFF1F18E000E004ED00E0ABAAAAAA69
:109090002DE9F843054672B6204F214B214A1B6843
:1090A0003C68126862B6520102D5322B88BF013487
:1090B00095B3C3F5BB331C4EDFF86490DFF86480D2
:1090C000FF334FF47A72A6FB031302FB04F404EBA4
:1090D000931472B6D9F800103A68D8F800E062B676
:1090E000C1F5BB33FF33A6FB03031EF0806FC4EB57
:1090F00093134FF47A7002D0322988BF013200FBFB
:109100000233B3F57A7F04D3013D05D004F57A74B8
:10911000DFE701F0C3FBDCE7BDE8F8836C9BFF1FD2
:1091200018E000E004ED00E0ABAAAAAAF8B52D4BC8
:109130002D49DFF8D0E0DFF8D0C02C4E2C4D2D4C5F
:109140002D4A2E4F4FF4000018604FF080701860C9
:109150004FF0007018604FF0806018604FF00060B2
:1091600018600020086028234BF6FF71CCF800102F
:10917000CEF80030336013602B6023603B60B36235
:109180009362092245F8242CC4F8D80F05F57F65B1
:10919000C7F8D41F07F5FF2707F5FA67C6F8F83FA9
:1091A0002B6006F5FF26C4F8D42F05F5FD2504F540
:1091B000FF24386006F2F4761148316005F5FF654A
:1091C00004F5FD642B6023600260FFF76BF9192042
:1091D000FFF75EFF00F0B6FF40F21310BDE8F84065
:1091E000FFF756BF08E100E004800340148003400D
:1091F000248003402C8003401C80034034800340C3
:1092000000800B400C800340088003402DE9F84F9C
:10921000214B1B6807460BB101221A70DFF88890BA
:109220001E4D99F80040DFF884801D4E0134272C34
:109230008ABF4FF0000A5FFA84FA5446AB462B7897
:10924000A34216D1FFF7E2FB40281FDC33791B064F
:10925000F5D59BF800300133272B86BF002213463B
:10926000DAB218F80330DBB2F3712A702B78A3421C
:10927000E8D00C490A4BFFB208F804700120AC2278
:10928000087089F800A0DA70BDE8F88FFF28D6DDF5
:1092900001F004FBD3E700BFE49BFF1FE19BFF1F2E
:1092A00000C00640E09BFF1FE89BFF1F789BFF1F4D
:1092B0001C4BDFF894C01A681B49F0B542F4805289
:1092C0001A4D1A60DFF884E0194F1A4E1A4C002329
:1092D0008CF800304FF451722B701F2840F2133578
:1092E0008EF800303B70337025600A6012D8194642
:1092F0000124124A124D11701248547000212C277B
:10930000402693724FF4003491701174D7702E7010
:109310000460F0BDC0F34431C0F3471400F01F03F4
:10932000E7E700BF348004400CC00440759BFF1F7A
:10933000E19BFF1FE09BFF1F08C0044000C00640E8
:1093400031E400E004E100E0749BFF1FE89BFF1F95
:10935000034B1B68DB0401D5FFF758BF704700BF04
:109360003480044010B5044C237823B101F096FA00
:109370002378002BFAD110BDE09BFF1F054A064B56
:1093800010781B78C0B2DBB2984238BF4030C01AA8
:10939000704700BF749BFF1F759BFF1F30B42B4BA2
:1093A0001A7994061FD52A48DA79037829490133B6
:1093B0003F2B0978C8BF00238B42D2B203D0264C82
:1093C000D9B2E2540170254A116861B1244A127879
:1093D000D2B2934236BFC2F140029B1A9B18272B90
:1093E000C4BF01230B70194AD378DBB2180611D41D
:1093F0005A060DD5154B1B795B0609D5194B1A4931
:109400001B6800220A7003B11A70104B2C22DA700C
:1094100030BC704711790906EAD5144910480C7818
:109420000178C9B28C420DD04A1C272A84BF002182
:109430000A460F4D054C98BFD1B2AA5CD2B2E27178
:109440000170D5E76C21D170D2E700BF00C00640A3
:10945000749BFF1F759BFF1FA09BFF1F709BFF1F2F
:10946000E19BFF1FE49BFF1FE09BFF1FE89BFF1F8B
:10947000789BFF1F21282FD8184B195CFF292BD070
:10948000174B184ADFF870C003EBC000F0B5436813
:10949000DFF868E0144F154D154E00241C60DEF80F
:1094A0000030012043F020038840CEF800301460E3
:1094B0004FF4A07338602E60C2F800C0013BFDD1AC
:1094C00013689B05FCD42023013BFDD1094B09B255
:1094D00033F8110080B2F0BD0020704758E400005E
:1094E00048E3000000500440085004400450044089
:1094F000000002030051044080014A00388004400B
:10950000431E032B14D872B60A4951F8230068B1E0
:1095100070B4094C058834F81320466841F823607C
:10952000521B24F8132062B670BC704762B67047B5
:1095300000207047449CFF1F889EFF1F01380328AE
:109540000BD872B6074B53F8203043B100205B684C
:109550000130002BFBD162B67047002070471846DF
:10956000F9E700BF989CFF1F30B472B62B4A1378FE
:109570001D0706D52A4B196A002936D0996A002999
:1095800041D053781C0706D5254B196C00293ED0D5
:10959000996C002939D09378190705D5204B196E9D
:1095A000002936D0996E89B1D3781B0707D51C4B9B
:1095B000D3F880207AB3D3F8882011213AB162B66B
:1095C000184B00221A7030BC00F04ABE0D21154C19
:1095D000154D227843F8315003EBC1030830013AAE
:1095E0005860227062B630BC704704220D4C0F4D9B
:1095F000217843F8325003EBC20308304A1E58600A
:10960000227062B6EFE70521E1E70921DFE70822D2
:10961000ECE70C22EAE71022E8E700BF7CE4000058
:109620000080FF1FC19CFF1FC80040008800400051
:10963000431E032B1DD81B4A400140F0100030B4DC
:10964000104472B6184CE25C032A1BD8DFE802F023
:109650000212151703220D88E25410F0080F14BFF0
:10966000C823882343EA054308310360416062B69A
:1096700030BC704708300222EDE70522EBE70830E6
:109680000422E8E7094A52F8230038B1084A52F8A0
:109690002300416042F8231062B6E9E742F8231044
:1096A000034AF7E70080FF1FD09CFF1F989CFF1F15
:1096B000A89CFF1F00BE70472DE9F04FDFF818B3DC
:1096C000DFF818A387B044E0AD4F4FEA930807EBEB
:1096D000C809013ED9F8042003F00803F6B2A2F14C
:1096E000080003F0FF04002B40F0018157F83830E8
:1096F0001B0C99B222F8081C002B00F0EF80A14B44
:1097000022F8064C42F8044C53F82620002A00F0B8
:10971000CF819D4D55F8263058609C4C45F8260069
:1097200034F81630194424F8161000F079FD00289A
:1097300000F0C281964A974B19F0080F00F108001B
:1097400018BF1346C9F8040047F8383008238BF8CF
:1097500000309BF80040E4B265071CD58E4B1B78A7
:10976000B3B18E490A7802F0FF0322B1013BDBB2AC
:109770000B7003B900BE8A490A7802F0FF032AB1D0
:10978000013BDBB20B70002B00F0688100F000FEA3
:1097900004238BF8003004F0080303F0FF02002BD1
:1097A00000F0C9809AF80030DBB21E098CD19A080B
:1097B000DFF8CC9159F8321009EBC200C1F38301F4
:1097C000013940680C2900F28580DFE801F07A7ADF
:1097D0008383838383834683838307000168714D7A
:1097E0004068714F714E6860296088B240F28161B3
:1097F0000024674B49F832304FF0010E88423C603C
:10980000C9F81040C9F8184086F800E05C4A00F238
:10981000E780B0F5D06F80F01B82B0F5817F00F05B
:10982000D98100F26981802800F02A82822840F0E4
:10983000D781A98801F07F01042900F2D1815C4819
:109840005C4A890008441470547001788C0740F118
:10985000608382F800E0022173E1534F3A682AB333
:10986000554B524E554819883478057840298E4614
:1098700045F0020828BF4FF0400E002C84F0010490
:109880003470CEEB01010CBF8824C82409EBC80654
:1098900089B285F0010544EA0E447260198049F8E6
:1098A000384072440570002965D03A603D4B1A88F3
:1098B000B2F5A06F0ED100219A785970404B1A7002
:1098C00008E038493F4C0D68A54200F098803049C7
:1098D00049F832103C4A0123137037E72C4A2D4BCC
:1098E00019F0080F18BF134647F838302EE700F07C
:1098F000B7FC364A364952F82630002B00F0E38098
:1099000058688C5D42F8260003F10802C9F804206B
:10991000032C05D8DFE804F02C02292602228A5500
:109920001A8819F0080F0CBF8823C82343EA0243A2
:1099300047F838300AE7E00700F19380210600F18C
:10994000D180A20706D5234A234913780220DBB22F
:1099500013700870E30602D51F4B10221A7007B06F
:10996000BDE8F08F04228A55DAE705228A55D7E749
:1099700003228A55D4E7BEF1400F18BF002294E7B6
:109980000080FF1F449CFF1FF09BFF1F889EFF1F4E
:10999000C800400088004000CC9CFF1F559CFF1F62
:1099A000409DFF1FB89CFF1FEC9BFF1F549CFF1F97
:1099B000C0200740C49CFF1F009CFF1FC09CFF1FCE
:1099C000982007402109000394200740989CFF1F1E
:1099D000D09CFF1F88200740802007409020074030
:1099E000B0F5106F00F07C8140F2A38040F62112A8
:1099F000904240F07B82A54A012313706AE74C68CD
:109A0000A3498C427FF463AF0178A9297FF45FAF4B
:109A1000417845297FF45BAF8178C2297FF457AF45
:109A2000C1786B297FF453AF9A489B4E0178347804
:109A300081F00105002C41F0020105700CBF882067
:109A4000C82084F0010449F8310009EBC1019348B2
:109A50003470002505244D60047038E700F0FEFEE8
:109A600094E68F4B89488B491A614FF0020E80F8BB
:109A700000E08C4F0A708C49196099608B4E8C4DB8
:109A80008C4C9A610D213970FF213170DFF84CE266
:109A900029702270884D894A8EF800109F27012472
:109AA00006F8047C5D600470DA6007B0BDE8F08FF2
:109AB00043F82600824D30E6824A47F83800137892
:109AC0000133137042E68B5D032B00F2BA8001A2D2
:109AD00052F823F04D9700004D9700002D9B000099
:109AE000279B00006F49724B80220D2008701A706E
:109AF000A2077FF52FAF26E740F20232904240F0F6
:109B0000ED81AA8802F07F02042A69D86D88002DB1
:109B100066D16449CDF804E0920011440A7842F01D
:109B200002020A70C1E101238B550FE600238B5519
:109B30000CE6B0F5086F53D16349644A0978117097
:109B40007146ED888D4280F0E88252480478402DBD
:109B5000AE4644F0020C28BF4FF0400E02EB0E035D
:109B600009EBCC01029301234A604FEA0E48CEEB89
:109B7000050101930025C82242EA080384F001028E
:109B800049F83C3035700270DFF814C1424BDFF801
:109B9000048149BBBEF1400F7FF42DAF42F0020CAF
:109BA00009EBCC03029ADFF8F8E05A608DBB0D0494
:109BB00045F088059DF804304EF83C500A44337057
:109BC0000470134640297FF416AF0021404A3B60E1
:109BD000118010E7AA8802F07F02042A40F28B81EC
:109BE000304A0F23137006E74029D7D942F002020A
:109BF0000CEBC200029E4660BDB19DF80450354892
:109C00001D703346403988F8004040334CF832002C
:109C1000DCE79DF8043033700D04029B047045F0BE
:109C2000C8050B444EF83C50CCE79DF804501D701D
:109C3000029B1D4888F80040403940334CF8320000
:109C4000C4E719F0080F0CBF022303238B557DE5F1
:109C500021494A68002AC3D06C88B5F804E003E0C3
:109C60000C314A68002ABBD00B88A342F8D14B883C
:109C70007345F5D1240A032C0CBF1178098960E7DC
:109C8000124A0221147054705BE700BF9420074011
:109C900001000400C09CFF1F549CFF1F559CFF1F28
:109CA0000080FF1FC0200740880040008820074038
:109CB0008020074098200740049CFF1F589CFF1FEE
:109CC000F09BFF1FC19CFF1FCC9CFF1FC49CFF1F6C
:109CD000009CFF1FC800400080E400008C2007406B
:109CE000B248116AAC7804700C0600F19881D9F87A
:109CF0002820AF49100600F1DB81D9F83020AC49AB
:109D0000120600F1D081D9F83820A949130600F1D4
:109D1000C581D9F84020A649150600F1BA81D9F8C5
:109D20004820A349140600F1AF81D9F85020A0497A
:109D3000100600F1A481D9F858209D49120600F1BF
:109D40009981D9F860209A49130600F18E81D9F8DB
:109D500068209749150600F18381D9F8702094494D
:109D6000140600F17881D9F878209149100600F1A5
:109D70006D81D9F880208E49120600F16181D9F8F1
:109D800088208B49130600F15581D9F89020884925
:109D9000150600F14981D9F898208549140600F18B
:109DA000FF808448844A854901908548854D864CCA
:109DB000049700230596029580460F4616461D46D9
:109DC0000394306828B1446800F04AFA2046002C19
:109DD000F9D100233360029B38681A46002342F809
:109DE000253028B1446800F03BFA2046002CF9D118
:109DF00000223A60019A98F800301146002241F89A
:109E0000042B039A0191023B4FF0000122F8151038
:109E1000032B07D8DFE803F05D025D024FF001037A
:109E200088F800300135042D06F1040607F1040717
:109E300008F10108C5D1654C654D2278654B049F3A
:109E4000059E0021100729701A7000F19280624966
:109E500062780A700021C9F83010C9F8381011076B
:109E6000DFF84C816ED4A2785C49DFF844810A7037
:109E700000211207C9F85010C9F858104BD4E278E5
:109E800057494B4C0A7013074FF00001C9F8701086
:109E9000C9F8781000F1AE8033780193002283F086
:109EA0000105C9F89020C9F8982000210291884640
:109EB0008E460A464B48047844F0020C09EBCC036A
:109EC0000393019B002B039B5A600CBF8822C8227E
:109ED00052E64FF0000388F80030A3E7B0F5A06F1A
:109EE0007FF47EAE012300250193DEE740F62122B8
:109EF0009042F7D074E66D88002D7FF471AE3A4938
:109F0000CDF804E0920011440A7822F002020A70AF
:109F1000CBE7022115E600F083F9002800F0EB8082
:109F20000830324AC8F86400C8F8602000F078F9B8
:109F3000002800F0DA8008302D4AC9F86C00C9F812
:109F400068209CE700F06CF9002800F0E080083001
:109F5000264AC8F84400C8F8402000F061F90028FB
:109F600000F0CF800830224AC9F84C00C9F84820D8
:109F700079E700F055F9002800F0A58008301B4A69
:109F8000C9F82400C9F8202000F04AF9002800F0A0
:109F900094800830164AC9F82C00C9F8282056E7E2
:109FA000D1F89C00083800F05BF9FAE6CC9CFF1F62
:109FB0000080FF1FA89CFF1F449CFF1F989CFF1F51
:109FC000D09CFF1FF09BFF1F889EFF1F7CE40000BA
:109FD000C19CFF1FC4200740C8200740CC20074079
:109FE000D0200740C09CFF1FC020074088004000D1
:109FF000C800400000F014F9002870D008304F4A23
:10A00000C4F88400C4F8802000F00AF9002860D069
:10A0100008304B4AC9F88C00C9F888203CE7506AE0
:10A02000083800F01DF962E6D1F89400083800F015
:10A0300017F9B0E6D1F88C00083800F011F9A4E661
:10A04000D1F88400083800F00BF998E6C86F08389A
:10A0500000F006F98DE6486F083800F001F982E655
:10A06000C86E083800F0FCF877E6486E083800F053
:10A07000F7F86CE6C86D083800F0F2F861E6486D54
:10A08000083800F0EDF856E6C86C083800F0E8F83B
:10A090004BE6486C083800F0E3F840E6C86B083837
:10A0A00000F0DEF835E6486B083800F0D9F82AE60B
:10A0B000C86A083800F0D4F81FE62A78C9F82800E2
:10A0C00001322A70C3E62A78C9F8200001322A70CA
:10A0D0005AE72A78C9F8880001322A70DCE62A7823
:10A0E000C4F8800001322A708EE72A78C9F8680027
:10A0F00001322A70C3E62A78C8F8600001322A705B
:10A1000014E72A78C9F8480001322A70ABE62A78A9
:10A11000C8F8400001322A701FE740298E4628BF48
:10A120004FF0400E02EB0E0302930123CEEB010130
:10A130004FEA0E4800250193BCE600BF88004000AE
:10A14000C8004000F8B500F029FD294B29482A4CE9
:10A150002A4F2B4DDFF8BCC0DFF8BCE0294E0022AF
:10A160001A605A609A60DA601A615A619A61DA611B
:10A170001A625A629A62DA621A635A639A63DA63FB
:10A180001A645A649A64DA641A655A659A65DA65DB
:10A190001A665A669A66DA661A675A679A67DA67BB
:10A1A000C3F880200168C3F8842041F48021016055
:10A1B000C3F307212170C3F30740134938701B0E06
:10A1C0002B70FF238CF80030104D8EF800301048B3
:10A1D0000B700123337084F8642070264FF40074F0
:10A1E000102207F82C3C2E70046081F8F820F8BD8E
:10A1F0000080FF1F348004409C200740B0200740AF
:10A20000B4200740942007401020074049E400E0B4
:10A2100008E100E08020074088200740704700BF29
:10A2200072B60D480268B2FA82F30F2B10DC4FF0C1
:10A230000041D94022EA0102026062B6074803EBFE
:10A24000C303DB00C2180021C150104651607047A3
:10A2500062B60020704700BFFC8FFF1FBC83FF1F4A
:10A260000D4B0E4AC31AA2FB03231B090F2B0CD85C
:10A270000B4A127852B972B60A484FF00041026890
:10A2800021FA03F31A43026062B67047064A127855
:10A29000002AF0D0FFF768B9BC83FF1F398EE3387E
:10A2A000C19CFF1FFC8FFF1FCC9CFF1F38B50E4BBE
:10A2B0000E4C1B68218805468BB1B1F5917F05D204
:10A2C0000B4A4B1C55549BB2238038BD00220848D2
:10A2D00098470021064A55540123238038BDB1F523
:10A2E000917FEDD338BD00BFF89CFF1F929EFF1FEA
:10A2F000989EFF1F2DE9F843214E224F316801231C
:10A3000080463B70B1B1204D4B8801EB8302013395
:10A3100000240F2BC2F808802C7004D84B80002337
:10A320003B70BDE8F88340230B800320FFF780F9E2
:10A330003460F4E7DFF8549099F80030002BF0D047
:10A34000114D45F6215408E0013C12D02B7883B919
:10A3500000F0A4FA99F800307BB10320FFF7EEF883
:10A360000528F1D8FFF75CFF014630600028EBD0EC
:10A37000CAE701232B70BDE8F883BDE8F88300BF6E
:10A38000149DFF1FE89CFF1F189DFF1FCC9CFF1F03
:10A3900038B5084B1C7824B9074D296809B14B889A
:10A3A00003B938BD9B000B800320FFF741F92C60F7
:10A3B00038BD00BFE89CFF1F149DFF1F2DE9F04131
:10A3C000AD4E33680746002B00F092801D885A88F6
:10A3D000910803EB81010432AA428C6842D25A8070
:10A3E00004F00F064FEA1428A449A6F1080208F069
:10A3F0000F00C4F30313062A00F101050B701AD9EC
:10A40000B31E012B5FFA88F04ED9052E48D0042EDA
:10A4100000F0A481731F022B7FD90F2E0ED1F728D5
:10A4200042D8F02802D0964B1B883BB1FFF73EFF85
:10A430000020BDE8F08127B1BD4202D00020BDE878
:10A44000F081082EC4F3033300F08780092E11D069
:10A450000A2E40F094800A2BF0D18A4B8A4A1B685E
:10A46000A02181E01846FFF7FBFE0420FFF748F823
:10A470003060B5E7092BE1D1270E00F07B81834BDB
:10A48000814A1B689021C4F307461170EDB2FCB2FB
:10A49000002B00F09D80224631462846984797E0E1
:10A4A000F02843D9F72841D0F1380E28C6D801A3A7
:10A4B00053F820F06BA600004FA600003DA6000058
:10A4C0003DA400003DA400002FA600003DA4000014
:10A4D0000FA700003DA40000D9A60000F3A60000CD
:10A4E00017A600003DA40000FFA50000E3A50000A2
:10A4F000674B1B78002BA1D00420FFF701F803461F
:10A50000306000289AD00588002D7FF460AFFFF7F7
:10A51000A7FE35602846BDE8F081FFF7C7FEC4F30B
:10A520000740FFF7C3FE072E02D1200EFFF7BEFE45
:10A53000534B584A198858481468584D524A01706C
:10A5400000270E0AF0201F802E7010700CB301221D
:10A550005348A0470120BDE8F081082B7FF46EAF7F
:10A56000504B494A1B688021C4F307461170EDB275
:10A57000240E6BB3284622463146984728E00B2E1E
:10A5800011D10B2B7FF45AAF474B3F4A1B68B021C8
:10A59000EAE7464B1B68002B00F0FB8040489847D9
:10A5A0000120BDE8F0810C2E40F000810C2B7FF4DF
:10A5B00045AF3F4B344A1B68C0211170EDB2C4F364
:10A5C0000746002B00F0C88028463146240E9847E5
:10A5D0003849314A314B0D7016701C700120BDE8AE
:10A5E000F081354B1B68002B00F0D6809847C4F3F0
:10A5F0000746254BEDB2240E83F80080E8E72F4B89
:10A600001B68002BF2D12E4B1B68A3B1FE2098478C
:10A61000C4F30746EDE72B4B1B68002BE6D1284B14
:10A620001B6843B1FC209847C4F30746E1E7264B7B
:10A630001B68002BDAD1C4F30746DAE7234B1B680B
:10A64000C4F30746002BD4D030469847D1E7204BBF
:10A650001A68002AEFD0260C630C06F07F0003F482
:10A660007E531843F6B29047C3E71A4B1B68C4F3F6
:10A670000746002BE8D1BCE7209DFF1F969EFF1FD9
:10A68000929EFF1FFC9CFF1F909EFF1F309DFF1F8F
:10A69000CC9CFF1FF89CFF1F949EFF1F959EFF1FE1
:10A6A000989EFF1F289DFF1F2C9DFF1F109DFF1FC1
:10A6B000EC9CFF1F979EFF1FD89CFF1FDC9CFF1F79
:10A6C000E09CFF1F1C9DFF1F0C9DFF1F249DFF1F73
:10A6D000F49CFF1F089DFF1F3F4B1B68002B85D17B
:10A6E0003E4B1B68002BA6D0FA209847C4F30746C0
:10A6F0007FE73B4B1B68002B7FF478AF374B1B6821
:10A70000002B98D0FB209847C4F3074671E7354BE0
:10A710001B68002B7FF46AAF304B1B68002B8AD07C
:10A72000F8209847C4F3074663E70E2B7FF486AE04
:10A730002D4A2E4B1268E0211970002A47D0260CB2
:10A74000610C06F07F0301F47E511943EDB2A1F5CF
:10A75000005128469047F6B2240E39E7FFF7A6FDD0
:10A76000C4F30740FFF7A2FD200EFFF79FFD002076
:10A77000BDE8F0811E4B1D4A1B6880211170EDB2AF
:10A78000C4F3074683B1314628463A4698473C46CB
:10A790001EE70120BDE8F081104B1B68002B3FF441
:10A7A0004AAFFF20984746E71C4611E70D2EBCD163
:10A7B0000D2B7FF443AE0F4B0C4A1B68D021117058
:10A7C000EDB2C4F30746002B7FF4FEAEC4E7C4F33A
:10A7D0000746EDB2240EFBE6049DFF1FE09CFF1F21
:10A7E000E49CFF1FD49CFF1FF09CFF1F909EFF1F47
:10A7F000289DFF1F009DFF1F38B5164D2868E0B14A
:10A8000001884488A14213DD03191B7A83B104F146
:10A810000803C2180C1B002302E012F8011F21B12B
:10A820000133A342F9D1204638BD1C46204638BD2D
:10A83000FFF716FD0020286038BD074B1B780BB9C9
:10A84000002038BD0220FEF75BFE28600028D7D12B
:10A85000F6E700BF3C9DFF1FCC9CFF1F0D4B1B78F4
:10A86000BBB910B50C4C216803F0FF024B883F2B9D
:10A8700007DC07330B4401F1470003F8012F834243
:10A88000FBD140230B800120FEF7D2FE0023236082
:10A8900010BD7047349DFF1F389DFF1F38B5224CF7
:10A8A000237803B138BD01232370FFF7A5FF70BBE8
:10A8B00000F048F840BB00F0DBF810BBFEF75EFD8F
:10A8C000E0B900232370EFF30583002BEAD1EFF307
:10A8D000108172B6154B1868E0B1154C2278CAB9D0
:10A8E00045691D6001232370C5B1AA6101B962B633
:10A8F00000254577836898472570D3E700F020F856
:10A90000DFE700F01BF8D9E700F016F8D3E7FFF710
:10A9100085FCCDE70029C5D162B638BD054B1D6069
:10A920000029E5D1E3E700BF419DFF1F589BFF1FB2
:10A930005C9BFF1F549BFF1F704700BF704700BF09
:10A94000704700BF054A064B10781B78C0B2DBB2D7
:10A95000984238BF4030C01A704700BF489DFF1F63
:10A96000499DFF1FF0B4384B1A7912F0300F2CD0EC
:10A9700072B6997D01F0FF0200293DD062B6334FD7
:10A98000334938780D78334E1C46C0B2EDB2431CC3
:10A99000402BE17928BF0023AB4202F1FF32C9B25C
:10A9A0001CBFF154184612F0FF02F0D12A4B1B686D
:10A9B000C2B23A704BB1A84236BFC5F14005401B48
:10A9C00040192728C4BF01221A701F49CA78D2B281
:10A9D000150616D452060DD51B4B1B795B0609D5FF
:10A9E0001E4B1F491B6800220A7003B11A70164BD8
:10A9F0003C22DA70F0BC70474022D9795A7462B6B2
:10AA0000E3E70B791C06E5D5164B174E1C78337817
:10AA1000E4B2DBB29C420ED0144D01E0A3420AD056
:10AA20000133402B28BF00230879E85CC0B2C8710D
:10AA3000087D0728F2D9DBB2034933700B79180679
:10AA400044BF7C23CB70C5E700A00640489DFF1F94
:10AA5000499DFF1F8C9DFF1F449DFF1FD09DFF1F21
:10AA6000CC9DFF1FD49DFF1FCD9DFF1F4C9DFF1F41
:10AA7000054A064B10781B78C0B2DBB2984238BF4B
:10AA80004030C01A704700BF489EFF1FDD9DFF1F6A
:10AA9000F0B4384B1A7912F0300F2CD072B6997D81
:10AAA00001F0FF0200293DD062B6334F33493878B8
:10AAB0000D78334E1C46C0B2EDB2431C402BE179F9
:10AAC00028BF0023AB4202F1FF32C9B21CBFF154D0
:10AAD000184612F0FF02F0D12A4B1B68C2B23A703E
:10AAE0004BB1A84236BFC5F14005401B401927288D
:10AAF000C4BF01221A701F49CA78D2B2150616D4F3
:10AB000052060DD51B4B1B795B0609D51E4B1F4901
:10AB10001B6800220A7003B11A70164B3C22DA70CF
:10AB2000F0BC70474022D9795A7462B6E3E70B79DA
:10AB30001C06E5D5164B174E1C783378E4B2DBB211
:10AB40009C420ED0144D01E0A3420AD00133282BC1
:10AB500028BF00230879E85CC0B2C871087D0728C7
:10AB6000F2D9DBB2034933700B79180644BF7C235A
:10AB7000CB70C5E700B00640489EFF1FDD9DFF1F5C
:10AB8000089EFF1FD89DFF1F4C9EFF1FDC9DFF1FCF
:10AB9000509EFF1F499EFF1FE09DFF1F70B584B0B0
:10ABA00072B6194B194D1A48702241260F24802184
:10ABB0001A702E701A460470197013781B06FCD593
:10ABC000144B186862B6144B144C984298BF00EBB3
:10ABD000800001A998BF40000A22FDF735FF01A9B6
:10ABE0002046002311F8012B01333AB10A2B20F83B
:10ABF000022FF7D11623237004B070BD5B00DBB2C7
:10AC0000237004B070BD00BF000002400700024086
:10AC100006000240080002407F969800C890FF1F7F
:10AC20002DE9F043DFF8EC808BB006460F4600F0CC
:10AC300073F898F90030013304460D4637D030469A
:10AC4000394600F0DFF9002831D02BA3D3E90023E7
:10AC50003046394600F026FE814668BB28A3D3E97A
:10AC600000233046394600F0FFFD00B398F900306C
:10AC7000254ACDF82090042400200021022BCDE9A4
:10AC80000467CDE9026700940192CDE906012CD05A
:10AC9000684600F0BDF940B3089B1BB101F0AAF96A
:10ACA000089B0360DDE906010BB0BDE8F083204698
:10ACB00029460BB0BDE8F083134A98F900300192A1
:10ACC00003210022CDE90467CDE9026700910892D3
:10ACD0002BB90E4B4FF06042CDE90623D8E70C4963
:10ACE0000020022BCDE90601D2D101F083F9222305
:10ACF0000360D1E7AFF30080EF39FAFE422E8640C1
:10AD000051302DD5104987C0ECE40000FFFFEF471C
:10AD10000000F07FDE90FF1F2DE9F04FB04F21F0D3
:10AD20000042BA4283B00C464FEAD17605460DD9AF
:10AD3000AC4FBA4225D9C1F31303034340F0EF806F
:10AD40000EB10020014603B0BDE8F08FA64B9A4239
:10AD500000F2CC80A54B9A4200F2DE808AA3D3E9B0
:10AD6000002300F05DF90022A14B00F09BFD0028BC
:10AD700000F005812846214600229D4B00F050F945
:10AD8000E1E783A3D3E9002300F08CFD002840F025
:10AD9000CB802846214680A3D3E9002300F064FD40
:10ADA0000028CED1934B284603EBC60821467CA34E
:10ADB000D3E9002300F0E6FAD8E9002300F030F9E7
:10ADC00000F07AFD804600F077FA77A3D3E90023FC
:10ADD00006460F4600F0D6FA02460B4628462146A4
:10ADE00000F01CF972A3D3E90023CDE9000130463D
:10ADF000394600F0C7FA82468B4652465B46DDE98B
:10AE0000000100F00BF905460C462A462346284669
:10AE1000214600F0B7FA68A3D3E9002306460F469F
:10AE200000F0B0FA66A3D3E9002300F0F7F8324649
:10AE30003B4600F0A7FA64A3D3E9002300F0F0F842
:10AE400032463B4600F09EFA61A3D3E9002300F0AE
:10AE5000E5F832463B4600F095FA5FA3D3E90023BC
:10AE600000F0DEF832463B4600F08CFA02460B4614
:10AE70002846214600F0D2F806460F4628462146CD
:10AE800032463B46B8F1000F56D000F07BFA32460E
:10AE900004460D463B4600204FF0804100F0BEF8CE
:10AEA00002460B462046294600F096FB02460B461A
:10AEB0005046594600F0B2F8DDE9002300F0AEF844
:10AEC0000B4602464A49002000F0A8F86FF47F7351
:10AED00098454FDA08F57A7801EB085100224FF0D7
:10AEE000B87300F04FFA03B0BDE8F08F424B9A42BE
:10AEF0003FF658AF414BF4002344D3E9002300F060
:10AF00008DF83F4BC6F101081C44CDE90001D4E99E
:10AF100000ABC6EB080870E74FF0000875E7024683
:10AF20000B4600F07DF80EE717A3D3E90023104687
:10AF3000194600F027FA06E700F024FA00228046BE
:10AF400089464FF080433046394600F067F80246A4
:10AF50000B464046494600F03FFB2A46234600F098
:10AF60005DF802460B460020214900F057F803B077
:10AF7000BDE8F08F01EB085103B0BDE8F08F8046CB
:10AF800043E700BFAFF300809C7500883CE4377E48
:10AF9000EF39FAFE422E864051302DD5104987C038
:10AFA000FE822B654715F73F0000E0FE422EE63F8C
:10AFB000763C7935EF39EA3DD0A4BE726937663EFA
:10AFC000F16BD2C541BDBB3E2CDE25AF6A56113FA9
:10AFD00093BDBE166CC1663F3E5555555555C53F90
:10AFE000412E8640FFFFEF7F422ED63FFFFF2F3ED0
:10AFF0000000F03FF0E40000B1A2F03F10E50000D7
:10B0000000E5000041F0004101F58010C00F7047DD
:10B010000020704781F0004102E000BF83F0004350
:10B0200030B54FEA41044FEA430594EA050F08BFE3
:10B0300090EA020F1FBF54EA000C55EA020C7FEAA7
:10B04000645C7FEA655C00F0E2804FEA5454D4EB24
:10B050005555B8BF6D420CDD2C4480EA020281EAEE
:10B06000030382EA000083EA010180EA020281EA26
:10B070000303362D88BF30BD11F0004F4FEA013178
:10B080004FF4801C4CEA113102D0404261EB410187
:10B0900013F0004F4FEA03334CEA133302D052420D
:10B0A00063EB430394EA050F00F0A780A4F10104C9
:10B0B000D5F1200E0DDB02FA0EFC22FA05F2801803
:10B0C00041F1000103FA0EF2801843FA05F35941E9
:10B0D0000EE0A5F120050EF1200E012A03FA0EFC68
:10B0E00028BF4CF0020C43FA05F3C01851EBE37192
:10B0F00001F0004507D54FF0000EDCF1000C7EEBAF
:10B1000000006EEB0101B1F5801F1BD3B1F5001FEC
:10B110000CD349085FEA30004FEA3C0C04F101040B
:10B120004FEA445212F5800F80F09A80BCF1004F34
:10B1300008BF5FEA500C50F1000041EB045141EAB6
:10B14000050130BD5FEA4C0C404141EB010111F4B7
:10B15000801FA4F10104E9D191F0000F04BF014662
:10B160000020B1FA81F308BF2033A3F10B03B3F140
:10B1700020020CDA0C3208DD02F1140CC2F10C02D0
:10B1800001FA0CF021FA02F10CE002F11402D8BF2E
:10B19000C2F1200C01FA02F120FA0CFCDCBF41EAFA
:10B1A0000C019040E41AA2BF01EB0451294330BDC9
:10B1B0006FEA04041F3C1CDA0C340EDC04F11404A6
:10B1C000C4F1200220FA04F001FA02F340EA03007D
:10B1D00021FA04F345EA030130BDC4F10C04C4F1C3
:10B1E000200220FA02F001FA04F340EA03002946A3
:10B1F00030BD21FA04F0294630BD94F0000F83F4ED
:10B20000801306BF81F480110134013D4EE77FEACF
:10B21000645C18BF7FEA655C29D094EA050F08BF1B
:10B2200090EA020F05D054EA000C04BF19461046FC
:10B2300030BD91EA030F1EBF0021002030BD5FEA40
:10B24000545C05D14000494128BF41F0004130BD68
:10B2500014F580043CBF01F5801130BD01F00045BC
:10B2600045F0FE4141F470014FF0000030BD7FEA2F
:10B27000645C1ABF194610467FEA655C1CBF0B462A
:10B28000024650EA013406BF52EA033591EA030F41
:10B2900041F4002130BD00BF90F0000F04BF002139
:10B2A000704730B54FF4806404F132044FF000056C
:10B2B0004FF0000150E700BF90F0000F04BF0021E5
:10B2C000704730B54FF4806404F1320410F000454B
:10B2D00048BF40424FF000013EE700BF42004FEA46
:10B2E000E2014FEA31014FEA02701FBF12F07F43C3
:10B2F00093F07F4F81F06051704792F0000F14BFC0
:10B3000093F07F4F704730B54FF4607401F0004503
:10B3100021F0004120E700BF50EA010208BF70475A
:10B3200030B54FF000050AE050EA010208BF70474F
:10B3300030B511F0004502D5404261EB41014FF4B8
:10B34000806404F132045FEA915C3FF4DCAE4FF0BC
:10B3500003025FEADC0C18BF03325FEADC0C18BFA3
:10B36000033202EBDC02C2F1200300FA03FC20FAF4
:10B3700002F001FA03FE40EA0E0021FA02F1144441
:10B38000C1E600BF70B54FF0FF0C4CF4E06C1CEA56
:10B3900011541DBF1CEA135594EA0C0F95EA0C0FCB
:10B3A00000F0DEF82C4481EA030621EA4C5123EA3E
:10B3B0004C5350EA013518BF52EA033541F480116D
:10B3C00043F4801338D0A0FB02CE4FF00005E1FB20
:10B3D00002E506F00042E0FB03E54FF00006E1FB6A
:10B3E00003569CF0000F18BF4EF0010EA4F1FF04AD
:10B3F000B6F5007F64F5407404D25FEA4E0E6D41ED
:10B4000046EB060642EAC62141EA55514FEAC520FD
:10B4100040EA5E504FEACE2EB4F1FD0C88BFBCF579
:10B42000E06F1ED8BEF1004F08BF5FEA500E50F12A
:10B43000000041EB045170BD06F0004646EA0101F0
:10B4400040EA020081EA0301B4EB5C04C2BFD4EB22
:10B450000C0541EA045170BD41F480114FF0000E1B
:10B46000013C00F3AB8014F1360FDEBF002001F089
:10B47000004170BDC4F10004203C35DA0C341BDC03
:10B4800004F11404C4F1200500FA05F320FA04F0D5
:10B4900001FA05F240EA020001F0004221F0004109
:10B4A00010EBD37021FA04F642EB06015EEA430E7C
:10B4B00008BF20EAD37070BDC4F10C04C4F12005AC
:10B4C00000FA04F320FA05F001FA04F240EA02005F
:10B4D00001F0004110EBD37041F100015EEA430E30
:10B4E00008BF20EAD37070BDC4F1200500FA05F250
:10B4F0004EEA020E20FA04F301FA05F243EA0203CF
:10B5000021FA04F001F0004121FA04F220EA0200DD
:10B5100000EBD3705EEA430E08BF20EAD37070BD23
:10B5200094F0000F0FD101F00046400041EB010103
:10B5300011F4801F08BF013CF7D041EA060195F0E5
:10B54000000F18BF704703F00046520043EB03039F
:10B5500013F4801F08BF013DF7D043EA060370478C
:10B5600094EA0C0F0CEA135518BF95EA0C0F0CD097
:10B5700050EA410618BF52EA4306D1D181EA0301DD
:10B5800001F000414FF0000070BD50EA410606BFD7
:10B590001046194652EA430619D094EA0C0F02D11C
:10B5A00050EA013613D195EA0C0F05D152EA033661
:10B5B0001CBF104619460AD181EA030101F000417F
:10B5C00041F0FE4141F470014FF0000070BD41F0C8
:10B5D000FE4141F4780170BD70B54FF0FF0C4CF4A2
:10B5E000E06C1CEA11541DBF1CEA135594EA0C0FC1
:10B5F00095EA0C0F00F0A7F8A4EB050481EA030E0E
:10B6000052EA03354FEA013100F088804FEA0333F4
:10B610004FF0805545EA131343EA12634FEA0222C2
:10B6200045EA111545EA10654FEA00260EF0004183
:10B630009D4208BF964244F1FD0404F5407402D2D5
:10B640005B084FEA3202B61A65EB03055B084FEA66
:10B6500032024FF480104FF4002CB6EB020E75EB63
:10B66000030E22BFB61A754640EA0C005B084FEA8B
:10B670003202B6EB020E75EB030E22BFB61A754608
:10B6800040EA5C005B084FEA3202B6EB020E75EB53
:10B69000030E22BFB61A754640EA9C005B084FEACB
:10B6A0003202B6EB020E75EB030E22BFB61A7546D8
:10B6B00040EADC0055EA060E18D04FEA051545EAC7
:10B6C00016754FEA06164FEAC30343EA52734FEA70
:10B6D000C2025FEA1C1CC0D111F4801F0BD141EAE9
:10B6E00000014FF000004FF0004CB6E711F4801F4E
:10B6F00004BF01430020B4F1FD0C88BFBCF5E06F2E
:10B700003FF6AFAEB5EB030C04BFB6EB020C5FEA3D
:10B71000500C50F1000041EB045170BD0EF0004E92
:10B720004EEA113114EB5C04C2BFD4EB0C0541EAC4
:10B73000045170BD41F480114FF0000E013C90E6C1
:10B7400045EA060E8DE60CEA135594EA0C0F08BF85
:10B7500095EA0C0F3FF43BAF94EA0C0F0AD150EA84
:10B7600001347FF434AF95EA0C0F7FF425AF104617
:10B7700019462CE795EA0C0F06D152EA03353FF43F
:10B78000FDAE1046194622E750EA410618BF52EABC
:10B7900043067FF4C5AE50EA41047FF40DAF52EA90
:10B7A00043057FF4EBAE12E74FF0FF3C06E000BF2D
:10B7B0004FF0010C02E000BF4FF0010C4DF804CD3A
:10B7C0004FEA410C7FEA6C5C4FEA430C18BF7FEAFA
:10B7D0006C5C1BD001B050EA410C0CBF52EA430C28
:10B7E00091EA030F02BF90EA020F0020704710F1A8
:10B7F000000F91EA030F58BF994208BF90422CBF37
:10B80000D8176FEAE37040F0010070474FEA410C2F
:10B810007FEA6C5C02D150EA013C07D14FEA430C4D
:10B820007FEA6C5CD6D152EA033CD3D05DF8040BBE
:10B83000704700BF8446104662468C4619466346F0
:10B8400000E000BF01B5FFF7B7FF002848BF10F1C7
:10B85000000F01BD4DF808EDFFF7F4FF0CBF01200C
:10B8600000205DF808FB00BF4DF808EDFFF7EAFF88
:10B8700034BF012000205DF808FB00BF4DF808ED43
:10B88000FFF7E0FF94BF012000205DF808FB00BF38
:10B890004DF808EDFFF7CEFF94BF012000205DF8C2
:10B8A00008FB00BF4DF808EDFFF7C4FF34BF0120CF
:10B8B00000205DF808FB00BF4FEA410212F50012BC
:10B8C00015D211D56FF47873B3EB625212D94FEAE7
:10B8D000C12343F0004343EA505311F0004F23FAD1
:10B8E00002F018BF404270474FF00000704750EA26
:10B8F000013005D111F0004008BF6FF000407047E3
:10B900004FF00000704700BF4FEA4102B2F1E04340
:10B9100024BFB3F5001CDCF1FE5C0DD901F0004C36
:10B920004FEAC0024CEA5070B2F1004F40EB830086
:10B9300008BF20F00100704711F0804F21D113F1B2
:10B940003872BCBF01F00040704741F480114FEAEB
:10B950005252C2F11802C2F1200C10FA0CF320FA74
:10B9600002F018BF40F001004FEAC1234FEAD32391
:10B9700003FA0CFC40EA0C0023FA02F34FEA4303FB
:10B98000CCE77FEA625307D150EA01331EBF4FF084
:10B99000FE4040F44000704701F0004040F0FE409F
:10B9A00040F40000704700BF80F0004002E000BF9C
:10B9B00081F0004142001FBF5FEA410392EA030F9A
:10B9C0007FEA226C7FEA236C6AD04FEA1262D2EBE4
:10B9D0001363C1BFD218414048404140B8BF5B42E9
:10B9E000192B88BF704710F0004F40F4000020F082
:10B9F0007F4018BF404211F0004F41F4000121F098
:10BA00007F4118BF494292EA030F3FD0A2F10102E1
:10BA100041FA03FC10EB0C00C3F1200301FA03F11F
:10BA200000F0004302D5494260EB4000B0F5000F42
:10BA300013D3B0F1807F06D340084FEA310102F101
:10BA40000102FE2A51D2B1F1004F40EBC25008BFB3
:10BA500020F0010040EA03007047490040EB00007D
:10BA600010F4000FA2F10102EDD1B0FA80FCACF1AC
:10BA7000080CB2EB0C0200FA0CF0AABF00EBC250AB
:10BA800052421843BCBFD0401843704792F0000F99
:10BA900081F4000106BF80F400000132013BB5E7EC
:10BAA0004FEA41037FEA226C18BF7FEA236C21D062
:10BAB00092EA030F04D092F0000F08BF08467047C7
:10BAC00090EA010F1CBF0020704712F07F4F04D195
:10BAD000400028BF40F00040704712F100723CBFA8
:10BAE00000F50000704700F0004343F0FE4040F4D2
:10BAF000000070477FEA226216BF08467FEA236390
:10BB00000146420206BF5FEA412390EA010F40F47A
:10BB1000800070474FF0000304E000BF10F00043C6
:10BB200048BF40425FEA000C08BF704743F09643AD
:10BB300001464FF000001CE050EA010208BF7047C8
:10BB40004FF000030AE000BF50EA010208BF70474F
:10BB500011F0004302D5404261EB41015FEA010C64
:10BB600002BF84460146002043F0B64308BFA3F15C
:10BB70008053A3F50003BCFA8CF2083AA3EBC2533E
:10BB800010DB01FA02FC634400FA02FCC2F120025D
:10BB9000BCF1004F20FA02F243EB020008BF20F094
:10BBA0000100704702F1200201FA02FCC2F12002FA
:10BBB00050EA4C0021FA02F243EB020008BF20EAEF
:10BBC000DC7070474FF0FF0C1CEAD0521EBF1CEA1D
:10BBD000D15392EA0C0F93EA0C0F6FD01A4480EA0B
:10BBE000010C400218BF5FEA41211ED04FF00063F4
:10BBF00043EA501043EA5111A0FB01310CF0004020
:10BC0000B1F5000F3EBF490041EAD3715B0040EA45
:10BC1000010062F17F02FD2A1DD8B3F1004F40EB15
:10BC2000C25008BF20F00100704790F0000F0CF0E8
:10BC3000004C08BF49024CEA502040EA51207F3AAC
:10BC4000C2BFD2F1FF0340EAC250704740F4000087
:10BC50004FF00003013A5DDC12F1190FDCBF00F078
:10BC600000407047C2F10002410021FA02F1C2F126
:10BC7000200200FA02FC5FEA310040F1000053EAC2
:10BC80004C0308BF20EADC70704792F0000F00F010
:10BC9000004C02BF400010F4000F013AF9D040EA16
:10BCA0000C0093F0000F01F0004C02BF490011F4AA
:10BCB000000F013BF9D041EA0C018FE70CEAD153A8
:10BCC00092EA0C0F18BF93EA0C0F0AD030F0004C28
:10BCD00018BF31F0004CD8D180EA010000F00040DC
:10BCE000704790F0000F17BF90F0004F084691F09A
:10BCF000000F91F0004F14D092EA0C0F01D14202D4
:10BD00000FD193EA0C0F03D14B0218BF084608D19C
:10BD100080EA010000F0004040F0FE4040F40000E6
:10BD2000704740F0FE4040F4400070474FF0FF0C79
:10BD30001CEAD0521EBF1CEAD15392EA0C0F93EAC0
:10BD40000C0F69D0A2EB030280EA010C49024FEA12
:10BD5000402037D04FF0805343EA111143EA1013CB
:10BD60000CF000408B4238BF5B0042F17D024FF483
:10BD7000000C8B4224BF5B1A40EA0C00B3EB510F5E
:10BD800024BFA3EB510340EA5C00B3EB910F24BF47
:10BD9000A3EB910340EA9C00B3EBD10F24BFA3EBCC
:10BDA000D10340EADC001B0118BF5FEA1C1CE0D194
:10BDB000FD2A3FF650AF8B4240EBC25008BF20F047
:10BDC000010070470CF0004C4CEA50207F32C2BF9B
:10BDD000D2F1FF0340EAC250704740F400004FF038
:10BDE0000003013A37E792F0000F00F0004C02BF69
:10BDF000400010F4000F013AF9D040EA0C0093F033
:10BE0000000F01F0004C02BF490011F4000F013B8C
:10BE1000F9D041EA0C0195E70CEAD15392EA0C0FF4
:10BE200008D142027FF47DAF93EA0C0F7FF470AF2C
:10BE3000084676E793EA0C0F04D14B023FF44CAF6F
:10BE400008466EE730F0004C18BF31F0004CCAD104
:10BE500030F000427FF45CAF31F000437FF43CAF40
:10BE60005FE700BF4FF0FF3C06E000BF4FF0010C62
:10BE700002E000BF4FF0010C4DF804CD4FEA400244
:10BE80004FEA41037FEA226C18BF7FEA236C11D08E
:10BE900001B052EA530C18BF90EA010F58BFB2EB41
:10BEA000030088BFC81738BF6FEAE17018BF40F0C1
:10BEB000010070477FEA226C02D15FEA402C05D175
:10BEC0007FEA236CE4D15FEA412CE1D05DF8040BFA
:10BED000704700BF844608466146FFE70FB5FFF78D
:10BEE000C9FF002848BF10F1000F0FBD4DF808ED45
:10BEF000FFF7F4FF0CBF012000205DF808FB00BF36
:10BF00004DF808EDFFF7EAFF34BF012000205DF88F
:10BF100008FB00BF4DF808EDFFF7E0FF94BF0120DC
:10BF200000205DF808FB00BF4DF808EDFFF7D2FFD9
:10BF300094BF012000205DF808FB00BF4DF808ED1C
:10BF4000FFF7C8FF34BF012000205DF808FB00BFE9
:10BF50004FEA4002B2F1FE4F0FD34FF09E03B3EB16
:10BF600012620DD94FEA002343F0004310F0004F56
:10BF700023FA02F018BF404270474FF000007047AC
:10BF800012F1610F01D1420205D110F0004008BF4B
:10BF90006FF0004070474FF00000704742000ED233
:10BFA000B2F1FE4F0BD34FF09E03B3EB126209D4F4
:10BFB0004FEA002343F0004323FA02F070474FF0AA
:10BFC0000000704712F1610F01D1420202D14FF01F
:10BFD000FF3070474FF00000704700BF0B4601462E
:10BFE000184600F001B800BF13460A460146022079
:10BFF00000F008BC014B1868704700BF0895FF1F90
:10C0000070B50F4E0F4D761BB61018BF002405D02B
:10C01000013455F8043B9847A642F9D10A4E0B4D1E
:10C02000761B02F07FFAB61018BF002406D0013448
:10C0300055F8043B9847A642F9D170BD70BD00BFCA
:10C0400030E5000030E5000040E5000030E500008C
:10C05000024B0146186800F00BB800BF0895FF1F9F
:10C06000024B0146186800F091BC00BF0895FF1F05
:10C070002DE9F04F01F10B05162D83B0064640F275
:10C080009F8035F0070500F1BF80A94200F2BC8017
:10C0900000F0F4FAB5F5FC7FC0F09C826B0A00F06A
:10C0A000BA80042B00F28381A80900F1390E4FEA0F
:10C0B0004E033830C44F07EB8303A3F108015C68DB
:10C0C000A14207D1ACE0002A80F2AC80E468A14232
:10C0D00000F0A680636823F003035A1B0F2AF2DDE9
:10C0E000B9493C6901F1080E744500F0B3816368F9
:10C0F00023F003035A1B0F2A00F39981002AC1F889
:10C1000014E0C1F810E080F29E80B3F5007F80F06B
:10C110006781DB0803F1010C01229B1002FA03F393
:10C120004A6851F83C80C4F8088001EBCC091A43F6
:10C13000A9F10803E3604A6041F83C40C8F80C40AC
:10C14000831001249C40944200F28A80144206D15C
:10C1500020F003006400144200F10400FAD007EB61
:10C16000C009CC468046DCF80C108C4507D173E141
:10C17000002A80F28181C9688C4500F06D814B688E
:10C1800023F003035A1B0F2AF2DD0C46D1F80CC032
:10C1900054F8088F4B1945F001054D6042F001013C
:10C1A000C8F80CC03046CCF808807B613B61C3F80E
:10C1B0000CE0C3F808E059609A5000F061FA1FE003
:10C1C000102921D800F05AFA1025062302207E4FAC
:10C1D00007EB8303A3F108025C68944200F04581F9
:10C1E0006368E168A56823F00303234430465A6876
:10C1F000E96042F001028D605A6000F041FA0834B3
:10C20000204603B0BDE8F08F00240C2320463360A5
:10C2100003B0BDE8F08F80234FF0400E3F2049E788
:10C2200070465DE72344E1685A68A56842F0010260
:10C23000E96030468D605A6000F022FA08342046EA
:10C2400003B0BDE8F08F234430465A6842F0010243
:10C250005A6000F015FA0834204603B0BDE8F08FAC
:10C26000BC68636823F00308A84504D3C5EB080342
:10C270000F2B00F38C80554BDFF860911A68D9F8CA
:10C28000003001332A4404EB080A00F0608102F513
:10C2900080520F3222F47F6222F00F0211463046A4
:10C2A000019200F0EFF9B0F1FF3F8346019A00F0F0
:10C2B0005881824500F2FC80454B1968DA451144EB
:10C2C000196000F05381D9F80000DFF810E1013067
:10C2D0001BBFCAEB0B0A5144CEF800B019601BF02B
:10C2E000070100F01781C1F10800C1F580518344B6
:10C2F00008315A44C2F30B02C2EB010949463046E9
:10C30000019300F0BFF9431C019B00F03F81CBEB90
:10C3100000024A4442F001021968C7F808B04944D3
:10C32000BC42CBF804201960DFF8A49016D0B8F115
:10C330000F0F40F2FD806268A8F10C0323F00703A1
:10C34000E01802F001024FF0050E1A430F2B626055
:10C35000C0F804E0C0F808E000F21C811D4BBC6886
:10C360001A68914288BF19601B4B1A689142626833
:10C3700088BF196022F003029542A2EB050301D8A1
:10C380000F2B04DC304600F07BF9002438E76219FB
:10C3900043F0010345F0010565603046BA60536023
:10C3A00000F06EF90834204603B0BDE8F08F142B7E
:10C3B00071D9542B00F2A480280B00F16F0E4FEAC4
:10C3C0004E036E3076E600BF0C95FF1F5C9EFF1F8C
:10C3D000609EFF1F589EFF1F549EFF1F1899FF1F4E
:10C3E0005A0A042A5ED9142A00F2B38002F15C01D1
:10C3F00049005B3207EB810C57F82110DFF8DC8134
:10C40000ACF1080C8C4500F088804A6822F00302E9
:10C41000934202D289688C45F7D1D1F80CC07A6872
:10C42000C4F80CC0A160CCF80840CC6088E6631961
:10C4300042F0010745F00105656030464B610B6134
:10C44000C3F80CE0C3F808E05F609A50083400F0CD
:10C4500017F9D5E64A6873E608F1010818F0030FEA
:10C460000CF1080C7FF47FAE30E0DC68A34208BF1B
:10C4700002303FF435AEB3E60B440C465A68C96847
:10C4800054F8085F42F001025A603046E9608D605E
:10C4900000F0F6F8B4E603F15C0E03F15B004FEA3E
:10C4A0004E0307E69A0902F1390149003832A1E743
:10C4B000BC424A4B3FF400AF9C68626822F0030222
:10C4C0005AE759F80839994540F0828010F0030F77
:10C4D00000F1FF30F5D17B6823EA04037B60640040
:10C4E0009C423FF6BDAE002C3FF4BAAE1C42404623
:10C4F0007FF435AE64001C4200F10400FAD02EE651
:10C50000B3F5AA7F18D8E80B00F1780E4FEA4E0376
:10C510007730CFE54FF48051EBE60121D8F80430B5
:10C52000921001FA02F21A43C8F80420614677E734
:10C530000123CBF8043025E740F25452934220D82F
:10C54000A80C00F17D0E4FEA4E037C30B2E51032AC
:10C55000A4E6542A26D81A0B02F16F0149006E3264
:10C5600048E7BC68626822F0030205E7CAF30B00E3
:10C5700000287FF4A8AE4244BB6842F001025A6032
:10C58000ECE6FE234FF07F0E7E2093E501224FF074
:10C590000009C1E604F10801304600F0F7F9D9F8C6
:10C5A0000010DBE6B2F5AA7F05D8DA0B02F17801BC
:10C5B000490077321EE740F254518A4205D89A0C5E
:10C5C00002F17D0149007C3214E7FE217E2211E751
:10C5D0007B6884E7E808431C5B00F8E50C95FF1FC7
:10C5E00070B4840746D0541E002A41D0CDB2034611
:10C5F00002E0621EE4B3144603F8015B9A07F8D127
:10C60000032C2ED9CDB245EA05250F2C45EA054568
:10C6100019D903F110022646103E0F2E42F8105C85
:10C6200042F80C5C42F8085C42F8045C02F110022B
:10C63000F2D8A4F1100222F00F0204F00F0410321D
:10C64000032C13440DD91E462246043A032A46F809
:10C65000045BFAD8221F22F003020432134404F0D0
:10C6600003042CB1C9B21C4403F8011BA342FBD143
:10C6700070BC704714460346C2E700BF704700BF56
:10C68000704700BF38B5074C0023054608462360B5
:10C69000FCF7A4F9431C00D038BD2368002BFBD065
:10C6A0002B6038BDBC9FFF1FFFFFFFFFFFFFFFFF99
:10C6B000FFFFFFFFFFFFFFFFFFFFFFFFFFFFFFFF8A
:10C6C00090F800F06DE9024520F007016FF0000CD2
:10C6D00010F0070491F820F040F049804FF000047A
:10C6E0006FF00700D1E9002391F840F000F1080055
:10C6F00082FA4CF2A4FA8CF283FA4CF3A2FA8CF38D
:10C700004BBBD1E9022382FA4CF200F10800A4FAF3
:10C710008CF283FA4CF3A2FA8CF3E3B9D1E9042347
:10C7200082FA4CF200F10800A4FA8CF283FA4CF37E
:10C73000A2FA8CF37BB9D1E9062301F1200182FA38
:10C740004CF200F10800A4FA8CF283FA4CF3A2FA3E
:10C750008CF3002BC6D0002A04BF04301A4612BA4C
:10C76000B2FA82F2FDE8024500EBD2007047D1E94F
:10C77000002304F00305C4F100004FEAC50514F0DE
:10C78000040F91F840F00CFA05F562EA05021CBFAF
:10C7900063EA050362464FF00004A9E740EA01039B
:10C7A0009B0770B42BD1032A29D90C460346214696
:10C7B00054F8046BA6F1013525EA060515F0803F13
:10C7C00006D1043A032A43F8046B2146EFD8A2B1FC
:10C7D0000C781C70013A013301313CB16AB111F897
:10C7E000014B03F8014B013A002CF7D12AB11A444E
:10C7F000002103F8011B9A42FBD170BC704703462D
:10C80000E5E700BF2DE9F047254C2568D5F84841FC
:10C810000646884692469946C4B360681F2817DCCE
:10C82000431C76B104EB80050122C5F888A0D4F83A
:10C83000881182401143022EC4F88811C5F808916E
:10C840001ED00230636044F820800020BDE8F087ED
:10C85000144B03B34FF4C870FFF7FAFB0446D0B192
:10C86000D5F84831002780E88800C5F848413846A7
:10C870000123C4F88871C4F88C71002EE1D0D1E78F
:10C88000D4F88C110A43C4F88C21DAE705F5A674B4
:10C89000C5F84841C1E74FF0FF30BDE8F08700BF61
:10C8A00020E5000051C00000024B13B1024800F027
:10C8B00005B8704700000000C9C800000023014609
:10C8C0001A461846FFF79EBF38B5074D074C2C1B7C
:10C8D000A41005D0013C55F8043D9847002CF9D12F
:10C8E000BDE8384001F02CBE000000000000000050
:10C8F000F8B5234F0C460646FFF7C0FEBB685D68DF
:10C9000025F00305291B01F6EF7121F47F6121F069
:10C910000F01A1F58054B4F5805F07DB002130469C
:10C92000FFF7B0FEBB682B44984204D03046FFF7B7
:10C93000A7FE0020F8BD61423046FFF7A3FE01309C
:10C940000DD0104BBA6819682D1B45F00105304613
:10C95000091B55601960FFF793FE0120F8BD002107
:10C960003046FFF78FFEBA68831A0F2BDEDD064CC8
:10C970000449246843F00103001B53600860D5E7B5
:10C980000C95FF1F609EFF1F1899FF1F002945D0BF
:10C990002DE9F0410D468046FFF770FE55F8047C06
:10C9A0006A4927F00103A5F10804E2188E6850686F
:10C9B000B24220F0030062D0FE0750600BD455F85D
:10C9C000087CE41B01F1080EA56875453B446FD057
:10C9D000E768EF60BD6015186D68ED0742D543F05C
:10C9E00001026260E350B3F5007F18D2DB085A1CE5
:10C9F0004D6851F83270A76001209B1000FA03F3D4
:10CA000001EBC2001D430838E0604D6041F8324040
:10CA1000FC604046BDE8F041FFF732BE70475A0A5D
:10CA2000042A53D89A0902F139077F0002F1380528
:10CA300001EB870051F827204449083890424DD037
:10CA4000516821F003018B4202D292689042F7D1E3
:10CA5000D068E060A2608460D4604046BDE8F041E8
:10CA6000FFF70EBE95683A4FBD4203443FD0D068F1
:10CA7000E86043F0010285606260E350B3E7FF07BE
:10CA8000034407D455F8082CA41A1344A068E2689C
:10CA9000C26090602F4A126843F0010093426060C8
:10CAA0008C60B6D32C4B40461968FFF721FFB0E7E6
:10CAB00011184968C90744D49168D268CA60034410
:10CAC00043F0010091606060E350A2E7142A17D898
:10CAD00002F15C077F0002F15B05A9E7AA104B6831
:10CAE000012505FA02F213434B600246B1E743F019
:10CAF00001024C610C61E560A5606260E35088E76B
:10CB0000542A06D81A0B02F16F077F0002F16E0556
:10CB10008EE7B2F5AA7F06D8DA0B02F178077F001C
:10CB200002F1770584E740F25450824206D89A0C0D
:10CB300002F17D077F0002F17C0579E7FE277E2563
:10CB400076E743F001026260E35062E70C95FF1F55
:10CB50001495FF1F1499FF1F5C9EFF1F0000CC104F
:10CB6000581BFC21AC26C62A7C2E3831F4334C36B7
:10CB7000A438983A5A3C543D803E7A3FFF3FFFFF2D
:10CB80000000580246056608540BD80E5C12701758
:10CB9000FC21F82A70305834DC37663A8C3C803EF1
:10CBA000FF3FFFFF0000FF03FF07FF0BFF0FFF1317
:10CBB000FF17FF1BFF1FFF23FF27FF2BFF2FFF3355
:10CBC000FF37FF3BFF3FFFFF0000580246056608A6
:10CBD000540BD80E5C12E015FA19141E6022AC2614
:10CBE0005C2B0C30BC34023AFF3FFFFF0000900189
:10CBF00020031405D0075A0AAC0DCC10B4146A18DF
:10CC0000E81C342180252A2B70301437FF3FFFFFAA
:10CC10000000C800F4018403140508072E091C0C49
:10CC2000D80EF811AE159619401F1C25F22B58345A
:10CC3000FF3FFFFF00006400C8009001BC021A041F
:10CC4000DC059E07F609800CA00F2413A2174C1DCB
:10CC50005424442FFF3FFFFF00005802460566089A
:10CC6000540BA00FD4172823F82A442F643284359C
:10CC70004038663A8C3C803EFF3FFFFF000078055D
:10CC8000220B0410B4143219B01DFC214826FE29D1
:10CC9000822D383126344637663A223DFF3FFFFF6A
:10CCA0000000540BEC13FA1908201C253629EC2C33
:10CCB0000C302C33E8357238663AF63B863D163F29
:10CCC000FF3FFFFF5CCB0000A0CC00005CCD00006C
:10CCD0007CCC0000A4CB0000C8CB0000ECCB000053
:10CCE00010CC000034CC000080CB000058CC0000F9
:10CCF00080CD0000F8CC00000000D007800CD80EDA
:10CD00000010C012EC130C17FA19141E6022AC2686
:10CD10005C2B0C30BC34023AFF3FFFFF00000000E8
:10CD2000CDCC4C3DCDCCCC3D9A99193ECDCC4C3E92
:10CD30000000803E9A99993E3333B33ECDCCCC3E31
:10CD40006666E63E2C011301FA00E100C800AF0060
:10CD500096007D0064004B00320019000000D007EF
:10CD6000100E88133219AA1E282374275C2B442F17
:10CD7000643284354038663A8C3C803EFF3FFFFF8A
:10CD8000000078053408540B800C3C0F5C12E01551
:10CD9000FA19141E6022AC265C2B0C30BC34023A0B
:10CDA000FF3FFFFF14CE0000B699FF1F0000FF0FEA
:10CDB000929AFF1F0000FF0FB9330000E0CD000082
:10CDC000189AFF1F32005E01000000000000000002
:10CDD0005933000054485200534E53004D415800FF
:10CDE000544F5543482053454E53450045585452DF
:10CDF0004120434F4E54524F4C4C455200000000CE
:10CE000050495443482042454E440000424954454D
:10CE10000000000042524541544800FFECCD0000A4
:10CE20005E9AFF1FF401A00FEE99FF1FF401A00FFF
:10CE3000653300000CCE0000449AFF1FBC025C1258
:10CE40002E9AFF1FBC025C129D33000000CE000032
:10CE50005C9AFF1FF401A00F109AFF1FF401A00FAE
:10CE600081330000FCD4000090D50000A4D5000060
:10CE7000A8D50000ACD50000B0D50000B4D50000A6
:10CE8000B8D50000BCD5000098D50000C0D5000082
:10CE9000FCD40000F8D40000A0D50000FCD40000B1
:10CEA00090D5000094D5000098D500009CD50000D6
:10CEB000C4D50000C8D50000CCD50000D0D50000F6
:10CEC000D4D50000D8D50000DCD50000E0D50000A6
:10CED000E4D50000E8D50000ECD50000F0D5000056
:10CEE000F4D50000000000005CD7000044D700002B
:10CEF000529AFF1F0000300000000000F9440000BB
:10CF0000254A0000000000000000000000000000B2
:10CF10000000000000000000000000000000000011
:10CF20000000000000000000000000000000000001
:10CF300000000000000000000000000000000000F1
:10CF400000000000000000000000000000000000E1
:10CF500000000000000000000000000000000000D1
:10CF600000000000000000000000000000000000C1
:10CF700000000000000000000000000000000000B1
:10CF800000000000000000000000000000000000A1
:10CF90000000000000000000000000000000000091
:10CFA0000000000000000000000000000000000081
:10CFB0000000000000000000000000000000000071
:10CFC0000000000000000000000000000000000061
:10CFD0000000000000000000000000000000000051
:10CFE0000000000000000000000000000000000041
:10CFF0000000000000000000000000000000000031
:10D000000000000000000000000000000000000020
:10D010000000000000000000000000000000000010
:10D020000000000000000000000000000001FFFF01
:10D03000FFE3600007736000000000000001FFFFD5
:10D04000FFE360000EE360000000000000018000CC
:10D05000000360001DC36000000000000001BFFF6E
:10D06000FFE360003B836000000000000001BFFFA1
:10D07000FFE3600077036000000000000001B000E3
:10D0800000036000EE036000000000000001B0003B
:10D0900000036001DC036000000000000001B0003C
:10D0A00000036003B8036000000000200001B0002E
:10D0B0000003600770036000000000600001BFFF14
:10D0C000FFE3600EE0036000000000600001BFFFAE
:10D0D000FFE3601DC00360000003006000018000EA
:10D0E0000003603B80036000000300E00001BFFF1D
:10D0F000FFE3607700036000000300C00001BFFF92
:10D10000FFE360EE00036000000380C00001B00098
:10D11000000361DC00036000000780C00001B00074
:10D12000000363B8000360000007C0C00001B00046
:10D1300000036770000360000006C0C00001B0007B
:10D1400000036EE000036000000660C10101B00052
:10D1500000037DC000036000000630C30301BFFF71
:10D16000FFE37B8000036000000C30C30701BFFFBA
:10D17000FFE3770000036000000C1CC30601800081
:10D1800000030E0000036000000C0CC20E01FFFF44
:10D19000FFE3FC0000036000000C0EC61E01FFFF51
:10D1A000FFE3F80000036000000C07C61E0000004B
:10D1B0000000000000000000000C03C67600000024
:10D1C0000000000000000000000C01C7E6000000A5
:10D1D0000000000000000000000C00C7C6000000B6
:10D1E0000000000000000000000C0003060000002A
:10D1F0000000000000000000000C00000000000023
:10D200000000000000000000000C00000000000012
:10D21000000000000000000000000000000000000E
:10D2200000000000000000000000000000000000FE
:10D2300000000000000000000000000000000000EE
:10D2400000000000000000000000000000000000DE
:10D2500000000000000000000000000000000000CE
:10D2600000000000000000000000000000000000BE
:10D2700000000000000000000000000000000000AE
:10D28000000000000000000000000000000000009E
:10D29000000000000000000000000000000000008E
:10D2A000000000000000000000000000000000007E
:10D2B000000000000000000000000000000000006E
:10D2C000000000000000000000000000000000005E
:10D2D000000000000000000000000000000000004E
:10D2E000000000000000000000000000000000003E
:10D2F000000000000000000000000000000000002E
:10D3000000000000000000000000000074D70000D2
:10D3100044D70000609AFF1F0000300000000000AA
:10D32000E944000069460000000000000100000020
:10D33000A8D700000300000000000000010000006A
:10D34000953D00000100000088D7000009000000A2
:10D3500001000000F8D500000700000000000000F8
:10D3600050D7000044D70000549AFF1F000030003F
:10D3700000000000F9440000254A00000000000001
:10D380000100000090D70000050000000000000030
:10D3900001000000AD5200000100000080D7000035
:10D3A0000800000000000000CCD60000CCD6000031
:10D3B0001A9AFF1F00000C0003000000614D0000DE
:10D3C00079460000000000000000000038D700008F
:10D3D00044D70000569AFF1F0000300000000000F4
:10D3E000F9440000254A0000000000000000000091
:10D3F000B0D70000B8D70000B899FF1F0100100097
:10D40000060000000D50000049460000FD450000E8
:10D410002C010000D53C00000600000008000000C0
:10D42000A88CFF1F10D700000200030006000000B8
:10D43000348DFF1F88D700000000050105000000A3
:10D44000E88AFF1FA4D600000000010108000000C8
:10D45000708DFF1F0000000068D7000044D7000057
:10D46000509AFF1F0000300000000000F944000047
:10D47000254A000000000000F8D500000000040567
:10D4800008000000888CFF1F0000000020D700006B
:10D490002CD700007E99FF1F000001000100000052
:10D4A0000D4100005946000000000000000000008F
:10D4B00054D6000020D60000FA99FF1F0000090092
:10D4C000000000003141000089460000000000001B
:10D4D000010000009CD700000400000000000000D4
:10D4E00001000000994600005CD600000000020127
:10D4F00006000000848AFF1F4F4E00004F46460082
:10D50000424154004C4F5720000000005553420048
:10D510004D454E55202020202020202020585858AE
:10D5200020592E595600000058000000524F540058
:10D530004D454C0044594E006D730000312F0000E2
:10D54000424954004C5652004E524D00524556002E
:10D550005042440043560000762E0000312E332EF8
:10D56000390000004E754556490000006669726D2D
:10D570007761726520762E0053455400434C52006B
:10D58000444F4E275400000050414E4943000000D4
:10D590004D57000046500000434600005350000025
:10D5A0005357000042520000564C000045580000FE
:10D5B0004D572B0042522B00564C2B0045582B0048
:10D5C000554E4F002D3400002D3300002D32000049
:10D5D0002D3100004C494E002B3100002B32000051
:10D5E0002B3300002B340000533100005332000075
:10D5F0005A3100005A3200005649425241544F00FD
:10D60000444952454354494F4E000000434F4E5445
:10D61000524F4C00535155454C43482042000000A6
:10D620004C4556454C00000053454E53452042544E
:10D6300045000000535155454C4348204C00000024
:10D6400053454E5345204C56520000005245545508
:10D65000524E000044455054480000005345545574
:10D6600050204354524C530050494E4B59204B4587
:10D67000590000004445474C49544348000000000D
:10D6800045585452412043545200000050495443DD
:10D690004842454E44000000504F52542F474C44DE
:10D6A0000000000053455455502042524541544813
:10D6B0000000000056454C20424941530000000044
:10D6C00056454C2044454C415900000043555256A4
:10D6D0004500000056454C4F434954590000000096
:10D6E00042524541544820415400000043433220F7
:10D6F00052495345000000004252544820434332EF
:10D700000000000042525448204343310000000012
:10D71000524F5441544F522053455455500000002D
:10D720005052494F52495459000000004D4F4E4F3E
:10D73000205052494F000000524F5441544520346C
:10D740000000000053454D49544F4E455300000022
:10D75000524F54415445203300000000524F544171
:10D760005445203200000000524F544154452031AE
:10D7700000000000504152414C4C454C000000005C
:10D7800041424F5554000000455854524153000047
:10D7900053455455502043544C00000053455455B4
:10D7A000502042520000000041444A5553540000AA
:10D7B0004D494449204348004D4944492043484E7F
:10D7C0004C000000574C20504F57455200000000BD
:10D7D00053504543204B45590000000047415445F4
:10D7E00020484F4C440000004C45474143592042DB
:10D7F000520000004C454741435920504200000070
:10D800004F435441564500005452414E53504F53DC
:10D810004500FFFF002111020200FFFF3480044099
:10D82000400000001211FFFFFF0202000000131071
:10D83000FFFFFF02020000001800000034800440D7
:10D84000800000001EFFFFFFFF02000000001DFF20
:10D85000FFFFFF02000000001900000000000000B0
:10D8600000000000C55E0000895E00003D5E000013
:10D87000855E0000415E00004D5E00006D5E0000B0
:10D88000000103070F1F3F7F2200FF2100FFFFFF62
:10D890000080C0E0F0F8FCFE000000000000000086
:10D8A000557F0000858200003D5E00008169000018
:10D8B000196A0000FD770000B1770000E5770000ED
:10D8C000BD770000D1770000CD760000FD77000025
:10D8D00025780000156C00005D740000F9730000ED
:10D8E000F57800000178000059790000F97900000E
:10D8F000DA02818FDA1281FF000060000000000070
:10D90000000000000000000000E000000000000037
:10D910000000000000000001E00000000000000026
:10D9200000000000000001F0000000000000000006
:10D93000000000000003F0000000000000000000F4
:10D940000000000007F000000000000000000000E0
:10D9500000000007F80000000000000000000000C8
:10D9600000000FF800000003C0007E000001E0008E
:10D970007F0FF800000003C000FE000001E000FF80
:10D98000EFF800000003C000FE000001E000FFFF10
:10D99000F800000003C000F00000000F007FFE7FD1
:10D9A000C0000003C000F00000000F003FFE7FF841
:10D9B0003FF1FBCFFCFEF3BC3DEFE01FFE7FFF7F9E
:10D9C000FBFFDFFEFEFFBC3DEFE01FC6FFFF7FFB5E
:10D9D000FFDFFEFEFFBC3DEFE00FE3C7FE787BC339
:10D9E000DE1EF0FFBC3DEF0007FF87FC787BC3DE47
:10D9F0001EF0F83C3DEF0001FFFFF0007BC3C01EAE
:10DA0000F0F03C3DEF0001F37FE03FFBC3CFFEF0C1
:10DA1000F03C3DEF0003E33F807FFBC3DFFEF0F00F
:10DA20003C3DEF0007E73C00787BC3DE1EF0F03C96
:10DA30003DEF0007FFBE00787BC3DE1EF0F03C3DEB
:10DA4000EF0007FFFE00787BC3DE1EF0F03C3DEFE9
:10DA5000000FFFFE007FFBFFDFFEF0F03FFDEFE079
:10DA60000FFFFF007FFBFFDFFEF0F03FFDEFE00F59
:10DA7000F9FF003E79F9CF9EF0F01F3DE7E01FF17E
:10DA8000FF0000000000000000000000001F80FFF9
:10DA9000007FFFFFFFFFFFFFFFFFFFE01C007F0095
:10DAA0007FFFFFFFFEB46D888D18E000001F007F30
:10DAB000FFFFFFFE95AD7DB577E000000F007FFF13
:10DAC000FFFFFEA5AD9D8D19E0000006007FFFFF62
:10DAD000FFFEB5ADEDB57EE0AED580A8D300408D9C
:10DAE0002000A1C8DB40A4A62EAFFFFF000000006D
:10DAF0000001800000000000000000000380000022
:10DB00000000000000000007C0000000000000004E
:10DB1000000007C00000000000000000000FC0006F
:10DB200000000000000000001FE0000000000000F6
:10DB30000000001FE00000000000000000003FE0C7
:10DB40000000000000000000003FF00000000000A6
:10DB5000000000007FF0000000000000001FF87FC0
:10DB6000F0000000000000003FFE7FF00000000019
:10DB70000000003FFF7FF0000000000000001FFFDA
:10DB8000FBE0000000000000000FFFF9FFC00000F4
:10DB9000000000000FFFF9FFF80000000000000780
:10DBA000FFF1FFFF00000000000003FC73FFFF8097
:10DBB000000000000001FE3FFFFF800000000000A9
:10DBC00000FF1E0FFF000000000000007FFE1FFC92
:10DBD000000000000000003FFFFFF8000000000010
:10DBE00000000FDFFFE0000000000000001F19FF31
:10DBF000C0000000000000003F3CFF0000000000EB
:10DC00000000007E7CF800000000000000007FFEA5
:10DC10007C0000000000000000FFFFFC000000008E
:10DC200000000000FFFFFE0000000000000000FFF9
:10DC3000FFFE0000000000000001FFEFFE000000FA
:10DC40000000000001FFCFFE000000000000000304
:10DC5000FF07FE0000000000000003FC07FE0000BC
:10DC6000000000000003F003FE00000000000000C0
:10DC7000018000FE000000000000000000007E00A7
:10DC80000000000000000000003E00000000000056
:10DC9000000000000C000000000000078000FC00F5
:10DCA0000003C0000000078001FC000003C000006A
:10DCB00000078001FC000003C0000000078001E0B5
:10DCC0000000001E000000078001E00000001E00B0
:10DCD0007FE3F79FF9FDE7787BDFC0FFF7FFBFFD2C
:10DCE000FDFF787BDFC0FFF7FFBFFDFDFF787BDF27
:10DCF000C0F0F787BC3DE1FF787BDE00F0F787BC22
:10DD00003DE1F0787BDE0000F787803DE1E0787B45
:10DD1000DE007FF7879FFDE1E0787BDE00FFF7877D
:10DD2000BFFDE1E0787BDE00F0F787BC3DE1E07805
:10DD30007BDE00F0F787BC3DE1E0787BDE00F0F7AA
:10DD400087BC3DE1E0787BDE00FFF7FFBFFDE1E04F
:10DD50007FFBDFC0FFF7FFBFFDE1E07FFBDFC07CA3
:10DD6000F3F39F3DE1E03E7BCFC0000000000000E8
:10DD70000000000000FFFFFFFFFFFFFFFFFFFFC0ED
:10DD8000FFFFFFFFFD68DB111A31C0FFFFFFFFFD42
:10DD90002B5AFB6AEFC0FFFFFFFFFD4B5B3B1A33C3
:10DDA000C0FFFFFFFFFD6B5BDB6AFDC0DA0281FF96
:10DDB0000000000000000000557F00008582000088
:10DDC0003D5E000081690000098A0000FD770000C7
:10DDD000B1770000E5770000BD770000D177000043
:10DDE000CD760000FD770000257800002178000046
:10DDF00049780000A1780000F57800000178000063
:10DE000059790000F979000000000000003E5B4FE6
:10DE10005B3E3E6B4F6B3E1C3E7C3E1C183C7E3C8A
:10DE2000181C577D571C1C5E7F5E1C00183C180098
:10DE3000FFE7C3E7FF0018241800FFE7DBE7FF3028
:10DE4000483A060E2629792926407F050507407F96
:10DE500005253F5A3CE73C5A7F3E1C1C08081C1C09
:10DE60003E7F14227F22145F5F005F5F06097F01FF
:10DE70007F006689956A606060606094A2FFA294EA
:10DE800008047E040810207E201008082A1C0808B8
:10DE90001C2A08081E101010100C1E0C1E0C303806
:10DEA0003E3830060E3E0E06000000000000005F07
:10DEB00000000007000700147F147F14242A7F2A23
:10DEC00012231308646236495620500008070300E5
:10DED000001C2241000041221C002A1C7F1C2A0831
:10DEE000083E080800807030000808080808000094
:10DEF00060600020100804023E5149453E00427F08
:10DF0000400072494949462141494D331814127F56
:10DF10001027454545393C4A4949314121110907F6
:10DF20003649494936464949291E00001400000077
:10DF30004034000000081422411414141414004149
:10DF400022140802015909063E415D594E7C121106
:10DF5000127C7F494949363E414141227F4141413E
:10DF60003E7F494949417F090909013E41415173B9
:10DF70007F0808087F00417F41002040413F017F2A
:10DF8000081422417F404040407F021C027F7F04F2
:10DF900008107F3E4141413E7F090909063E41513B
:10DFA000215E7F09192946264949493203017F012B
:10DFB000033F4040403F1F2040201F3F4038403F2C
:10DFC000631408146303047804036159494D430042
:10DFD0007F4141410204081020004141417F040279
:10DFE0000102044040404040000307080020545410
:10DFF00078407F28444438384444442838444428EE
:10E000007F385454541800087E090218A4A49C7840
:10E010007F0804047800447D40002040403D007F9C
:10E020001028440000417F40007C047804787C087C
:10E030000404783844444438FC1824241818242450
:10E0400018FC7C08040408485454542404043F4435
:10E05000243C4040207C1C2040201C3C4030403C64
:10E0600044281028444C9090907C4464544C4400C4
:10E070000836410000007700000041360800020128
:10E080000204023C2623263C1EA1A161123A404014
:10E09000207A385454555921555579412254547891
:10E0A00042215554784020545579400C1E5272122A
:10E0B00039555555593954545459395554545800B3
:10E0C00000457C410002457D420001457C407D12B7
:10E0D00011127DF0282528F07C5455450020545419
:10E0E0007C547C0A097F4932494949323A444444C4
:10E0F0003A324A4848303A4141217A3A42402078FF
:10E10000009DA0A07D3D4242423D3D4040403D3CFF
:10E1100024FF2424487E4943662B2FFC2F2BFF0924
:10E1200029F620C0887E0903205454794100004418
:10E130007D413048484A32384040227A007A0A0A03
:10E14000727D0D19317D2629292F28262929292676
:10E1500030484D4020380808080808080808382FBB
:10E1600010C8ACBA2F102834FA00007B0000081445
:10E170002A142222142A14085500550055AA55AA1B
:10E1800055AAFF55FF55FF000000FF00101010FFBB
:10E1900000141414FF001010FF00FF1010F010F016
:10E1A000141414FC001414F700FF0000FF00FF1407
:10E1B00014F404FC141417101F10101F101F141453
:10E1C000141F00101010F0000000001F101010109D
:10E1D0001F10101010F010000000FF101010101091
:10E1E00010101010FF10000000FF140000FF00FFCF
:10E1F00000001F10170000FC04F41414171017146B
:10E2000014F404F40000FF00F7141414141414148C
:10E21000F700F7141414171410101F101F141414FF
:10E22000F4141010F010F000001F101F0000001F69
:10E2300014000000FC140000F010F01010FF10FF9C
:10E24000141414FF141010101F00000000F010FF31
:10E25000FFFFFFFFF0F0F0F0F0FFFFFF0000000015
:10E2600000FFFF0F0F0F0F0F3844443844FC4A4A99
:10E270004A347E02020606027E027E02635549414E
:10E28000633844443C04407E201E2006027E020285
:10E2900099A5E7A5991C2A492A1C4C7201724C3099
:10E2A0004A4D4D303048784830BC625A463D3E4970
:10E2B0004949007E0101017E2A2A2A2A2A44445F14
:10E2C000444440514A444040444A51400000FF0108
:10E2D00003E080FF000008086B6B08361236243616
:10E2E000060F090F0600001818000000101000307B
:10E2F00040FF0101001F01011E00191D1712003C03
:10E300003C3C3C00000000000D0AFFFF050E080920
:10E310000D0C06070F0400130393050E08090D0CDE
:10E3200006070F04FFFFC585848687C4FFFF00131F
:10E3300003931A9217FFFFFF6FF07F0303700378B8
:10E3400013F0800FFBD070474008FE4340A004400C
:10E350004408FE4344A004400018FE4300C00440AB
:10E360003000FE43309004403400FE4334900440BB
:10E370001C18FE431CC004401018FE4310C004408B
:10E380000818FE4308C004400C18FE430CC00440AB
:10E390000C10FE430CB004401010FE4310B00440BB
:10E3A0001810FE4318B004401C10FE431CB004407B
:10E3B0001410FE4314B004400418FE4304C004408B
:10E3C0000010FE4300B004400008FE4300A00440DB
:10E3D0000408FE4304A004400C08FE430CA00440C3
:10E3E0000808FE4308A004401418FE4314C004406B
:10E3F0001818FE4318C004400410FE4304B0044043
:10E400000810FE4308B004401400FE43149004407A
:10E410004C08FE434CA004400420FE4304D00440BA
:10E420002410FE4324B004402010FE4320B00440DA
:10E430002810FE4328B004402C10FE432CB00440AA
:10E440000020FE4300D004404808FE4348A004409A
:10E450001000FE4310900440090AFFFFFFFFFFFF7A
:10E46000FFFFFFFFFFFFFF0D00060807FFFF0E0F76
:10E47000FF0CFFFFFFFFFFFF0B05FFFF151915192D
:10E48000000100000090FF1F1200000000020000C9
:10E490002C90FF1F7300000000220100A090FF1FBE
:10E4A00021000000002101008890FF1F09000000EA
:10E4B00000030000C490FF1F0000000001030904D6
:10E4C0001490FF1F0000000002030904208EFF1FAC
:10E4D0000000000003030904C890FF1F00000000B3
:10E4E00000000000000000000000000065787000DF
:10E4F000000000000000E03F000000000000E0BF5E
:10E50000763C7935EF39EA3D763C7935EF39EABD2D
:10E510000000E0FE422EE63F0000E0FE422EE6BF95
:10E52000E090FF1FF8B500BFF8BC08BC9E467047DE
:10E53000A9C800003504000031330000C94A0000BA
:04E54000F8B500BF6B
:10E5440038B5084B1C681C6054B1074D94FAA4F309
:10E55400B3FA83F355F823309847631E1C40F5D172
:10E5640038BD00BFA0D00440F08FFF1F38B5084B62
:10E574001C681C6054B1074D94FAA4F3B3FA83F3F6
:10E5840055F823309847631E1C40F5D138BD00BFB1
:10E59400A0C00440D08FFF1F38B5084B1C681C6016
:10E5A40054B1074D94FAA4F3B3FA83F355F8233026
:10E5B4009847631E1C40F5D138BD00BFA0B004408D
:10E5C400A08FFF1F38B5084B1C681C6054B1074D61
:10E5D40094FAA4F3B3FA83F355F823309847631EEF
:10E5E4001C40F5D138BD00BFA0A00440508FFF1FD0
:10E5F40038B5084B1C681C6054B1074D94FAA4F359
:10E60400B3FA83F355F823309847631E1C40F5D1C1
:10E6140038BD00BFA0900440188FFF1F0000000009
:10E624000020000032000000002000000020000054
:10E6340000100000AB0A000000080000660600009D
:10E644005505000092040000000400008E03000041
:10E6540033030000E8020000AB02000024000000C5
:10E66400002000000200020001000C00140500005C
:10E674000C0000000000F041000102070B0102073A
:10E684000B4A1400FBFFFFFF000000000000000025
:10E694000000000000000000000000000000000076
:10E6A40000000000000000000200FFFFFFFF000068
:10E6B400A4CD000034CE00004CCE00001CCE0000DF
:10E6C400BCCD00000000000034D6000020D60000BD
:10E6D4006A89FF1F01001E00000000000000000006
:10E6E400000000000000000000000000E0D6000070
:10E6F400E0D60000209AFF1F000001000100000086
:10E704000000000000000000000000000000000005
:10E7140040D6000020D600006489FF1F01000C00D1
:10E7240000000000000000000000000000000000E5
:10E7340000000000010000000000000000000000D4
:10E74400B4D60000B4D600005099FF1F00000900A1
:10E7540001000000000000000000000000000000B4
:10E76400000000004CD6000020D60000A889FF1F3E
:10E774000000040000000000000000000000000091
:10E7840000000000208BFF1F9C8AFF1F648CFF1F6A
:10E7940050D30000B08BFF1F4C8DFF1F0000000002
:10E7A4008CD600008CD60000329AFF1F00000C00AB
:10E7B4000000000000000000000000000000000055
:10E7C4000000000000D8000000D80000E499FF1FFA
:10E7D400000006000000000000000000000000002F
:10E7E4000000000001000000FC8AFF1F908DFF1F45
:10E7F4001C8CFF1FD48BFF1FD88DFF1F000000004F
:10E80400F4D70000F4D700005A9AFF1F000001005B
:10E8140001000000000000000000000000000000F3
:10E824000000000098D6000098D60000EC99FF1F65
:10E8340000000200010000000000000000000000D1
:10E844000000000000000000F8D60000F8D6000028
:10E854002C9AFF1F00007F00010000000000000050
:10E86400000000000000000000000000C0D600000E
:10E87400C0D60000249AFF1F00001E000100000003
:10E884000000000000000000000000000000000084
:10E89400ECD60000ECD600007099FF1F01000A00BE
:10E8A4000100000000000000000000000000000063
:10E8B4000000000074D6000074D60000909AFF1F78
:10E8C40000004600000000000000000000000000FE
:10E8D4000000000000000000D0D70000D0D70000E6
:10E8E4004C9AFF1F0000010001000000000000001E
:10E8F40000000000000000000000000008D8000034
:10E9040008D800008099FF1F0000180000000000D4
:10E9140000000000000000000000000000000000F3
:10E92400DCD70000DCD70000089AFF1F00000100BC
:10E9340001000000000000000000000000000000D2
:10E944000000000000D6000000D600008E9AFF1FD1
:10E9540000000100010000000000000000000000B1
:10E96400000000000000000080D6000080D60000F7
:10E97400589AFF1F0000040001000000000000007E
:10E984000000000000000000FC8DFF1FACD400005C
:10E99400608AFF1F408CFF1F0C8AFF1FC489FF1F62
:10E9A400C88CFF1FEC8CFF1FF88BFF1FC08AFF1F52
:10E9B400ECD300002CD30000D0D4000080D300009E
:10E9C40044D3000098D300000000000028D60000C3
:10E9D40020D600006689FF1F01000C000000000023
:10E9E4000000000000000000000000000000000023
:10E9F40014D6000020D600007089FF1F01001E00FD
:10EA04000000000000000000000000000000000002
:10EA14000000000004D7000004D700006299FF1F23
:10EA240000000A00010000000000000000000000D7
:10EA34000000000008D3000054D40000E4CE00001D
:10EA44005CD30000C8D3000088D40000000000009C
:10EA540068D6000068D60000889AFF1F00001800DE
:10EA640000000000000000000000000000000000A2
:10EA7400108DFF1F448BFF1F8C8BFF1FE889FF1F26
:10EA8400B48DFF1FA4D30000688BFF1F3C8AFF1FB7
:10EA940000000000E8D70000E8D70000DC99FF1F61
:10EAA4000000010001000000000000000000000060
:10EAB4000000000000000000D4D60000D4D60000FE
:10EAC4004099FF1F00007F000100000000000000CB
:10EAD400000000000000000000000000C4D7000097
:10EAE400C4D700008C99FF1F000003000000000041
:10EAF4000000000000000000000000000000000012
:10EB04000CD600000CD60000B299FF1F00000100D3
:10EB140001000000000000000000000000000000F0
:10EB240016034E00750045005600490020004D00B4
:10EB3400490044004900000064D8000000000000BF
:10EB4400E803000000000000006006401CD800003C
:10EB540000000000000000000000000000000000B1
:10EB640000000000000000000000000000000000A1
:10EB74000000000000000000000000000000000091
:10EB84000000000000000000000000000000000081
:10EB94000000000000000000000000000000000071
:10EBA4000000000064D8000000000000E80300003A
:10EBB40000000000007006403CD800000000000087
:10EBC4000000000000000000000000000000000041
:10EBD4000000000000000000000000000000000031
:10EBE4000000000000000000000000000000000021
:10EBF4000000000000000000000000000000000011
:10EC04000000000000000000000000000000000000
:10EC14000A040000C09FFF1F958A0000958A000027
:10EC2400958A0000958A0000958A0000958A000064
:10EC3400958A0000958A0000958A0000958A000054
:10EC4400958A0000958A0000958A0000958A000044
:10EC5400958A0000958A0000958A0000958A000034
:10EC6400958A0000958A0000958A0000958A000024
:10EC7400958A0000958A0000958A0000958A000014
:10EC8400958A0000958A0000958A0000958A000004
:10EC9400958A0000958A0000958A0000958A0000F4
:10ECA400958A0000958A0000958A0000958A0000E4
:10ECB400958A0000958A0000958A0000958A0000D4
:10ECC400958A0000958A0000958A0000958A0000C4
:10ECD400958A0000958A0000958A0000958A0000B4
:10ECE400958A0000958A0000958A0000958A0000A4
:10ECF400958A0000958A000008000000FFFFFFFFCE
:10ED04001201100100000040C016850475020102C2
:10ED14000301000018035400650065006E007300D1
:10ED240079006400750069006E006F0009027300C9
:10ED3400020100C03209040000020103000007249C
:10ED4400010001250006240201010006240202023A
:10ED54000009240301030102010009240302040140
:10ED6400010100090504024000000000052501011D
:10ED74000109058302400000000005250101030983
:10ED840004010002030000000921110100012221F5
:10ED9400000705810340000107050203200002006B
:10EDA40006C9FF0904A15C7508150026FF009540FB
:10EDB4000975810295200976910295040976B102BC
:10EDC400C0000000040309040C030000000000005C
:10EDD400000000000000000000000000000001002E
:10EDE40000000000CC93FF1F3494FF1F9C94FF1F6E
:10EDF400000000000000000000000000000000000F
:10EE040000000000000000000000000000000000FE
:10EE140000000000000000000000000000000000EE
:10EE240000000000000000000000000000000000DE
:10EE340000000000000000000000000000000000CE
:10EE440000000000000000000000000000000000BE
:10EE540000000000000000000000000000000000AE
:10EE6400000000000000000000000000000000009E
:10EE7400000000000000000000000000000000008E
:10EE8400000000000000000001000000000000007D
:10EE94000E33CDAB34126DE6ECDE05000B00000042
:10EEA400000000000000000000000000000000005E
:10EEB400000000000000000000000000000000004E
:10EEC400000000000000000000000000000000003E
:10EED400000000000000000000000000000000002E
:10F204000000000000000000E090FF1F000000006C
:10F21400000000000C95FF1F0C95FF1F1495FF1FA5
:10F224001495FF1F1C95FF1F1C95FF1F2495FF1F9E
:10F234002495FF1F2C95FF1F2C95FF1F3495FF1F4E
:10F244003495FF1F3C95FF1F3C95FF1F4495FF1FFE
:10F254004495FF1F4C95FF1F4C95FF1F5495FF1FAE
:10F264005495FF1F5C95FF1F5C95FF1F6495FF1F5E
:10F274006495FF1F6C95FF1F6C95FF1F7495FF1F0E
:10F284007495FF1F7C95FF1F7C95FF1F8495FF1FBE
:10F294008495FF1F8C95FF1F8C95FF1F9495FF1F6E
:10F2A4009495FF1F9C95FF1F9C95FF1FA495FF1F1E
:10F2B400A495FF1FAC95FF1FAC95FF1FB495FF1FCE
:10F2C400B495FF1FBC95FF1FBC95FF1FC495FF1F7E
:10F2D400C495FF1FCC95FF1FCC95FF1FD495FF1F2E
:10F2E400D495FF1FDC95FF1FDC95FF1FE495FF1FDE
:10F2F400E495FF1FEC95FF1FEC95FF1FF495FF1F8E
:10F30400F495FF1FFC95FF1FFC95FF1F0496FF1F3C
:10F314000496FF1F0C96FF1F0C96FF1F1496FF1FE9
:10F324001496FF1F1C96FF1F1C96FF1F2496FF1F99
:10F334002496FF1F2C96FF1F2C96FF1F3496FF1F49
:10F344003496FF1F3C96FF1F3C96FF1F4496FF1FF9
:10F354004496FF1F4C96FF1F4C96FF1F5496FF1FA9
:10F364005496FF1F5C96FF1F5C96FF1F6496FF1F59
:10F374006496FF1F6C96FF1F6C96FF1F7496FF1F09
:10F384007496FF1F7C96FF1F7C96FF1F8496FF1FB9
:10F394008496FF1F8C96FF1F8C96FF1F9496FF1F69
:10F3A4009496FF1F9C96FF1F9C96FF1FA496FF1F19
:10F3B400A496FF1FAC96FF1FAC96FF1FB496FF1FC9
:10F3C400B496FF1FBC96FF1FBC96FF1FC496FF1F79
:10F3D400C496FF1FCC96FF1FCC96FF1FD496FF1F29
:10F3E400D496FF1FDC96FF1FDC96FF1FE496FF1FD9
:10F3F400E496FF1FEC96FF1FEC96FF1FF496FF1F89
:10F40400F496FF1FFC96FF1FFC96FF1F0497FF1F37
:10F414000497FF1F0C97FF1F0C97FF1F1497FF1FE4
:10F424001497FF1F1C97FF1F1C97FF1F2497FF1F94
:10F434002497FF1F2C97FF1F2C97FF1F3497FF1F44
:10F444003497FF1F3C97FF1F3C97FF1F4497FF1FF4
:10F454004497FF1F4C97FF1F4C97FF1F5497FF1FA4
:10F464005497FF1F5C97FF1F5C97FF1F6497FF1F54
:10F474006497FF1F6C97FF1F6C97FF1F7497FF1F04
:10F484007497FF1F7C97FF1F7C97FF1F8497FF1FB4
:10F494008497FF1F8C97FF1F8C97FF1F9497FF1F64
:10F4A4009497FF1F9C97FF1F9C97FF1FA497FF1F14
:10F4B400A497FF1FAC97FF1FAC97FF1FB497FF1FC4
:10F4C400B497FF1FBC97FF1FBC97FF1FC497FF1F74
:10F4D400C497FF1FCC97FF1FCC97FF1FD497FF1F24
:10F4E400D497FF1FDC97FF1FDC97FF1FE497FF1FD4
:10F4F400E497FF1FEC97FF1FEC97FF1FF497FF1F84
:10F50400F497FF1FFC97FF1FFC97FF1F0498FF1F32
:10F514000498FF1F0C98FF1F0C98FF1F1498FF1FDF
:10F524001498FF1F1C98FF1F1C98FF1F2498FF1F8F
:10F534002498FF1F2C98FF1F2C98FF1F3498FF1F3F
:10F544003498FF1F3C98FF1F3C98FF1F4498FF1FEF
:10F554004498FF1F4C98FF1F4C98FF1F5498FF1F9F
:10F564005498FF1F5C98FF1F5C98FF1F6498FF1F4F
:10F574006498FF1F6C98FF1F6C98FF1F7498FF1FFF
:10F584007498FF1F7C98FF1F7C98FF1F8498FF1FAF
:10F594008498FF1F8C98FF1F8C98FF1F9498FF1F5F
:10F5A4009498FF1F9C98FF1F9C98FF1FA498FF1F0F
:10F5B400A498FF1FAC98FF1FAC98FF1FB498FF1FBF
:10F5C400B498FF1FBC98FF1FBC98FF1FC498FF1F6F
:10F5D400C498FF1FCC98FF1FCC98FF1FD498FF1F1F
:10F5E400D498FF1FDC98FF1FDC98FF1FE498FF1FCF
:10F5F400E498FF1FEC98FF1FEC98FF1FF498FF1F7F
:10F60400F498FF1FFC98FF1FFC98FF1F0499FF1F2D
:0CF614000499FF1F00000200FFFFFFFF31
:00000001FF
